:100000000C94870E0C94AF0E0C94AF0E0C94AF0EA4
:100010000C94AF0E0C94AF0E0C94AF0E0C94AF0E6C
:100020000C94AF0E0C94AF0E0C94AF0E0C94836B2B
:100030000C94196F0C94B06B0C94AF0E0C94D118F7
:100040000C94BF180C94AF0E0C944D740C94B772B2
:100050000C94AF0E0C94AF0E0C94AF0E0C94AF0E2C
:100060000C94D96E0C942F190C941B6C0C94E86CA6
:100070000C94AF0E0C94AF0E0C94AF0E0C94AF0E0C
:100080000C94AF0E0C94AF0E0C94AF0ED970DD70C3
:10009000E570EF700671207135714471597170719E
:1000A0007A7198719E71A371A971AF7109721372FF
:1000B000B871BE71C471CD71D171D671DE71F0713C
:1000C000F671FC710172E170E171E671EB715370D0
:1000D0006C617368008040000000000000000000B8
:1000E0000000000000000000000000000000000010
:1000F0000000000000000000000000000000000000
:1001000000000000000000000000000000000000EF
:1001100000000000000000000000000000000000DF
:10012000000080C0E0E0F0F8F8FCFCFCF8F8F8F023
:1001300040000000000080808000000000000000FF
:1001400000000000000000000000000080C0C0E0CF
:10015000E0E0F0F0F0E0C00000000000C0F8FFFFB9
:100160009F8783838383838383838383838383833F
:1001700083838383838383830383808383838383D2
:10018000838383838383838383838383838383833F
:100190008383C3E3733F1F0000000080E0F0F8FC9E
:1001A000FEFFFFFFFF7F3F1F1F0F0783C3E1E1E05B
:1001B000E0C0000E1F3F7F7FFFF3E0E08000000003
:1001C0000000000000000080F0FCFEFFFFFFFF7F4A
:1001D0003F0F0301010100000080F0FEFFFFC7C1D7
:1001E000C1C1C1C1C1C1C1C1C1C1C1C1C1C1C1C1FF
:1001F000C1C1C1C1C101C1F0FEFF3F0F070F0D0D0D
:100200000D1D191919193131313171616161E1C166
:10021000C1C18100000080E0F8FCFFFFFFFF2F1745
:100220000F038180C0E0F0F8FCFEFFFFFFFFFFFF3F
:100230007F010000000000000001010307070E1EFF
:100240001C3870E0F0F8FEFFFF7F1F0F0300010075
:10025000000000000000000000000000000000009E
:10026000000000000000000000000000000000008E
:10027000000000000000000000000000000000007E
:10028000000000000000000000000000000000006E
:1002900000000000007EFFFFFFFFFFFFFBF8FCFCFB
:1002A000FEFF7F3F1F0F07C3FFFFFFFFFFFF7F071B
:1002B0000000000000000000000000000000C0E09E
:1002C000F8FEFFFF7F1F0F1F3D7CF8F8F0E0800075
:1002D000000000000000000000000000000000001E
:1002E000000000000000000000000000000000000E
:1002F00000000000000000000000000000000000FE
:1003000000000000000000000000000000000000ED
:1003100000000000000000010101010103070707C0
:100320000301000000E0FCFFFFFFFFFF1F030000D0
:10033000000000000000000000C0F078DE27130974
:100340000E0703000000000000000001030F7FFF04
:10035000FC7878F800000000000000000000008039
:10036000808080808080808000808000808000008D
:1003700000000000008080808080808080808080FD
:1003800080808080808080000000000000000000ED
:10039000000000000000000000000000000000005D
:1003A000000080F0FEFFFFFFFF3F0F010000000094
:1003B00000000000C0E0381E0F0300010000000034
:1003C000000000000000000000000000000000002D
:1003D0000000030301000000000000000000000E08
:1003E0000E02020202020303000F0F000F0F0808A3
:1003F00008080808080F0F08080808080F0F000071
:1004000000000F0F000000000000000000000000CE
:1004100000000000000000000000000000000000DC
:10042000C0F8BFFFFFFF1F7F0100000000000000B9
:1004300000F0FCFF7F7830000000000000000000AA
:1004400000000000000000000000000000000000AC
:10045000000000000000000000000000000000009C
:10046000000000000000000000000000000000008C
:10047000000000000000000000000000000000007C
:10048000000000000000000000000000000000006C
:100490000000000000000000000000000000301C10
:1004A000070E0F0701000000000000000000000020
:1004B000000000000000000000000000000000003C
:1004C000000000000000000000000000000000002C
:1004D00000000000000000001B1E272D36394B4E87
:1004E000636C7278878D939CB1B4C6C9D2D8E1E4AD
:1004F00001020304010302040402030104030201D4
:1005000003010200040506076D656E75537461638F
:100510006B206F766572666C6F77006D656E7553D4
:100520007461636B20756E646572666C6F770070C2
:100530007265737320616E79204B657900414C457B
:100540005254004D455353414745004C4F41444997
:100550004E47002020202020202020202020202066
:1005600020202020202020202000506C6561736511
:1005700020526573657420537769746368657300EE
:100580005377697463686573205761726E696E672B
:1005900000204F6C642056657273696F6E2045456C
:1005A00050524F4D202020434845434B2053455443
:1005B00054494E47532F43414C494200416C6172AC
:1005C0006D732044697361626C6564005265736584
:1005D00074207468726F74746C65005468726F7400
:1005E000746C65206E6F742069646C650050726570
:1005F000737320616E79206B657920746F20736B43
:10060000697000414C45525400454550524F4D20B1
:100610006C6F77206D656D004F46464142535255D1
:1006200073525525454C73454C2554487354482501
:10063000414C73414C2550312050312550322050CF
:1006400032255033205033250054485252554445EA
:100650004C4549443049443149443241494C47456D
:100660004154524E535731535732535733535734E3
:1006700053573553573653573753573853573953C2
:100680005741535742535743004F4646004F4E2061
:10069000002D2D2D004348002D2D2D2000525544B6
:1006A00020454C45205448522041494C20005031AF
:1006B000202050322020503320204D4158204655D4
:1006C0004C4C4359433143594332435943335050BF
:1006D0004D3150504D3250504D3350504D3450509C
:1006E0004D3550504D3650504D3750504D38434891
:1006F0003120434832204348332043483420434884
:100700003520434836204348372043483820434863
:10071000392043483130434831314348313243482E
:10072000313343483134434831354348313641440D
:10073000312041443220002D2D2D2D00564552539D
:100740003A2056312E353439372D6572657A00449A
:100750004154453A2031312E30322E323031320080
:1007600054494D453A2031303A31303A3237002041
:1007700053564E3A20657239782D72373038002042
:100780004D4F443A204652534B59204E4854202056
:100790000012081200081C0808081C0800000822A3
:1007A00000490022080000000000227F2200000013
:1007B00008220049002208000008220049002208FF
:1007C000000000227F2200000000000822004900F3
:1007D00022080000081C0808081C0800D7356C4ACD
:1007E0005B3043298C5B6E58A04F4E51AB21882063
:1007F000F351DE1EFE233424D4244F264E4F2044D2
:100800004154410054783D0052783D0041203D0064
:1008100056343D0756353D0E56363D0056313D07A0
:1008200056323D0E56333D005370643D096B747370
:10083000204D61783D00416C743D004C6F6E3D0071
:100840004C61743D0054783D0052783D0041323D8A
:100850000041313D00416C743D0052504D3D00540B
:10086000323D0054313D0054783D0052783D004601
:1008700075656C3D0041203D0054546D0045787015
:10088000457846466E654D656443727300544F5417
:100890000053544B1153542500544D451154535794
:1008A0000053544154005B4D454E555D20746F20FC
:1008B0007265667265736800537461636B0F6200E2
:1008C000746D61696E0F6D7300746D7231204A69C9
:1008D000747465720F757300746D72314C6174209D
:1008E0006D696E0F757300746D72314C6174206D9B
:1008F00061780F7573005354415432004D6F646535
:10090000005761726E31205761726E322043686504
:1009100061702052696E67202053636946692052D6
:100920006F626F7420436869727020546164612043
:1009300020437269636B74536972656E20416C6DFC
:10094000436C6B5261746174615469636B2020481D
:1009500061707463314861707463324861707463AC
:100960003300416C657274205B5265645D00416CBC
:10097000657274205B4F72675D00416C6572742014
:100980005B59656C5D00496E742E204672736B79FD
:1009900020616C61726D0042616E6447617000504D
:1009A0006F745363726F6C6C00416C61726D205791
:1009B00061726E696E67004D656D6F727920576167
:1009C000726E696E670054524530313241470054AF
:1009D000524530313241470044656661756C742080
:1009E000537700537769746368205761726E696E3C
:1009F00067005468726F74746C65205761726E6919
:100A00006E670053706C617368204E616D650053B2
:100A1000706C6173682073637265656E004F464643
:100A2000004C69676874206F6E2053746B204D769C
:100A3000004C69676874206F666620616674657231
:100A4000004C696768742073776974636800466C4A
:100A5000617368206F6E2062656570004265657025
:100A600020636F756E74646F776E004D696E757478
:100A7000652062656570005468726F74746C6520DF
:100A8000726576657273650053494E474F534D50FA
:100A900046494C540046696C7465722041444300D9
:100AA000496E616374697669747920616C61726DF5
:100AB0000042617474657279207761726E696E6745
:100AC00000436F6E7472617374004861707469637F
:100AD00020537472656E67746800537065616B654E
:100AE0007220506974636800426565706572506970
:100AF00053706B7200536F756E64204D6F646500A8
:100B00005175696574204E6F4B6579207853686F15
:100B1000727453686F7274204E6F726D20204C6F28
:100B20006E672020784C6F6E6720004265657065A7
:100B300072004F776E6572204E616D6500524144C0
:100B4000494F2053455455500043616C004D756C1E
:100B50007469706C696572006368316368326368D8
:100B600033636834006F6666202B3D203A3D006D8C
:100B70006F64650A25207372632020737700536CBD
:100B800061766500545241494E455200000303030B
:100B9000030056455253494F4E005472696D2D2043
:100BA0002B00204D656E75204578697420446F7761
:100BB0006E20202055705269676874204C656674F9
:100BC000004449414700424700414E41005B4D45CA
:100BD0004E555D205748454E20444F4E45004D4FE1
:100BE000564520535449434B532F504F54530053B1
:100BF0004554204D4944504F494E54005B4D454E9D
:100C0000555D20544F205354415254005354415287
:100C1000542043414C4942524154494F4E004341B4
:100C20004C4942524154494F4E0066726565004D31
:100C30004F44454C53454C0044454C455445204D8C
:100C40004F44454C0F5B4D454E555D005432546842
:100C50005472696700547261696E657200452E2096
:100C60004C696D69747300504F534E45470053688B
:100C70006966742053656C004C50342F4C503520FD
:100C80002044534D326F6E6C792044534D322F44C3
:100C9000534D580044534D20547970650053656E90
:100CA00064205278204E756D626572205B4D454E12
:100CB000555D0050504D2046724C656E0D6D53656C
:100CC00063002052784E756D003443482036434807
:100CD000203843482031304348313243483134438F
:100CE00048313643480075530075536563005050D2
:100CF0004D20202050585820202044534D32202091
:100D000050504D3136200050726F746F0052455470
:100D100041313233004265657020436E7400547275
:100D2000696D20537700457870202020457846690A
:100D30006E6546696E6520204D656469756D436F0B
:100D400061727365005472696D20496E6300542DA1
:100D50004578706F00542D5472696D00436F756E45
:100D60007420446F776E436F756E74205570202029
:100D70000054696D6572200054726967676572007E
:100D800054696D6572004E616D6500534554555050
:100D90000000090100000000000006020044757018
:100DA0006C69636174696E67206D6F64656C005B6C
:100DB0004D454E555D20205B455849545D005945D1
:100DC000530B4E4F0044454C455445204D4F444530
:100DD0004C004455504C4943415445204D4F4445E7
:100DE0004C00204142434445464748494A4B4C4DFC
:100DF0004E4F505152535455565758595A61626389
:100E00006465666768696A6B6C6D6E6F707172732A
:100E10007475767778797A303132333435363738BD
:100E2000395F2D2E006578702020252020737731C2
:100E300020737732004558504F2F4452000003442E
:100E4000522048696768004452204C6F7700445232
:100E5000204D6964004472537732004472537731F5
:100E600000576569676874004578706F0045585091
:100E70004F2F445200002B2A52004D495845520032
:100E80005072657373205B455849545D20746F2020
:100E900061626F7274004D6178206D69786572735C
:100EA0002072656163683A200044454C45544520F2
:100EB0004D4958205B4D454E555D00536C6F772072
:100EC00020557000536C6F772020446F776E00447C
:100ED000656C61792055700044656C617920446FC0
:100EE000776E0041646420202020204D756C746969
:100EF000706C795265706C61636520004D756C741F
:100F00007078004F4646005761726E696E670053F5
:100F1000776974636800437572766573004F4E207D
:100F20004F4646005472696D004F46464F4E2000B2
:100F3000466C4D6F64657472696D004F66667365CB
:100F40007400466D5472696D56616C00576569672F
:100F5000687400536F757263650045444954204DB1
:100F600049582000494E53455254204D49582000BD
:100F70002D2D2D2D202020763E6F66732020763C6F
:100F80006F667320207C767C3E6F66737C767C3C3B
:100F90006F6673414E44202020204F522020202095
:100FA00020584F522020202076313D3D7632207649
:100FB00031213D76322076313E7632202076313C2A
:100FC0007632202076313E3D76322076313C3D76B9
:100FD000322000535700435553544F4D2053574927
:100FE0005443484553000002534146455459205349
:100FF00057495443484553000002566F6C742054BF
:10100000687265733D004F464631323234303000ED
:10101000416C74416C61726D002D2D2D59656C4FC2
:10102000726752656400547852535349616C726D13
:101030000054454C454D45545259320000010100C1
:101040003C3E002D2D2D59656C4F72675265640032
:10105000616C726D00762D564100412020636861FD
:101060006E6E656C004D6574496D70004672487512
:101070006257534868690055737250726F746F00FD
:1010800054454C454D45545259000001010202019E
:1010900002434F5059205452494D205B4D454E5507
:1010A0005D002D2D2D494E56004C494D495453009D
:1010B0000003030303030303030303030303030303
:1010C0000300435600435552564553005052455372
:1010D000455400454449542D3E0043555256450061
:1010E00009002D2D2D494E56004F46464F4E2000EB
:1010F0002D2D2D783E30783C307C787C663E3066F5
:101100003C307C667C63312063322063332063345F
:10111000206335206336206337206338206339200D
:10112000633130633131633132633133633134637E
:10113000313563313600454550524F4D206F76654D
:1011400072666C6F7700454550524F4D206F766543
:1011500072666C6F770067656E777269746520657B
:1011600072726F7200454550524F4D20466F726D3E
:10117000617474696E670042616420454570726FE6
:101180006D2044617461004D4F44454C2020202067
:1011900020004D45202020202020202000500850F5
:1011A00000000000000000006F00000700070014AE
:1011B0007F147F14242A7F2A12231308646236497D
:1011C0005522500005030000001C2241000041226E
:1011D0001C0014083E081408083E0808005030009F
:1011E00000080808080800606000002010080402D9
:1011F000003E49453E0000427F40006251494600A2
:1012000041494936001814127F0027454539003EF0
:10121000494932000179050300364949360006493B
:10122000291E000036360000005636000008142241
:101230004114141414144122140800020151090627
:1012400000060909067E0909097E7F494949363E9B
:10125000414141227F4141221C7F494949417F0947
:101260000909013E4149497A7F0808087F00417F0A
:1012700041002040413F017F081422417F4040400F
:10128000407F020C027F7F0408107F3E4141413EB7
:101290007F090909063E4151215E7F091929462629
:1012A0004949493201017F01013F4040403F1F2031
:1012B00040201F3F4030403F63140814630708700C
:1012C00008076151494543007F414100020408106D
:1012D000200041417F0004020102044040404040A0
:1012E000000102040020545454787F4844443838A4
:1012F00044444420384444487F3854545418087EA9
:101300000901020C5252523E7F0804047800447DC9
:1013100040002040443D007F1028440000417F40B1
:10132000007C041804787C08040478384444443869
:101330007C14141408081414187C7C08040408484D
:1013400054545420043F4440203C4040207C1C2006
:1013500040201C3C4020403C44281028440C505065
:10136000503C4464544C44000836410000007F0067
:101370000000413608000808221C08081C22080842
:10138000A0608000000000000000000000000000DD
:1013900000FFFF0000000000001F3F00003F1F0093
:1013A000003030FFFF3030FFFF30303078CCCCFFE2
:1013B000FFCCCC8C0C060F0F86C0E070381C0C3CA8
:1013C000FEC7E3F33B1E0C00000000333B1F0F0081
:1013D0000000000000F0F81C0E07030000000003EE
:1013E000070E1CF8F000003030E0C0FCFCC0E0301C
:1013F00030C0C0C0C0FCFCC0C0C0C00000000000C5
:101400000000000000C0C0C0C0C0C0C0C0C0C0005C
:1014100000000000000000000000000080C0E0703C
:10142000381C0C000000000000000000000000005C
:10143000003838000000000000000000000000003C
:101440000003033F3F03033F3F03030C0C0C0C3F1F
:101450003F0C0C07030C0E07030100183C3C180F4F
:101460001F383133331E1E333300000000000000EC
:10147000000000000003070E1C38300000000030A0
:10148000381C0E07030000030301000F0F000103C7
:1014900003000000000F0F000000000000333B1F9E
:1014A0000F0000000000000000000000000000002D
:1014B00000183C3C18000000000C0E07030100005F
:1014C0000000000000FCFE87C3E377FEFC00000C78
:1014D0000EFFFF0000000000000C0E0783C3E77E34
:1014E0003C00000303C3C3C3E7FE3C0000C0E07040
:1014F000381C0EFFFF00003F3F33333373E3C3005C
:1015000000FCFEC7C3C3C78E0C00000303C3E37314
:101510003B1F0F00003CFEE7C3C3E7FE3C00003C5E
:101520007EE7C3C3E7FEFC0000183C3C1800000047
:10153000000000183C3C18000000000000C0E0F073
:10154000381C0E070330303030303030303030034C
:10155000070E1C38F0E0C000000C0E07030383C325
:10156000E77E3C00000F1F3B3130381F0F0000307A
:10157000303F3F3030000000003C3E3733313030E8
:101580003000003030303030391F0F0000030303CB
:101590000303033F3F00000C1C383030381F0F009E
:1015A000000F1F383030391F0F000000003F3F0090
:1015B00000000000000F1F393030391F0F000000FD
:1015C0000030381C0E07030000060F0F0600000055
:1015D000000000333B1F0F0000000000000001036B
:1015E000070E1C3830030303030303030303033014
:1015F000381C0E0703010000000000000033330117
:1016000000000000003C7EE7C3C3E77E3CF0F8DC4E
:10161000CEC7C7CEDCF8F0FFFFC3C3C3C3C3E7FE2A
:101620003CFCFE0703030303070E0CFFFF03030349
:10163000070E1CF8F0FFFFC3C3C3C3C3C30303FFFC
:10164000FFC3C3C3C3C3C30303FCFE0703C3C3C3B6
:10165000C7CECCFFFFC0C0C0C0C0C0FFFF000003AA
:1016600003FFFF03030000000000000303FFFF036C
:1016700003FFFFC0E0F0381C0E0703FFFF0000006F
:101680000000000000FFFF0E1CF8F81C0EFFFFFF1B
:10169000FF3870E0C08000FFFFFCFE070303030378
:1016A00007FEFC000000000000000000003F3F00BB
:1016B00000000000003F3F3F3F3030303030391FE6
:1016C0000F0F1F3830303030381C0C3F3F30303077
:1016D000381C0E07033F3F30303030303030303F61
:1016E0003F00000000000000000F1F383030303095
:1016F000303F3F3F3F0000000000003F3F00003010
:10170000303F3F303000000C1C383030381F0F00A5
:10171000003F3F000103070E1C38303F3F303030A0
:1017200030303030303F3F0000000000003F3F3F8E
:101730003F0000000103033F3F0F1F3830303030BF
:10174000381F0FFFFFC3C3C3C3C3E77E3CFCFE07C4
:101750000303030307FEFCFFFFC3C3C3C3C3E77E4A
:101760003C3C7EE7C3C3C3C3C78E0C03030303FF24
:10177000FF03030303FFFF000000000000FFFFFF63
:10178000FF000000000000FFFFFFFF00000000005E
:1017900000FFFF0F1F38F0E0E0F0381F0F3F7FE041
:1017A000C08080C0E07F3F03030383C3E3733B1F1C
:1017B0000F0000FFFF0303030300000C1C3870E060
:1017C000C080000000000003030303FFFF0000309F
:1017D000381C0E07070E1C38300000000000000007
:1017E0000000003F3F00000000000000000F1F3815
:1017F0003033371E1C3F333F3F000003070E1C38B9
:10180000300C1C3830303030391F0F000000003FE2
:101810003F000000000F1F3830303030381F0F03FA
:10182000070E1C38381C0E07030F1F38381F1F38CF
:10183000381F0F3C3E0703010103073E3C00000038
:10184000013F3F010000003C3E3733313030303043
:101850003000003F3F30303030000000000000001A
:101860000103070E0C0000303030303F3F00000015
:101870000000000000000000003030303030303018
:10188000303030000003070E1C38300000000030FC
:101890003030303070E0C0FFFFC0E070303070E0BA
:1018A000C0C0E07030303030300000C0E070303008
:1018B00070E0C0FFFFC0E0703030303070E0C0C07A
:1018C000C0FCFEC7C303070E0CF0F89C0C0C0C0CFC
:1018D0000CFCFCFFFFC0E070303070E0C000003056
:1018E00030F3F300000000000000003030F3F3009C
:1018F00000FFFF0080C0E07030000000000303FF25
:10190000FF00000000F0F03070E0E07070E0C0F028
:10191000F0C0E070303070E0C0C0E0703030303087
:1019200070E0C0000000000000000000000C1E3F3E
:1019300033333333333F3F3F3F3030303030381F65
:101940000F0F1F3830303030381C0C0F1F3830303C
:101950003030303F3F0F1F3B33333333330303000B
:10196000003F3F00000000000000013333333333F9
:101970003B1F0F3F3F0000000000003F3F000030D2
:10198000303F3F303000000C1C383030381F0F0023
:10199000003F3F03070F1C38300000000030303F8D
:1019A0003F303000003F3F0000030300003F3F3F57
:1019B0003F0000000000003F3F0F1F383030303044
:1019C000381F0FF0F03030303030F0E0C0C0E0F0C1
:1019D000303030E0C0F0F0F0F0C0E070303070E057
:1019E000C0C0E0F0303030303000003030FFFF3029
:1019F0003000000000F0F0000000000000F0F0F007
:101A0000F0000000000000F0F0F0F0000000000026
:101A100000F0F03070E0C08080C0E07030F0F08006
:101A20000000000000F0F03030303030B0F0F070E6
:101A3000300000C0E03C3E0703000000000000FF53
:101A4000FF00000000000003073E3CE0C00000C0B3
:101A5000C0C0C00C1CF8F0E0C0C0E0F0F81C0CC026
:101A6000C0C0C03F3F0303030303030100000103A1
:101A700003030303033F3F3F3F000000000000005B
:101A800000303133333333333F1E0C00000F1F3827
:101A90003030381C0C0F1F383030381C0C3F3F03DF
:101AA000070E1C38381C0E07030F1F38381C1C3853
:101AB000381F0F30381C0F07070F1C383000013358
:101AC000333333333B1F0F30383C3E373331303004
:101AD00030000000010F1F38300000000000003F00
:101AE0003F00000000000030381F0F010000000020
:101AF0000000000C0E07030100000103070E0C009C
:101B0000000000408008042010020100008911122A
:101B1000239B322446AD573665BF74488CC19D5A0D
:101B2000AFD3BE6CCAE5DB7EE9F7F88110080193FC
:101B3000331A22A5562C47B7753E64C99C408DDBED
:101B4000BF52AEEDDA64CBFFF976E802218B30109C
:101B50000299132667AF763444BD554AADC3BC58CD
:101B60008ED19F6EEBE7FA7CC8F5D983310A2091BC
:101B7000121803A7772E66B5543C45CBBD42ACD9AD
:101B80009E508FEFFB66EAFDD874C904428D531650
:101B9000619F702004A9153227BB364CCEC5DF5E8D
:101BA000EDD7FC6888E1997AABF3BA85520C43977C
:101BB000711E60A1142805B3373A26CDDE44CFDF6D
:101BC000FD56ECE9986089FBBB72AA06638F72141C
:101BD000409D512225AB343006B9174EEFC7FE5C4D
:101BE000CCD5DD6AA9E3B8788AF19B87730E62953C
:101BF000501C41A3352A24B1163807CFFF46EEDD2D
:101C0000DC54CDEBB962A8F99A708B088481951ADF
:101C1000A793B62CC2A5D33EE1B7F04008C919522C
:101C20002BDB3A644EED5F766DFF7C899400859BDB
:101C3000B712A6ADD224C3BFF136E0C1184809D30C
:101C40003B5A2AE55E6C4FF77D7E6C0AA583B4187B
:101C50008691972EE3A7F23CC0B5D14229CB3850EC
:101C60000AD91B666FEF7E744CFD5D8BB502A4999B
:101C7000961087AFF326E2BDD034C1C3394A28D1CC
:101C80001A580BE77F6E6EF55C7C4D0CC685D71E2F
:101C9000E597F42880A1913AA3B3B2444ACD5B56AC
:101CA00069DF78600CE91D722FFB3E8DD604C79F5B
:101CB000F516E4A9902081BBB332A2C55A4C4BD78C
:101CC000795E68E11C680DF33F7A2E0EE787F61CFB
:101CD000C495D52AA1A3B03882B193466BCF7A546C
:101CE00048DD59622DEB3C700EF91F8FF706E69D1B
:101CF000D414C5ABB122A0B9923083C77B4E6AD54C
:101D0000585C49E33D6A2CF11E780F004E1B1124EC
:101D10001FBECFEFD0E1DEBFCDBF11E0A0E0B1E04C
:101D2000E2E8FDEE02C005900D92AA32B107D9F7A4
:101D30001FE0AAE2B1E001C01D92A033B107E1F7B4
:101D40001DE1CEE0DDE104C02297FE010E947A761B
:101D5000CC30D107C9F70E94791A0C94BF760C9445
:101D6000000030919D0422B780919D043817C9F777
:101D7000932F80E030E0282B392BC901089529E208
:101D8000820290011124359527953595279587FD79
:101D9000815C86FB880F880B80F9992787FD9095D9
:101DA000281B390BC9010895F8942091CC0D30916E
:101DB000CD0D7894C9010895482F50E09A01220F63
:101DC000331F63E0440F551F6A95E1F7240F351F59
:101DD0002C553E4FC901089590E09C01220F331FFE
:101DE000220F331F280F391F2C513D4FC901089571
:101DF000AF92BF92CF92DF92EF92FF920F931F9319
:101E0000CF93DF93C82E162FEA01F22ED02E57FF64
:101E100010C022FF02C08CE101C08FE09C2D981BF6
:101E2000892F612F4DE22F2D0E94F263D095C1952D
:101E3000DF4F2D2D2F218C2D612F4AE30E94F2635D
:101E40008F2D90E0B4E0AB2EB12CA822B922F2FE87
:101E500002C0E2E001C0E0E0CE016CE370E00E946D
:101E600028769B01442737FD4095542F0F2D0061A4
:101E70008E2F8C0D612FA2E0EA2E0E94F265A11434
:101E8000B10411F0ECE101C0E1E1CE016CE370E0DE
:101E90000E9428769C01442737FD4095542F0D2D34
:101EA00000618E2F8C0D612FF2E0EF2E0E94F26503
:101EB000DF91CF911F910F91FF90EF90DF90CF9026
:101EC000BF90AF9008950F931F93062F122F20629B
:101ED00050E00E94286717FD07C080919E0D602F7B
:101EE00046E7212F0E94F2631F910F910895242F3E
:101EF000409108010E94630F08950F93022F44231D
:101F000019F447E357E020C04530A8F4E0916E0192
:101F1000F0E0EE0FFF1FEE0FFF1F3197E40FF11DF2
:101F2000E051FB4F449150E0440F551F440F551FA3
:101F30004756594F09C0473250F450E0440F551FDF
:101F4000440F551F4656594F24E00E94B5640F9127
:101F50000895FF920F931F93182FF62E022F4423FC
:101F600021F448E956E024E00EC08A5E4A3008F4C5
:101F700085506F2D50E0202F0E942867812F6F2DF4
:101F800045E956E022E00E94B5641F910F91FF9051
:101F900008950F931F93DF93CF9300D0CDB7DEB793
:101FA000382F162F942F022F442329F0463139F071
:101FB0004A3E81F408C08A5F41E956E007C08A5F63
:101FC0004DE856E003C08A5F49E856E0202F0E94A2
:101FD000E56428C04095441F4427441F81E2841BC8
:101FE000482F832F39839A830E94F2633981832F8C
:101FF0008A5F9A81E92FFF27E7FDF095F7FF03C07D
:10200000F095E195FF4FFF27E7FDF0953197AF0180
:10201000440F551F4E0F5F1F475B594F612F23E041
:102020000E94B5640F900F90CF91DF911F910F9197
:10203000089589E496E00895DF92EF92FF920F935E
:102040001F93D82EE62EF42E10919501E12FFF2735
:10205000E7FDF095F7FF03C0F095E195FF4FE03104
:10206000A4F483E0E802F0011124E85EF94F8D2D1D
:102070006E2DAF0123E00F2D0E94B5641F3F3CF58C
:102080008D2D86506E2D41E21FC08D2D8650E5327C
:1020900064F411161CF4412F4F5002C0412F415FD0
:1020A0006E2D2F2D0E94C90F12C011161CF4412F46
:1020B000445202C0412F4C5D6E2D2F2D0E94C90F3E
:1020C0008D2D8E5E6E2D4DE62F2D0E94F2631F9199
:1020D0000F91FF90EF90DF900895CF92DF92EF92F3
:1020E000FF920F931F93CF93DF93F82ED62EE22FFC
:1020F000102F242F30E040E050E0F0E0DF01AA0F85
:10210000BB1FAA0FBB1FA65DBB4F0C910295069586
:1021100006950370CC24C394023009F0CC24EE2041
:1021200071F1EE0FFF1FEE0FFF1FE95DFB4F808186
:10213000C82FD0E0CC2011F0CC0FDD1FBE0180E015
:1021400090E00E94E975033051F1C436D10580F466
:102150009B01AC01CA01B901660F771F881F991F47
:1021600023E330E040E050E00E943B7610631FC064
:102170002FEF30E040E050E00E943B7618C0CC20CA
:1021800021F0220F331F441F551F033081F4CA0171
:10219000B9012FEF30E040E050E00E94E97524E6FD
:1021A00030E040E050E00E943B76106202C0002325
:1021B00011F0CC2091F0012F00628F2D6D2D75E074
:1021C000E72E0E94F26517FD0EC080919E0D6D2DC9
:1021D00046E7212F0E94F26306C08F2D6D2DA901C5
:1021E000212F0E942867DF91CF911F910F91FF90BF
:1021F000EF90DF90CF9008958C3038F4E82FF0E026
:10220000EE0FFF1FE952FB4F2AC0803198F4E82FF0
:10221000F0E0DF01AA0FBB1FAC58BB4FEE0FFF1F52
:10222000EC5BFE4F2D913C91119780819181281B91
:10223000390B0AC0843158F4E82FF0E0EE0FFF1F8D
:10224000EC58FB4F20813181220F331F1AC084329A
:1022500048F4E82FF0E0EE0FFF1FE354FB4F20811E
:1022600031810FC0863258F4E82FF0E0EE0FFF1FE7
:10227000EE0FFF1FE75FF14F208130E002C020E04A
:1022800030E0C9010895AF92BF92CF92DF92EF92F2
:10229000FF920F931F93DF93CF930F92CDB7DEB7CB
:1022A000F82EE42E463008F0EAC0882309F4EAC08C
:1022B000863119F08A3E19F4E2C061E0E3C0992743
:1022C00087FD90959C0197FF04C022273327281B88
:1022D000390B2A307CF41F144CF02DE030E0A901BA
:1022E000481B590BCA010E949268C6C00D960E94F5
:1022F0009268C7C02A50A22EBB249501220F331F1B
:102300002A0D3B1D26573E4FF901E85AFD4F4081EB
:10231000442309F4B4C05E2D553029F4F501E85981
:10232000FB4F8081A7C0F901EA5AFD4FC080295AAE
:102330003D4FF901D080453008F4B1C04830C8F0B5
:102340008C2D815049830E94FC108C018D2D815071
:102350000E94FC100BC02D2D332727FD30952358EC
:102360003F4F0BC08D2D49830E94BF0E9C014981B8
:1023700004C020E030E000E010E0483088F4453050
:1023800080F5423009F460C0433020F4413009F058
:102390006CC055C04330C9F0443009F066C01BC062
:1023A0004A3009F44CC04B3030F44830F1F1493038
:1023B00009F05BC03FC04C3009F44BC04C3008F40E
:1023C00043C04D3009F051C049C017FF38C01095C7
:1023D00001951F4F34C017FF37C0109501951F4F4F
:1023E00033C0E3948C2D60E04E2D0E944311082FE2
:1023F0008D2D60E04E2D0E944311F501EE0FFF1F61
:10240000EA0DFB1DEE51FC4F9081953029F400231D
:1024100061F1882341F52AC0963029F4002319F58B
:10242000882319F120C0802721C081E002171307FB
:10243000E1F41CC081E002171307C1F416C081E06B
:10244000201731079CF011C081E00217130774F0C8
:102450000CC081E0021713074CF407C081E020177D
:10246000310724F402C081E001C080E0F501E859A1
:10247000FB4F80831F142CF061E0682703C060E0ED
:1024800001C0682F862F0F90CF91DF911F910F9180
:10249000FF90EF90DF90CF90BF90AF9008958C2D7C
:1024A000815049830E94FC108C014981FC2DF5323A
:1024B0000CF051CF57CF86B380958E7708950E9448
:1024C0005B128823E1F70E940168089580915B0107
:1024D00060E040E00E944311882331F4809185043C
:1024E00090918604009711F0C79A0895C7980895AF
:1024F0000F931F93CF93DF93EC018B010E948863AE
:1025000082E260E043E056E024E00E94E56480E27D
:10251000BE010E940C6588E2B8010E940C6580E350
:102520006DEE75E00E940C650E94926780915801E3
:102530000E9488670E945F12DF91CF911F910F91D7
:1025400008950F93AB0160E123E000E00E94B564C1
:102550000F910895DF92EF92FF920F931F93CF9305
:10256000DF9380916D0181FD83C080E895E06AE68C
:1025700075E00E94781290918501892F887341F04F
:10258000883131F0883221F0803311F0883329F41A
:10259000892F877C88608093850100E010E085E1C9
:1025A000E82EF12C08C0C701801B91090E94926897
:1025B000110F182B0F5F0830B0F3D0908501D12692
:1025C00080E060E143E555E026E100E00E94B5646B
:1025D000CD2DD0E0CE0180FF05C082E069E476E039
:1025E0000E94A112C1FF05C087E16CE476E00E9461
:1025F000A112C2FF05C08CE26FE476E00E94A11236
:10260000CE01887390700097B1F0012F13FF05C0C1
:1026100081E462E576E00E94A11204FF05C081E436
:1026200065E576E00E94A11205FF05C081E468E53A
:1026300076E00E94A112C6FF05C086E56BE576E054
:102640000E94A112D7FE05C08BE66EE576E00E94DF
:10265000A1120E94926780918501181749F00E948B
:102660005B12882329F40E94661200E010E09BCFE1
:10267000DF91CF911F910F91FF90EF90DF90089520
:102680001F93CF93DF930E945B1220E030E011E0B4
:10269000482F50E02F5F3F4FBA01022E02C07595C0
:1026A00067950A94E2F760FD03C01F5F183091F749
:1026B0001150163030F5812F0E94FC5D882309F1FE
:1026C00010935701812F0E94005E81E00E94D65E28
:1026D0000E94886386E160E04BE455E024E00E94BC
:1026E000E564CAE8D1E01AE04991812F68E124E06D
:1026F0000E94F263155F1837B9F70E9492670E9433
:102700005F12DF91CF911F910895CF93DF93EC017A
:102710000E94886382E260E043E455E024E00E9486
:10272000E56488E1BE010E940C650E949267809179
:1027300058010E948867DF91CF9108951F93CF932E
:10274000DF93EC01162F0E94886382E260E04DE384
:1027500055E024E00E94E56488E1BE010E940C651A
:102760008CE168E34FE255E00E9414650E94926795
:10277000112319F48091580101C089E10E948867F2
:1027800082E10E942D720E945F120E945B128823D8
:10279000C9F48091600E833019F4A8951092600EF0
:1027A00080915B0160E040E00E944311882331F496
:1027B00080917201882311F4112311F0C79AE5CF9B
:1027C000C798E3CFDF91CF911F910895809167045F
:1027D000882351F081E995E060E00E949E1380918A
:1027E00067048E7F80936704089580916D0187FD53
:1027F00007C0887329F48CEB95E060E00E949E137B
:10280000089580916D0182FD0AC00E94F75F883CA7
:10281000910528F489E096E060E00E949E130895F7
:10282000EF92FF92CF93DF93A82FAF70A6509091B5
:102830009C01923074F0292F332727FD30952150C9
:102840003040C1E0D0E002C0CC0FDD1F2A95E2F796
:102850009C2FA83008F09CC06A2F659570E0FB01A2
:10286000EE0FFF1FE050FF4F0190F081E02DB0818F
:10287000992379F4CB2FDD27C7FDD095D7FF03C06F
:10288000D095C195DF4F9C2FC7FD9D5F9595959580
:102890009F5F40916E0150E04170507022E030E047
:1028A000241B350B2617370769F420919B012F70E5
:1028B00009F473C021E094E03091700130FF03C04F
:1028C000919501C020E04B2F552747FD5095C92F0A
:1028D000DD27C7FDD095A0FF03C0C40FD51F04C0DE
:1028E000BA016C1B7D0BEB01209729F07E019F2D17
:1028F0009B2797FF0BC0222349F4BB2339F010829A
:102900000E94F16886E10E942D7241C0CE01845878
:102910009F4F893F9105B8F4C08386E00E94D65E40
:10292000CE0183589F4F8B3F910588F5D7FF03C099
:10293000D095C195DF4FD595C795D595C795BE0163
:10294000645C462F1FC01C161D0614F48DE701C0E1
:1029500083E8808386E00E94D65ECE0183589F4F35
:102960008B3F9105A0F4CE01D7FF03C090958195D0
:102970009F4F64E070E00E942876709561957F4FCC
:10298000462F445C8FE294E065E10E94BA7080E0DB
:10299000DF91CF91FF90EF90089520E08DCF8F923F
:1029A0009F92AF92BF92CF92DF92EF92FF920F93DE
:1029B0001F93CF93DF93182FEB015A016901802EEB
:1029C00084FF06C01F70106654E0952E05E003C01A
:1029D00045E0942E04E0802F8066181761F0802F68
:1029E0008064181741F080910605882369F013363A
:1029F00011F0133449F47E010894E11CF11C83E1C9
:102A00000E942D72892D18C0992D9066191761F0BA
:102A1000992D9064191741F0882309F474C0123677
:102A200019F0123409F06FC07E010894E108F10832
:102A300084E10E942D72802F90E00E94926888238A
:102A400051F0EE24FF24EC1AFD0A892D0E94F16852
:102A5000802F0E94F168A114B10491F481E0C8169E
:102A6000D10471F4103661F41092060531E0E32EC2
:102A7000F12C209711F0EE24FF2480E60E94F168EB
:102A80002091820430918304E21AF30ACE14DF0409
:102A900044F4812F0E94F16883E10E942D72760137
:102AA0000AC0EA14FB043CF4812F0E94F16884E11F
:102AB0000E942D727501EC16FD06A9F0E114F104D7
:102AC00051F4812F0E94E268D7FF02C083E101C068
:102AD00084E10E942D72882D83700E94D65E81E071
:102AE00080937F0402C010927F04C701DF91CF91D1
:102AF0001F910F91FF90EF90DF90CF90BF90AF901C
:102B00009F908F9008957E01A6CF0F93772767FD42
:102B10007095552747FD5095332727FD30950E9426
:102B2000CF140F9108950F93772767FD7095552760
:102B300047FD5095332727FD309502E00E94CF14C2
:102B40000F9108950F93772767FD7095552747FDDF
:102B50005095332727FD309501E00E94CF140F9147
:102B60000895E0917E04F0E0EE0FFF1FEA58FB4F5E
:102B700080819181089590917E04992319F488238E
:102B800031F418C0882319F4892F815001C080E0E6
:102B900080937E0487E10E942D72E0917E04F0E034
:102BA000EE0FFF1FEC58FB4F0190F081E02D8EEBF4
:102BB000099508958BE195E060E00E949E130895C9
:102BC000FC01A0917E04B0E0AA0FBB1FAC58BB4F24
:102BD000ED93FC938FEB099587E10E942D72089588
:102BE000CF93DF93EC0180917E04982F9F5F9093A9
:102BF0007E04953040F080937E0488E095E060E0AC
:102C00000E949E130FC087E10E942D72E0917E0406
:102C1000F0E0EE0FFF1FEC58FB4FD183C0838FEB2A
:102C2000FE010995DF91CF9108958FE294E00E9413
:102C3000B96F882311F084E105C080919E04882338
:102C400021F0815080939E0407C09091630081E041
:102C500091FF80E080939F0480919F0408951092DB
:102C6000890410928B0410928A04109288040895AB
:102C700020918504309186042115310531F02150D1
:102C800030403093860420938504882369F0409176
:102C9000720150E084EF91E0489F9001499F300D10
:102CA000589F300D112402C020E030E0809187044D
:102CB000882369F060917A0170E044EF51E0649FED
:102CC000C001659F900D749F900D112402C080E09B
:102CD00090E040918504509186044217530720F4F8
:102CE00030938604209385042091850430918604D6
:102CF0002817390720F490938604809385040E9456
:102D000066120895E82FF0E0E050FB4FE491F0E008
:102D1000EE0FFF1FEE55FB4F20813181C901089551
:102D2000CF92DF92EF92FF920F931F93DF93CF9397
:102D30000F92CDB7DEB720E0CC24DD24822F29838B
:102D40000E948216092F10E0C00ED11E29812F5F2C
:102D50002430A1F7C6010F90CF91DF911F910F9101
:102D6000FF90EF90DF90CF9008951F930E94D40EB4
:102D700041E02091D5043091D6048217930709F4DD
:102D800040E0409384040E94D40E9093D604809334
:102D9000D5048BE095E060E00E94193A80918404AC
:102DA000882309F4CBC08091880480FF14C08091EF
:102DB0008904982F9F5F90938904943660F083561E
:102DC0008093890480918A0490918B04019690935A
:102DD0008B0480938A0480E00E94E45E0E948863F2
:102DE0000E9404680E941014182F0E943816209127
:102DF000E3043091E4048091800490918104821B6B
:102E0000930B60E270E00E942876709383046093D5
:102E100082046115710591F08091D3049091D404DE
:102E2000821B930B62E070E00E942876709383040B
:102E30006093820430938104209380043093D404FF
:102E40002093D3048091700185FF04C01092830405
:102E500010928204E0917E04F0E0EE0FFF1FEC5828
:102E6000FB4F0190F081E02D812F09950E94926720
:102E70000E941516882321F0809165008F7E03C083
:102E8000809165008061809365000E94D40E8F71EF
:102E900090708230910509F04FC087E00E94821641
:102EA0009C0164E0220F331F6A95E1F768E070E04F
:102EB0000E94287640915A01552747FD50954A5F58
:102EC0005F4F649FC001659F900D749F900D11240A
:102ED000820F931F2091700126FD05C060910901AA
:102EE00070910A0102C060EF70E02091080130E0AB
:102EF0002F5F3F4F0E941476260F371F3595279579
:102F0000209308018091D204805E8093D2048823AC
:102F100099F480915901281778F4223368F081E1FF
:102F20000E942D728091700183FF06C082E390E0C1
:102F30009093860480938504109287041F910895CE
:102F4000A2EAB4E0E2EBF4E060E0862F806487B9A7
:102F5000369A408951898D919C91119796958795C4
:102F6000840F951F8E7F11969C938E9320813181C3
:102F7000C901840F951F96958795918B808B349B03
:102F8000FECF349A84B195B1820F931F96958795A1
:102F9000819391936F5F12966830B9F60895EF921E
:102FA000FF920F931F93CF93DF938091700184FD65
:102FB00044C00E9466120E94886380E060E045ED94
:102FC00050E020E000E00E9493638091760184FD50
:102FD00008C080E068E34BE751E02AE000E10E948E
:102FE000B5640E949267809158010E9488670E9490
:102FF0005F1200E20E94A0170150E1F70E949016B4
:103000008C010E94D40EEC01C057DE4F0DC00E940F
:10301000A0170E9490167C010E945B12882369F41D
:10302000E016F10651F406C00E94D40EC817D90765
:1030300071F703C00E946612F7CFDF91CF911F9105
:103040000F91FF90EF900895E2EAF4E040E012C0A3
:1030500067B9369A349BFECF349A24B135B1820FCA
:10306000931F5150A9F796958795819391934F5F40
:10307000483031F054E080E090E0642F6064E8CFA5
:103080000895E2EAF4E020E0822F806487B9369A5E
:10309000349BFECF349A84B195B1880F991F8193E8
:1030A00091932F5F283081F70895FF920F931F931C
:1030B000CF93DF9380916D0180FD3AC080916E01C6
:1030C00090E08170907002E010E0081B190BF8018D
:1030D000EE0FFF1FE65DFE4FC181D28160968785AE
:1030E0009089C81BD90B0E944118F02E802F0E9496
:1030F0008216C817D907E4F40E945B128823C1F432
:103100000DC00E9441188F2D0E948216C817D90742
:103110007CF40E945B12882341F00AC08BED95E09D
:103120006CEC75E00E947812ECCF0E946612E9CF39
:10313000DF91CF911F910F91FF9008958EE587B990
:10314000369A349BFECF349A84B195B1049640915F
:10315000090150910A019A0163E0220F331F6A9519
:10316000E1F7241B350B820F931F23E0969587957B
:103170002A95E1F790930A018093090108957894C4
:103180001F920F920FB60F9211248F9380919D047E
:103190008F5F80939D048F910F900FBE0F901F90B3
:1031A000189578941F920F920FB60F9211242F93B7
:1031B0003F934F935F936F937F938F939F93AF93BF
:1031C000BF93EF93FF93F89487B78D7F87BF789471
:1031D00081B78E5F81BF9091310480913304882341
:1031E00079F080917901882349F0813051F4809100
:1031F0002F0F890F80932F0F87FF02C01B9A01C0EA
:103200001B9880910B01982F915090930B0188236C
:1032100081F48DE480930B018FE294E00E94CD6FE6
:103220000E9402690E940A758091600E82608093FC
:10323000600EF89487B7826087BF7894FF91EF9112
:10324000BF91AF919F918F917F916F915F914F91BE
:103250003F912F910F900FBE0F901F90189578946B
:103260001F920F920FB60F9211241F932F933F932B
:103270004F935F936F937F938F939F93AF93BF937E
:10328000EF93FF932091800030918100F89480911A
:103290007D008F7D80937D0078948091A004909133
:1032A000A104A901481B590BCA0196958795309333
:1032B000A1042093A00410919C04212F21502830B8
:1032C00058F59C012152334055E02737350708F562
:1032D000E12FF0E0EE0FFF1FE657FB4FAC014C5D16
:1032E000554020917401332727FD3095265F3F4FCD
:1032F000429FC001439F900D529F900D11246AE0A0
:1033000070E00E942876718360831F5F10939C0495
:103310000CC010929C0409C0815A9F402EE28F3D40
:10332000920718F481E080939C04F89480917D00CA
:10333000806280937D007894FF91EF91BF91AF916F
:103340009F918F917F916F915F914F913F912F91BD
:103350001F910F900FBE0F901F901895E1E3FFE0B3
:103360009F0181918535E1F320533F40C9010895C4
:10337000EF92FF920F931F93CF93DF930E94B10EB2
:10338000EC0180917101813019F40E94A01707C0EF
:10339000823019F40E94241802C00E9441188EE560
:1033A00087B90E94B5160E949E188091600E8330E6
:1033B00019F4A8951092600E0E94B10E8C1B9D0B03
:1033C0002091AD063091AE062817390720F490936E
:1033D000AE068093AD068091980E882309F482C0D2
:1033E0001092980E8091970E882399F18091960102
:1033F000829586958695837090E00097C1F0823023
:10340000910519F420E931E002C02AE730E080910B
:10341000AF069091B0064091E90E5091EA0E840FEC
:10342000951F281739071CF481E00E942D72209106
:10343000280F90910404ECE1FFE080E008C0319196
:10344000391720F48DE10E942D7203C08F5F82171F
:10345000B0F38091960E882309F444C080E060E0C8
:103460000E94E3728C018330910539F180E061E0C4
:103470000E94E372EC018330910521F181E060E06C
:103480000E94E3727C018330910511F181E061E0DB
:103490000E94E3728330910509F10230110569F051
:1034A000C230D10579F022E0E216F10489F08230D1
:1034B0009105A1F00130110511F480E00AC0C1307E
:1034C000D10511F480E00BC021E0E216F10419F4FB
:1034D00081E060E005C08130910521F481E061E088
:1034E0000E943973DF91CF911F910F91FF90EF9060
:1034F00008951F938FEF8ABB1BBA91E897BB9EE795
:1035000098BB9EE394BB91EC95BB11BA82BB88E05B
:1035100082B987EF83B9109261001092620084E152
:10352000809364008BEF809365000E9452670E9435
:10353000D77480E487B985E886B987E083BF8CE9D2
:1035400081BF87B7836087BF1FBC8AE08EBD1092A2
:103550008B0082E880938A0080917D008062809356
:103560007D00EDB7FEB7329785E502C080833197C5
:103570009FE0E033F90709F0C8F7789487EF93E408
:10358000909375048093740489E10E9488670E9477
:103590008F5E109157010E944013809158010E9444
:1035A00088675091720140917A01451778F4652F30
:1035B00070E024EF31E0629FC001639F900D729F25
:1035C000900D11249093860480938504541770F411
:1035D00050E024EF31E0429FC001439F900D529F85
:1035E000900D112490938604809385040E946612A6
:1035F00080917901813039F48091700184FD03C09C
:1036000087E00E942D720E94CF170E9401140E9431
:1036100041180E9455180E94AA120E94F5130E9498
:10362000E6130E945F1280EF90E090930A0180936E
:1036300009010E94246E2DE088E190E00FB6F89415
:10364000A89581BD0FBE21BD8BE095E060E00E9492
:10365000193A87ED95E30E94F01581E00E94BB15B1
:10366000809158010E94886780915701181729F0AE
:1036700081E00E94D65E0E94725F80912A0F806472
:1036800080932A0F80ED97E09BBD8ABD80E186BFC5
:1036900087B7806187BF0E94B819FDCF8FE294E0A1
:1036A0000E94B66F089529E2820290011124359597
:1036B00027953595279587FD815C86FB880F880BBC
:1036C00080F9992787FD9095281B390BC90108952A
:1036D0009C01E5E035952795EA95E1F7AC01440FAB
:1036E000452F441F550B280F391F892F990F990B10
:1036F0008595280F391F241B350BC9010895F894AF
:103700002091CC0D3091CD0D7894C9010895AC0174
:1037100080E060E021E00E94E56408950F931F932C
:10372000CF93DF93182F81EA98E00E94871B113610
:1037300058F0133628F0133639F489E29CE102C0C0
:1037400087EF93E40E94E01586E068E049E958E0DD
:103750000E94146540912506509126068AE268E091
:1037600020E000E00E94F80E4091270650912806C4
:103770008EE468E020E00E94F80E86E060E141E916
:1037800058E00E9414654091290650912A068AE269
:1037900060E120E00E94F80E40912B0650912C062B
:1037A000F4E056954795FA95E1F78EE460E120E064
:1037B0000E94F80E86E660E04DE858E00E9414652D
:1037C00040912306509124068EE460E020E00E94A0
:1037D000F80E8091A9069091AA068937910528F0E4
:1037E0008091A806C82FD0E002C0C0E0D0E082E0FF
:1037F0006CE34EE70E94926585E06CE143E20E9433
:1038000096651BE0812F6BE343E00E9496651A5F8B
:103810001338C1F716E00CE3FE01E05DF94F40817B
:10382000602F641B812F0E9496652196C837D105B1
:1038300010F0C0E0D0E02091A80630E0C217D30716
:1038400019F01F5F1E3741F7DF91CF911F910F9144
:1038500008951F93182F86EF98E00E94871B123659
:10386000E1F0133628F4103631F01136E9F418C0BF
:103870001336D1F415C08FEF97E090930D0180932C
:103880000C011092AC061092AB061092AE0610928C
:10389000AD0687E10E942D7207C08EE89BE102C051
:1038A00087EF93E40E94E01588E067EE78E00E94DD
:1038B0000C654091AB065091AC065695479584E552
:1038C00068E00E94386780E168ED78E00E940C654E
:1038D00040910C0150910D015695479584E560E1AA
:1038E0000E94386788E169EC78E00E940C6540919D
:1038F000AB065091AC0680910C0190910D01481BD4
:10390000590B5695479584E568E10E94386780E237
:1039100060EC78E00E940C652091AD063091AE0617
:1039200084E690E0289FA001299F500D389F500DFC
:103930001124A4E056954795AA95E1F784E560E245
:1039400020E30E94286788E268EB78E00E940C651B
:103950000E94AE19AC018FE368E20E94186582E113
:1039600068E346EA58E00E9414651F91089580EFCD
:1039700090E108950F9393E0499FA00111244751CE
:103980005F4E01E0222309F400E023E00E94B564C9
:103990000F9108950F9393E0499FA00111244E5178
:1039A0005F4E01E0222309F400E023E00E94B564A9
:1039B0000F910895FF920F931F93F82E062F142F47
:1039C00080E860E0402F50E0212F0E9428670A30F5
:1039D00010F00FE601C005E7802F60E04FE2212FD5
:1039E0000E94F2634F2D50E04F5F5F4F802F60E0E9
:1039F000212F0E9428671F910F91FF9008956F92C9
:103A00007F928F929F92AF92CF92DF92EF92FF922E
:103A10000F931F93CF93DF93EC01162FD42E490100
:103A20006090DF047090E0048091BD089091BE0822
:103A30008619970920E430E0B9010E942876462FC4
:103A400060930905E091E104F091E2048091BB08E4
:103A50009091BC088E1B9F0BB9010E942876862F7F
:103A600060930A05442321F07092BE086092BD085D
:103A7000882321F0F093BC08E093BB0880910805EF
:103A8000882321F48091700185FF06C010920905FA
:103A900010920A051092080560910905662351F4F9
:103AA00080910A05882331F48091820490918304E7
:103AB000009781F04091720150E024EF31E0429F85
:103AC000C001439F900D529F900D11249093860446
:103AD000809385048114910409F456C08881882359
:103AE00009F04BC0662331F180910605882311F55A
:103AF000ED2DE61BE7FDE0E0202F30E08E2F99272B
:103B000087FD90958217930714F0E02FE150FF276F
:103B1000E7FDF0958D2D90E0E817F90749F0EE0FDD
:103B2000FF1FE80DF91D25913491C9010E94E01590
:103B300010920905153641F4DD2011F0ED2D01C07C
:103B4000E02FF0E031970FC01436C9F42D2D30E08E
:103B5000802F90E00197281739071CF4ED2DEF5FB7
:103B600001C0E0E0F0E0EE0FFF1FE80DF91D259128
:103B70003491C9010E94E01502C040E001C041E05B
:103B80008D2D602F0E94DA1CE114F10451F0988110
:103B90008C2D9C1508F4892FF701E80FF11D549125
:103BA00001C050E080910605882309F04FC0809144
:103BB0000A05882329F14881481B47FD40E0242F4E
:103BC000332727FD30958A2D90E0281739070CF010
:103BD0004A2D48838981E114F10459F0C41608F490
:103BE0004C2DF701E40FF11DE4918E1718F4E82F26
:103BF00001C0E0E0E98380E68093CE0D10920A05D3
:103C00008881882319F1909109059923F9F0498158
:103C1000E114F104B1F0491B47FD40E09C2D8C15E7
:103C200008F4982FF701E90FF11DE491242F3327B1
:103C300027FD30958E2F90E0281739071CF04E2F66
:103C400001C040E0498380E68093CE0D103651F1EB
:103C5000113690F4133409F480C0143430F4113266
:103C600079F1123409F09CC06AC0143409F43FC0E1
:103C7000153409F095C04FC01436E9F1153638F403
:103C8000123609F45FC0133609F08AC069C01138D2
:103C9000A1F01F3B21F0153609F082C040C0198207
:103CA000188212C0552309F47BC081E0909106056B
:103CB000911180E08093060573C0109206050DC037
:103CC00080910605882319F01092060569C0888145
:103CD000882319F08114910421F480E00E94BB151F
:103CE0005FC087E10E942D721982188256C08981B7
:103CF000851709F455C0E114F10409F451C080910D
:103D00000605882309F04CC08981851710F48F5F60
:103D100012C0198242C08981882309F441C0E1148C
:103D2000F10409F43DC0809106058823C9F5898115
:103D3000882319F08150898330C059832EC088812F
:103D40008A1571F180910605882351F588818A15BD
:103D500010F48F5F0DC018820EC08881882301F196
:103D6000809106058823E1F48881882319F0815029
:103D7000888301C0A8828981E114F10461F09881EF
:103D80009C1508F4C92EEC0CF11CF70194918917CD
:103D900018F4982F01C090E0998380E68093CE0DAF
:103DA000DF91CF911F910F91FF90EF90DF90CF9017
:103DB000AF909F908F907F906F9008954F925F92F9
:103DC0006F927F928F929F92AF92BF92CF92DF922B
:103DD000EF92FF920F931F93DF93CF930F92CDB784
:103DE000DEB7D82E84E89BE00E94871B8FE398E023
:103DF0006D2D41E020EF37E006E05CE8E52E5BE06A
:103E0000F52E15E0C12EB6E0AB2E0E94FF1C80906F
:103E10003F08909040088091630081FF07C08AE2CC
:103E200068E14EE75BE00E94146560C182E168E0F2
:103E30004FE65BE00E9414658A9480910605882312
:103E400019F0A2E0CA2E02C0CC24C394EE24FF24B1
:103E500010E1A82CBB24A7FCB094F4E06F2E712CC9
:103E60002701440C551C84E691E0480E591E4E2D46
:103E70004F5F80E0612F20E00E947D0FAE14BF04F1
:103E800011F491E0911090E0F201218122952695A4
:103E90002695237030E0A901440F551F420F531F90
:103EA0004B59544F992311F400E001C00C2D88E1C7
:103EB000612F23E099830E94B56499819923C1F011
:103EC000809106058823A1F0F201618162956695D3
:103ED000669563708D2D40E022E00E94A2158295C8
:103EE000880F880F807CF20191819F73982B9183BA
:103EF000AE14BF0421F401E0F92DF13009F000E027
:103F0000F2018181880F880F85958595FDE08F02EC
:103F1000C0011124B3010E942876AB01002311F4E3
:103F200020E001C02C2D82E4612F0E94286700232D
:103F3000A9F080910605882389F0F2016181660F5E
:103F4000660F659565958D2D41EE2FE10E94A215B6
:103F50008F73F2019181907C982B9183AE14BF04F2
:103F600021F491E0F92DF23009F090E0F201208186
:103F7000277030E0A901440F551F420F531F485AC4
:103F8000544F992311F400E001C00C2D88E4612FF7
:103F900023E099830E94B5649981992391F08091DF
:103FA0000605882371F0F201608167708D2D40E075
:103FB00023E00E94A2158770F2019081987F982BD0
:103FC0009083AE14BF0421F401E0F92DF33009F021
:103FD00000E0F2014081459545954595002311F497
:103FE00020E001C02C2D8AE5612F0E94C90F00231B
:103FF000B1F080910605882391F0F201608165950A
:10400000659565958D2D4AEE26E10E94A215880FD3
:10401000880F880FF20190819770982B9083185F1A
:104020000894E11CF11C103309F01ACF80E36DE411
:104030007BE00E940C6540917401552747FD509527
:10404000465F5F4FF82DF43011F421E201C020E209
:104050008EE460E30E942867282D243049F48D2DDA
:104060006091740146EF28E20E94A21580937401CA
:10407000EE24E394882D853009F0EE2480E068E397
:1040800049E45BE02E2D0E94E5644CE8A42E44E058
:10409000B42E0CE511E090E3F501419151915F01DF
:1040A000F801219131918F01421B530B440F551F91
:1040B000892F68E320E299830E9428679981985E9E
:1040C000903951F7EE2091F0FD2DF03679F4ACE502
:1040D000B1E0ECE8F4E088E001900D928150E1F766
:1040E00081E00E94D65E87E10E942D720F90CF91F1
:1040F000DF911F910F91FF90EF90DF90CF90BF90D5
:10410000AF909F908F907F906F905F904F900895A9
:104110006F927F928F929F92AF92BF92CF92DF92D7
:10412000EF92FF920F931F93CF93DF93B82E81E30B
:1041300090E10E94871B80EA98E06B2D49E02CED0E
:1041400037E00AE0ECE3EE2EE0E1FE2E73E0C72E4E
:1041500054E0A52E0E94FF1CF090A0089090A108AA
:104160008B2D8252843048F480910605882329F0F3
:1041700080912A0F806380932A0F809106058823FF
:1041800019F012E0A12E02C0AA24A394C7EBDEE02E
:10419000B5EBCB2EBEE0DB2E6624772410E1812F19
:1041A00066E270E10E940C65862D813031F480E07A
:1041B000612F42E520E00E94F2630894611C711CAB
:1041C0004881E3E04E9FA0011124475E5F4E862C9C
:1041D000F61411F4992011F000E001C00A2D82E4D8
:1041E000612F23E00E94B564F601208130E040E0B9
:1041F00050E0F81419F4F92DF13011F000E001C08D
:104200000A2D86E6612FA3E0EA2E0E94F265F814DB
:1042100031F580910605882331F4809182049091D4
:1042200083040097E1F0992021F0892D8130B9F4C1
:1042300009C08B2D688140E023E002E00E948515D3
:1042400088830DC0F60160818B2D70E040E050E066
:1042500028E730E002E00E94CF14F6018083219627
:104260000894C11CD11C183111F0185F98CF88E256
:1042700060E170E10E940C658091960182958695BF
:104280008695837090E0AC01440F551F480F591F6D
:104290004A5F5F4EFF2DF33011F000E001C00A2DA0
:1042A00082E468E223E00E94B5648F2D8330C9F474
:1042B0006091960162956695669563708B2D70E0AE
:1042C00040E050E022E030E002E00E94CF1482950E
:1042D000880F880F807C909196019F73982B909304
:1042E000960180E36AEF7FE00E940C652091040450
:1042F00030E0220F331F442737FD4095542FEF2D18
:10430000E43019F40A2D006301C000E384E560E3A2
:1043100074E0E72E0E94F265FF2DF43069F460919D
:1043200004048B2D70E040E050E022ED30E002E02C
:104330000E94CF1480930404DF91CF911F910F91BD
:10434000FF90EF90DF90CF90BF90AF909F908F90B5
:104350007F906F9008952F923F924F925F926F924D
:104360007F928F929F92AF92BF92CF92DF92EF9205
:10437000FF920F931F93DF93CF93CDB7DEB72997AB
:104380000FB6F894DEBF0FBECDBF982E80E890E147
:104390000E94871B82EA98E0692D48E02CED37E007
:1043A0000AE0EAE8EE2EE0E1FE2E76E0C72E57E0C6
:1043B000A52E0E94FF1CF090A2081091A308892D41
:1043C0008252843030F480910605882311F00E94D7
:1043D000B87580910605882319F042E0242E02C0AA
:1043E0002224239488E067E770E10E940C65909195
:1043F0009601969596959695937045E0949FA001A9
:10440000112444595F4E2F2D213011F401E0111178
:1044100000E08CE368E025E09F830E94B5649F8103
:104420008F2D8130B1F41123A1F4809106058823EA
:1044300081F0892D692F40E021E00E94931583705F
:10444000880F880F880F90919601977E982B9093F4
:1044500096019091960192959695917043E0949F64
:10446000A00111244B595F4EEF2DE13019F401E00A
:10447000113009F000E080E668E023E09F830E94AD
:10448000B5649F81FF2DF130B1F41130A1F480911A
:104490000605882381F0892D692F40E021E00E94E4
:1044A000931581708295880F807E909196019F7DF3
:1044B000982B9093960187E294E09A838983CC2489
:1044C000DD2432E0332E20E1822E922D90689E83EF
:1044D000882D6AE570E10E940C65CB824C2D4F5C03
:1044E00086E0682D0E94B164E981FA814081F3146D
:1044F00021F4112311F40E8101C000E880E6682D3B
:104500002B81EE240E946D10F601EE0FFF1FEE0FBF
:10451000FF1FE65DFB4F40814295469546954370EF
:1045200050E04B5A5F4EF31411F4113011F000E0DB
:1045300001C0022D80E6682D21E00E94B564F314CD
:10454000E1F580910605882331F4809182049091F1
:104550008304009791F1112319F0113071F510C007
:10456000E981FA816081892D70E040E050E02FEF11
:1045700030E002E00E94CF14E981FA8180831DC0FF
:104580005601AA0CBB1CAA0CBB1C8AE294E0A80E24
:10459000B91EF50160816295669566956370892DF7
:1045A00040E023E00E9493158295880F880F807C5D
:1045B000F50190819F73982B9083532C539408E0BE
:1045C000402E480C5601AA0CBB1CAA0CBB1C88E24E
:1045D00094E0A80EB91E66247724F601EE0FFF1FA3
:1045E000EE0FFF1FE65DFB4FF987E887E885F98549
:1045F0004081242F2F7030E0C301880F991F02C023
:10460000359527958A95E2F7F22FF370FC83842F76
:104610008295837090E0062C02C0959587950A9448
:10462000E2F7282F21702D8384E0642D40E550E1CE
:1046300020E00E94E5648C8193E0899FA001112411
:104640004D5B5F4EF51411F4112311F000E001C031
:10465000022D84E2642D23E00E94B564ED814E2F8B
:1046600050E0405C5F4EF51411F4113011F000E0A1
:1046700001C0022D82E4642D21E00E94B564F501A1
:104680004081F51421F4123011F40E8101C000E8CC
:1046900080E6642D2B81EE24E3940E946D10F514C6
:1046A00009F064C080910605882339F48091820462
:1046B00090918304009709F459C0113019F1113019
:1046C00020F0123009F052C044C0892D6C8140E0C6
:1046D00023E002E00E948515E885F98520816114B8
:1046E000710431F0982F990F990F2370922B03C00A
:1046F000922F9C70982B9F70E885F9858081807F30
:10470000892B33C0892D6D8140E023E002E00E94B7
:104710008515E885F985208122952370611471043F
:1047200029F0982F990F2D7F922B03C0922F9E7FF7
:10473000982B93709295907FE885F98580818F7C86
:10474000892B808380917F04882381F00E94B87533
:104750000DC0F5016081892D70E040E050E02FEF41
:1047600030E002E00E94CF14F50180835394F8E01A
:104770004F0E0894611C711C0894A11CB11C22E00E
:104780006216710409F032CF83E0380E98E1890E89
:104790000894C11CD11CE981FA813496FA83E9831B
:1047A000F82DF03409F094CE29960FB6F894DEBFB8
:1047B0000FBECDBFCF91DF911F910F91FF90EF9072
:1047C000DF90CF90BF90AF909F908F907F906F9031
:1047D0005F904F903F902F900895AF92CF92EF92BD
:1047E000FF920F93AE2CEE24FF24CC240E94FF1CDA
:1047F0000F91FF90EF90CF90AF900895EF920F93AD
:10480000DF93CF930F92CDB7DEB7682F82E99BE09D
:1048100069830E94871B81E498E0698142E020EF70
:1048200037E006E0EE240E94ED2380E16FE677E0BA
:104830000E940C6588E16CE377E00E940C6580E2E1
:104840006FE477E00E940C6588E260E677E00E9402
:104850000C6580E36FE777E00E940C650F90CF91C5
:10486000DF910F91EF900895CF92DF92EF92FF9238
:104870000F931F93DF93CF9300D0CDB7DEB7682F90
:1048800081EC9BE069830E94871B83E498E0698147
:1048900043E020EF37E006E0EE240E94ED23BEE087
:1048A000CB2ED12C00E010E0143020F0A8EFFA2E2F
:1048B000F00E01C0F02EC6010E949268E82E1F5F24
:1048C0008AE26F2D412F20E00E94C90F4E2D405DDE
:1048D00084E46F2D2E2D0E94F263085F0894C11CA2
:1048E000D11C193009F708E3CC24DD2410E0812F16
:1048F00090E00E949268F82EA6014E55544F80E039
:10490000602F25E00E94DF644F2D405D80E2602F24
:104910002F2D0E94F2631F5F85E090E0C80ED91E24
:104920000850163021F784E568E14AE95BE027E0AA
:104930000E94DF64F6E0EF2EF12C10E230E084E517
:10494000612F41E957E0232F00E03A830E949363EF
:10495000C7010E949268282FC701019629830E94EF
:104960009268082F2981422F405D8CE6612F0E94BA
:10497000F263402F405D88E7612F202F0E94F26391
:104980003A813F5F185FE2E0F0E0EE0EFF1E343048
:10499000B1F60F900F90CF91DF911F910F91FF9083
:1049A000EF90DF90CF9008958F929F92AF92BF9239
:1049B000DF92EF92FF920F931F93CF93DF93D82E46
:1049C00089EC9BE00E94871B85E498E06D2D44E014
:1049D00020EF37E006E0EE24E3940E94ED23F09010
:1049E0004508C7EDD4E010E000E0812C84E0982E6B
:1049F000A12CB12C88E1612F41E40E94B164402FC9
:104A00004F5C8EE1612F0E94B164802F0E9482165C
:104A1000AC018AE2612F0E9418650730B1F068810D
:104A20007981882777FD8095982F24E630E040E053
:104A300050E00E94E975A50194010E945D768AE527
:104A4000612FA9010E9438670AC08F2D813011F0B3
:104A500040E201C041E28AE5612F0E94770F0F5FBB
:104A6000185F2296083031F68CE668E246EC5BE08F
:104A700022E00E94DF644091090150910A0188E719
:104A800060E320E00E9428678F2D813059F4F09276
:104A900008058D2D60915A0141E82FE70E94A2156B
:104AA00080935A01DF91CF911F910F91FF90EF906A
:104AB000DF90BF90AF909F908F900895EF920F93EB
:104AC000E42E40E020E030E000E00E94ED230F9172
:104AD000EF900895AF92BF92CF92DF92EF92FF9244
:104AE0000F931F93DF93CF9300D0CDB7DEB78FE145
:104AF00061E247E10E9496658FE167E347E10E942A
:104B0000926585E361E247E10E9496658FE161E28B
:104B100047E10E9492658BE461E247E10E9496655D
:104B20008BE467E347E10E94926581E661E247E139
:104B30000E9496658BE461E247E10E9492658AE2F9
:104B40006BE243E00E94966589E26CE243E00E94DA
:104B5000926586E56BE243E00E94966585E56CE22E
:104B600043E00E9492658091D7049091D80471E748
:104B7000C72ED12CB6010E942876262F8091D90409
:104B80009091DA040FE81FEFB8010E942876362FC3
:104B900068E2E62EE20E5AE2F52EF30E8E2D6F2D10
:104BA00045E02A8339830E9496653981632F625DCF
:104BB0008E2D45E00E9492652A81822F845D6F2DA3
:104BC00045E00E9496658E2D6F2D45E00E9492650E
:104BD0008091DD049091DE04B6010E942876262F94
:104BE0008091DB049091DC04B8010E942876062FA6
:104BF00044E5F42EF20E162F165D8F2D612F45E041
:104C00002A830E949665602F625D8F2D45E00E9489
:104C100092652A81822F885A612F45E00E9496650D
:104C20008F2D612F45E00E9492653FEDA32E34E069
:104C3000B32E2AE3F22E0DE510E098E3E92EF501FC
:104C4000819191915F0180509C4FB8010E9428761C
:104C5000D62ED394CE2CCD188F2D6C2D4D2D0E9499
:104C600096658F2D8F5F6C2D4D2D0E9496658F2D33
:104C70008E5F6C2D4D2D0E949665F5E0FF0E8F2DF9
:104C80008934E9F60F900F90CF91DF911F910F912A
:104C9000FF90EF90DF90CF90BF90AF9008954F922C
:104CA0005F926F927F928F929F92AF92BF92CF92BC
:104CB000DF92EF92FF920F931F93DF93CF930F92A8
:104CC000CDB7DEB7B82E8EE19CE00E94871B82E74D
:104CD00098E06B2D45E020EF37E006E0EE24E3940A
:104CE0000E94ED231092720836E5E32E38E0F32E91
:104CF00028E4C22E28E0D22E8601470160E0862FEC
:104D000069830E948216D4014D915C911197282FDE
:104D1000392F6981421753070CF49A01F40121934A
:104D200031934F01D8014D915C911197282F392F64
:104D3000241735070CF49A01F801219331938F0160
:104D40006F5F6730E1F68091470880930805FB2D7F
:104D5000F03219F0FF3B71F40BC08F5F809347086E
:104D6000833041F487E10E942D7281E00E94D65E7B
:104D700010924708809147088130B1F0813020F0CF
:104D8000823009F0A4C03FC08CE060E14CE05CE000
:104D900021E100E00E94B56482E168E14CEF5BE054
:104DA0002FE00E94B56493C08EE160E14FEE5BE0BE
:104DB0002CE000E00E94B56482E168E14DEC5BE02C
:104DC00020E10E94B56494E6892E98E0992E20E0B7
:104DD00008E91AE388E6A82E85ECB82ED7010D93D2
:104DE0001D937D01F601A192B1926F01822F29835B
:104DF0000E948216D4018D939D934D0129812F5FCE
:104E0000273061F764C082E160E14EED5BE020E1B4
:104E100000E00E94B56482E168E14DEC5BE020E1D6
:104E20000E94B56414E6A12E18E0B12EBBE24B2E11
:104E3000B1E05B2EF201A0E48A2E912CD7018D9176
:104E40009D917D01D6016D907D906D019C0126198B
:104E5000370937FF03C0309521953F4F2333310584
:104E6000DCF0D5012D913C91318320838901081B11
:104E7000190BC801B4010E942876061B170B17876F
:104E80000687C301821B930B9C01B4010E94287604
:104E9000261B370B358F248FA2E0B0E0AA0EBB1E75
:104EA0003296B4E6EB16B8E0FB0641F680E090E0FF
:104EB000F201219131912F01820F931FF3E44F16DC
:104EC000F1E05F06A9F790935601809355010E9487
:104ED0006A250F90CF91DF911F910F91FF90EF9076
:104EE000DF90CF90BF90AF909F908F907F906F900A
:104EF0005F904F900895282F30E0C901880F991FC7
:104F0000A90163E0440F551F6A95E1F7840F951FCF
:104F1000A9014F5F5F4FBA01660F771FA3E0440FEF
:104F2000551FAA95E1F7640F751F6C557E4F2095AC
:104F30003095205E3F4FA901440F551FE3E0220F3B
:104F4000331FEA95E1F7420F531F8C559E4F0E9485
:104F50008D768AE0EAEDF2E0DF011D928A95E9F7AD
:104F600082E00E94D65E0E94725F08950F931F93A5
:104F7000CF93DF93282F30E0E901CC0FDD1FC9016B
:104F800013E0880F991F1A95E1F7C80FD91F8E01FA
:104F90000C551E4FA9014F5F5F4FCA01880F991F23
:104FA000A3E0440F551FAA95E1F7840F951F2095A4
:104FB0003095205E3F4FA901440F551FE3E0220FBB
:104FC000331FEA95E1F7420F531F8C559E4FB801EE
:104FD0000E948D768AE0D8011D928A95E9F780912A
:104FE0009408C657DE4F8A8F8B8F84E68C8F82E0C1
:104FF0000E94D65E0E94725FDF91CF911F910F9148
:105000000895FF920F931F9385EFEBE2F5E0DF0128
:105010001D928A95E9F780912006A4EAB1E050E05C
:1050200021E030E060E07C91772311F0472F01C050
:1050300040E1641738F5F22E032F162F1F5F802FE3
:1050400090E0FC01EE0FFF1FEE0FFF1FE80FF91FAE
:10505000E55DFA4F912F9F738081807C892B80645E
:105060008083F182F39453830F5F141738F3962FE4
:105070009095642F822F8F5F890F390F340F290F7E
:10508000240F840F772359F1832F90E0FC01EE0F5A
:10509000FF1FEE0FFF1FE80FF91FE55DFA4F4F737B
:1050A0008081807C5483842B8068808322832F5F5F
:1050B0001A968C911A97781719F41182138205C0E9
:1050C00021832F5F852F8F5F8383822F5F5F1A96E7
:1050D000503219F42093200604C03F5FA4CF809380
:1050E00020061F910F91FF900895E4EAF1E080E01F
:1050F00090819150903108F48F5F3A9692E0E43EAF
:10510000F907B1F708951F93182F80E166E97EE053
:105110000E940C650E947528482F88E760E150E0E6
:1051200020E00E94286780E260E87EE00E940C6533
:10513000113651F481E60E94F16881E00E94BB15AE
:1051400083E499E20E94F0151F9108950E9475284A
:10515000803230F083E898E20E94F01581E00895F3
:1051600080E00895EF92FF920F931F93DF93CF9308
:1051700000D0CDB7DEB7182F813208F07BC088236E
:1051800019F4442341F476C0803219F4442331F0F9
:1051900071C0442319F0012F0F5F02C0012F01508D
:1051A000812F4A8369830E94DC0E7C01802F0E943C
:1051B000DC0EFC01D7018C91982F91504A816981B6
:1051C000903108F057C02081213108F053C0662388
:1051D000A1F10E94A628882309F04CC0212F30E0BD
:1051E000A9014F5F5F4FCA01880F991F13E0440F59
:1051F000551F1A95E1F7840F951FB901660F771FA8
:10520000A901A3E0440F551FAA95E1F7640F751F8C
:105210006C557E4F20953095205E3F4FA901440F7D
:10522000551FE3E0220F331FEA95E1F7420F531FAA
:105230008C559E4F0E948D761DC0281759F044232F
:1052400031F08031B8F48F5FF701808313C0D7014C
:105250009C9310C0D701CF010A9604C020813C91D5
:1052600031932D93E817F907C9F782E00E94D65EC3
:105270000E94725F0F900F90CF91DF911F910F915D
:10528000FF90EF9008956F927F928F929F92AF92CE
:10529000BF92CF92DF92EF92FF920F931F93CF9323
:1052A000DF93182F8AE79EE00E94871BE09020067C
:1052B000EA9487E998E0612F43E02CED37E00AE0BB
:1052C0000E94ED23C0909708CC2011F4109296080C
:1052D0001236D9F1133670F41334A9F1143420F4D2
:1052E000123409F070C031C01036C1F0113609F027
:1052F0006AC045C0103809F452C0113820F4133682
:1053000009F061C020C01E3BB9F11F3B09F05BC032
:1053100081E080939508109296082EC01C143CF4EE
:1053200081E090919608911180E080939608809199
:1053300096088093950880919208882309F443C0C9
:105340001092960840C01092950880919608882384
:10535000D1F141E0123609F040E08091930860916C
:1053600095080E94B22880919508882319F0133679
:1053700009F4CA94109295080E94012824C08091D3
:105380009608882301F1809193080E947B27109250
:1053900096080E94012881E60E94F16814C01C143E
:1053A00094F480919208882341F00E94A6288823D3
:1053B00021F4809193080E94B6271092960885E404
:1053C00099E50E94F01538E0D32E77247A9423E6ED
:1053D000822E9924BB24BA9466246394E090050538
:1053E000E90CFF24F701EE0FFF1FEE0FFF1FEE0D7C
:1053F000FF1DE55DFA4F4081842F807C09F462C176
:1054000046FF06C04F7380E06D2D20E00E94A90F7B
:105410001C14E4F4E701CC0FDD1FCC0FDD1FCE0D13
:10542000DF1DC55DDA4F8981C81681F46D2D695F76
:1054300080E048E10E9492658B8180939308888187
:105440008F738093940860929208B92CF701EE0F45
:10545000FF1FEE0FFF1FEE0DFF1DE55DFA4F808170
:1054600087FF05C19481C92FDD27C7FDD095AA24E8
:10547000A3949281C912AA2486FD1FC0FE01EE0FDB
:10548000FF1FCE01A3E0880F991FAA95E1F7E80F4F
:10549000F91FE555FE4F40814695477050E04A5848
:1054A000514F80919608882311F400E001C00A2D25
:1054B00082E16D2D21E00E94B564FE01EE0FFF1F19
:1054C000CE0163E0880F991F6A95E1F7E80FF91F95
:1054D000E657FE4F448D552747FD50958DE26D2DC3
:1054E0002A2D0E94286780919608882311F420E0D5
:1054F00001C02A2D8DE26D2D45E20E94F263FE016E
:10550000EE0FFF1FCE0143E0880F991F4A95E1F788
:10551000E80FF91FE657FE4F438D809196088823C8
:1055200011F420E001C02A2D86E36D2D0E947D0F2D
:10553000FE01EE0FFF1FCE0123E0880F991F2A9571
:10554000E1F7E80FF91FE657FE4F458D442359F068
:1055500080919608882311F420E001C02A2D8EE462
:105560006D2D0E94C90FFE01EE0FFF1FCE01B3E0AB
:10557000880F991FBA95E1F7E80FF91FE657FE4F1C
:10558000468D442391F023E0429FA0011124405115
:105590005F4E80919608882311F400E001C00A2D27
:1055A00086E66D2D23E00E94B564FE01EE0FFF1F1D
:1055B000CE0173E0880F991F7A95E1F7E80FF91F84
:1055C000EC55FE4F21E08581882309F420E0FE019F
:1055D000EE0FFF1FCE0153E0880F991F5A95E1F798
:1055E000E80FF91FEC55FE4F8681882329F022230E
:1055F00009F498C04AE203C0222361F044E4809198
:105600000605882311F420E001C02A2D89E76D2DBD
:105610000E94F2638A2D813051F55E01AA0CBB1CF9
:1056200033E0CC0FDD1F3A95E1F7AC0EBD1EEAE882
:10563000F1E0AE0EBF1E812FF501648D43E82DE72A
:105640000E949315F501848FF701EE0FFF1FEE0FF7
:10565000FF1FEE0DFF1DE55DFA4F848180939308D7
:1056600080818F738093940810929208B92CF7016F
:10567000EE0FFF1FEE0FFF1FEE0DFF1DE55DFA4F52
:105680008181882331F088150CF4882E87150CF061
:10569000782EF701EE0FFF1FEE0FFF1FEE0DFF1D1F
:1056A000E55DFA4F8281882331F088150CF4882E4D
:1056B00087150CF0782E9394F8E0DF0E292D273013
:1056C00009F08CCECC20A1F08B2D8F3FF9F4C814BB
:1056D00064F48091050590E00197EFEF8F3F9E07FE
:1056E00011F480E090E0809305057C14ECF414C084
:1056F000FB2DFF3F59F48091050590E001972FEFB6
:105700008F3F920761F480E090E009C08B2D8630D6
:105710005CF0992D983040F0809105058F5F809363
:10572000050502C043E56BCFDF91CF911F910F912B
:10573000FF90EF90DF90CF90BF90AF909F908F90B1
:105740007F906F9008952F923F924F925F926F9249
:105750007F928F929F92AF92BF92CF92DF92EF9201
:10576000FF920F931F935C01CC24DD243B0188241E
:10577000992464E6262E312C412C512CC201B10112
:105780006619770988099909A60195010E94E975AA
:105790007B018C0182E390E0A0E0B0E0E80EF91E0E
:1057A0000A1F1B1FC601B5010E94E9750E94E97519
:1057B000BC0188279927A40193010E94E97544E060
:1057C00096958795779567954A95D1F7E60EF71EDA
:1057D000081F191FC801B701A20191010E943B7661
:1057E000C9011F910F91FF90EF90DF90CF90BF9074
:1057F000AF909F908F907F906F905F904F903F9071
:105800002F9008951F93CF93DF939C01611571052D
:1058100011F1132F111F1127111F19F03095219528
:105820003F4F77FF0EC0C0E0D4E0709561957F4F89
:10583000CE01821B930B0E94A32B9E01281B390BC8
:1058400005C0C9010E94A32B282F392F112319F05D
:10585000309521953F4FC901DF91CF911F91089558
:105860006F927F928F929F92AF92BF92CF92DF9270
:10587000EF92FF920F931F93DF93CF93CDB7DEB7D5
:10588000982E962F322F802F6E2D222359F04423ED
:1058900061F440918204509183044115510539F41B
:1058A00021E001C020E0FF2405C022E001C021E08A
:1058B000FF24F394332311F0911121E04A2D433654
:1058C00079F44C2D50E0440F551F8A0173E0000F0E
:1058D000111F7A95E1F7041B150B005C1C4F11C0DA
:1058E000FA2DF236D9F44C2D50E0440F551F8A01A1
:1058F00093E0000F111F9A95E1F7041B150B0F5B46
:105900001C4FF80140810E94C90FFF2009F463C0B9
:10591000F8016081892D4AEE26E159C06988772413
:10592000BB24882051F54C2D50E0440F551F6A01CF
:10593000B3E0CC0CDD1CBA95E1F7C41AD50AAA0C69
:10594000BB1CAA0CBB1CCA0CDB1CC60CD71C44E33A
:1059500053E0C40ED51EF6014081552747FD5095F2
:105960000E942867FF20B9F1F6016081892D4CE97A
:1059700024E60E949315F6012DC0DD24AA0CBB1C61
:10598000A601E3E0440F551FEA95E1F74C195D09C4
:10599000A40EB51EA80CB11CAA0CBB1CF301EA0D89
:1059A000FB1DEC5CFC4F4081552747FD50954C5941
:1059B0005F4F0E942867FF2071F08501060D171DBB
:1059C0000C5C1C4F892DF80160814CE920E00E949D
:1059D0009315F8018083CF91DF911F910F91FF9074
:1059E000EF90DF90CF90BF90AF909F908F907F907F
:1059F0006F9008952F923F924F925F926F927F9295
:105A00008F929F92AF92BF92CF92DF92EF92FF92CE
:105A10000F931F93DF93CF93CDB7DEB72A970FB6BF
:105A2000F894DEBF0FBECDBFD82E8DE69EE00E945B
:105A3000871B80E998E06D2D40E020E030E000E039
:105A400075E7E72E7EE0F72ECC2453E0A52E0E94CA
:105A5000FF1C409188084F5F80E360E020E00E94D7
:105A60007D0FF09090088091880890E0880F991F32
:105A7000FC0123E0EE0FFF1F2A95E1F7E81BF90B6D
:105A8000E05CFC4F808160E040E00E94431188238D
:105A9000C1F08091880890E0880F991FFC0113E005
:105AA000EE0FFF1F1A95E1F7E81BF90BEF5BFC4FB8
:105AB000808160E040E00E944311882321F411E0DE
:105AC00003C010E001C012E060918808462F50E04A
:105AD000FA01EE0FFF1FE952FB4F808191818A315D
:105AE00091051CF010928F0807C02FEF873E920798
:105AF0001CF481E080938F0820916E0130E02170CA
:105B0000307082E090E0821B930B8417950741F47C
:105B1000643030F480919B01807F11F010928F08E7
:105B200080E168E67EE00E940C650F92EDB7FEB75B
:105B3000319621E0F11020E080918F0880838D2D37
:105B400061E041E006E3A0E1EA2EC0908808A12EC2
:105B500088240E94302C0F9088E161E67EE00E944C
:105B60000C650F92EDB7FEB7319621E03F2D313035
:105B700009F020E080918F0880838D2D61E041E065
:105B800006E3F8E1EF2EC0908808A12E88248394C4
:105B90000E94302C0F9080E26BE57EE00E940C6545
:105BA0000F92EDB7FEB7319621E08F2D823009F0CC
:105BB00020E010828D2D61E041E00EE1E0E2EE2E6A
:105BC000C090880873E6A72E88240E94302C0F907E
:105BD00088E265E57EE00E940C650F92EDB7FEB7A6
:105BE000319621E09F2D933009F020E010828D2D19
:105BF00061E041E00EE158E2E52EC090880832E60F
:105C0000A32E88240E94302C0F90113019F01230EE
:105C100049F404C080E36EE47EE007C080E367E4FB
:105C20007EE003C080E36FE37EE00E940C6500919C
:105C30008808402F50E0812F90E0880F991F880F2F
:105C4000991FBA01660F771F9B01B3E0220F331F24
:105C5000BA95E1F7261B370B820F931F86579E4F8D
:105C6000FC01E655FE4FA081A983FC01E555FE4FDE
:105C7000B081BA83FC01E455FE4F9080E4E69E0EAD
:105C800083559E4FDC018C908E0E20916E0130E08A
:105C90002170307082E090E0821B930B841795078F
:105CA00009F062C0043008F05FC080919B01807FE2
:105CB00009F45AC0EE24FF24870120E030E0B981C6
:105CC0006B2E772467FC7094A1E24A2E512C292C6C
:105CD000332427FC3094F0E4CF2ED22ED801C70114
:105CE000B595A79597958795B30129873A870E941F
:105CF000022C880F991FB2010E942876629DC00174
:105D0000639D900D729D900D11246FE3A62EAD0C36
:105D100064E670E00E941476EC2DE61B6E2F8A2D4F
:105D20000E94466529853A85C90183709070009765
:105D300061F48A2D6FE30E9446656D2D6695605E65
:105D40008FE30E9446653A8529852F5F3F4F81E2A8
:105D500090E0A0E0B0E0E80EF91E0A1F1B1F2E33F2
:105D6000310509F0BACF7CC0DD249981492E552434
:105D700047FC509401E210E0A92DBB27A7FDB09588
:105D8000BC83AB8354E6652E712C40E2A42EBA810D
:105D90002B2E332427FC3094E82DFF27E7FDF095C8
:105DA000FE83ED83FD2D21E2F29F70011124C701D6
:105DB000B2010E94022CB8010E942876AB81BC81FE
:105DC0006A9FC0016B9F900D7A9F900D11243EE554
:105DD000C32ECD0CB3010E941476BA2DB61B6B2FC7
:105DE0008C2D0E944665ED2DF0E0E370F070F88791
:105DF000EF83309749F48C2D60E20E9446656D2D4B
:105E0000605E8EE50E944665C701B1010E94022CCA
:105E1000B8010E9428762D813E81629FC001639F58
:105E2000900D729F900D11242EE5F22EFD18B301F6
:105E30000E941476605E8F2D0E9446658F81988542
:105E4000009749F48F2D60E20E9446656A2D6D1916
:105E50008EE50E944665D3949D2D9F3109F0A2CF17
:105E6000E0918808F0E0EE0FFF1FE952FB4F408001
:105E700051805201CC24B7FCC094DC2CC601B50182
:105E800021E230E040E050E00E945D76822F825AAD
:105E900061E04EE30E9496654091880820916E0172
:105EA00030E02170307082E090E0821B930B242F51
:105EB00030E08217930709F050C0443008F04DC01D
:105EC00080919B01807F09F448C0C601B5016050F4
:105ED0007C4F8F4F9F4F22E030E040E050E00E9427
:105EE0005D76A9816A2F772767FD7095C9010E94A9
:105EF000022CBC01660F771F882777FD8095982FAD
:105F0000292D97FC2D5F25952595332727FD309565
:105F1000432F532F0E94E97529E130E040E050E023
:105F20000E945D7679018A01CA01B9012FED3FEF28
:105F30004FEF5FEF0E945D76622F605C8FE34EE370
:105F40000E949265C801B70122E030E040E050E0D5
:105F50000E945D7679018A013CC01A141B041C045E
:105F60001D0414F4698101C06A81772767FD70956B
:105F7000C2010E94022C9C01442737FD4095542FFA
:105F80001A141B041C041D0414F4692D01C0682D8F
:105F900067FD6D5F65956595772767FD7095872F20
:105FA000972F0E94E97529E130E040E050E00E941F
:105FB0005D7679018A01CA01B9012FED3FEF4FEFFC
:105FC0005FEF0E945D76622F605E8FE34EE30E947A
:105FD0009265C601B50129E130E040E050E00E9441
:105FE000E975612CB1E07B2E812C912CA4019301E9
:105FF0000E945D7682E760E3A90120E00E942867A5
:10600000C801B70129E130E040E050E00E94E975A5
:10601000A40193010E945D7684E568E0A90120E077
:106020000E9428671A141B041C041D0474F4B9810F
:106030006B2F772767FD7095C20144970E94022C51
:10604000F701E81BF90BCF010BC0FA816F2F7727FF
:1060500067FD7095C20144960E94022C8E199F091B
:106060009C01220F331F220F331F280F391F442793
:1060700037FD4095542F84E560E100E3F3E0EF2E17
:106080000E94F2652A960FB6F894DEBF0FBECDBF10
:10609000CF91DF911F910F91FF90EF90DF90CF9004
:1060A000BF90AF909F908F907F906F905F904F9038
:1060B0003F902F9008952F923F924F925F926F9250
:1060C0007F928F929F92AF92BF92CF92DF92EF9288
:1060D000FF920F931F93DF93CF93CDB7DEB72F9728
:1060E0000FB6F894DEBF0FBECDBF982E85E39EE0BD
:1060F0000E94871B8DE898E0692D42E02CED37E087
:106100000AE0FDE3EF2EFEE0FF2ECC24C394E4E092
:10611000AE2E0E94FF1CF0908D08FA9430908E08ED
:10612000292D203841F4F7FC06C0F09288088AEF48
:106130009CE20E94F01585E168E045E25EE00E9485
:10614000146580E493E09C838B8379E8472E78E0A4
:10615000572EE7EDF4E0FB87EA8710E16624772409
:106160002F2D332727FD30953A832983C901880FC6
:10617000991FFC0153E0EE0FFF1F5A95E1F7E81B52
:10618000F90BFE83ED83F62CEB81FC81808160E0CE
:1061900040E00E944311882361F0EB81FC81818102
:1061A00060E040E00E944311882329F4BB24B394AB
:1061B00004C0BB2402C042E0B42E2B2D30E038874F
:1061C0002F83C901880F991F880F991FA301440FBE
:1061D000551F9A0103E0220F331F0A95E1F7241B94
:1061E000350B820F931F86579E4FDC01A355BE4F80
:1061F000FC01E455FE4F3C912081321751F4FC0123
:10620000E555FE4F86559E4F41E02081FC0180817F
:10621000281340E0EA85FB8581919191FB87EA870D
:106220009C0197FF04C022273327281B390B2A31F2
:1062300031050CF040E0242E8A3191051CF0F2016A
:10624000108207C0FFEF873E9F071CF421E0F20198
:10625000208380916E0190E081709070E2E0F0E028
:10626000E81BF90BE615F70551F480919B01807F3F
:1062700031F0F301E757F74F1082222423944F2D7A
:106280004F5F80E0612F20E00E947D0F5D864C868D
:10629000F2013081F1E0F98731111986809106050C
:1062A000882351F4DD24D394809182049091830457
:1062B000009721F4DD2402C0DD24D39489819A81E2
:1062C0008615970511F421E0311020E00F92EDB70B
:1062D000FEB73183892D60E04D2D07E2E12ECF2CF2
:1062E000AB2C88240E94302C0F9029813A812615EE
:1062F000370509F0D2C0332009F0CBC0DD2009F406
:10630000CCC0222009F4C9C08F819885880F991FBD
:10631000880F991FED81FE818E0F9F1F86579E4F1C
:10632000F9858F0F911D86559E4F9F878E87892DEA
:10633000EE85FF8560814CE924E60E949315EE8589
:10634000FF858083AAC021E00F92F2018081EDB722
:10635000FEB78183892D60E04D2D09E3E12ECF2C1E
:10636000AB2C882483940E94302C0F9029813A8191
:106370002615370509F097C0332D313009F08FC04D
:10638000DD2009F490C0222009F48DC08F8198850A
:10639000880F991F880F991FED81FE818E0F9F1F17
:1063A00086579E4FF9858F0F911D84559E4F988774
:1063B0008F83892DEF81F88560814CE920E00E9470
:1063C0009315EF81F88580836EC021E00F92EDB7C1
:1063D000FEB71182892D60E04D2D0FE3E12ECF2C09
:1063E000F3E6AF2E88240E94302C0F9029813A8149
:1063F0002615370521F421E0332D333009F020E054
:106400000F92EDB7FEB71182892D60E04D2D07E5A3
:10641000E12ECF2CE2E6AE2E88240E94302C089488
:10642000411C511C0F90EC85FD858081882319F457
:10643000222031F008C0222031F48AE34FE705C062
:106440008BE34EE702C08AE34DE2612F0E94B16404
:10645000FB2DF13019F0F23049F404C085E7612FCB
:106460004DE407C085E7612F4CE403C085E7612F49
:1064700048E40E94B1640894611C711C2B813C812A
:10648000225F3F4F3C832B83185F103309F07BCE94
:106490000CC0332D313009F456CF20E055CF832D79
:1064A000823009F492CF20E091CF2F960FB6F89466
:1064B000DEBF0FBECDBFCF91DF911F910F91FF9037
:1064C000EF90DF90CF90BF90AF909F908F907F9094
:1064D0006F905F904F903F902F90089520E030E0B4
:1064E000F901EE51F24FE491E81711F4822F08956B
:1064F0002F5F3F4FEE23A1F780E00895823430F400
:10650000E82FF0E0EE51F24F8491089580E2089573
:10651000EF92FF920F931F93182FF62EE22E862FE5
:10652000BA010E940C6586E66F2D412F2E2D0E9428
:10653000BA1CEE2039F0802F612F40E021E00E944C
:10654000A215182F812F1F910F91FF90EF900895A2
:10655000FF920F931F93F82E10919501212F33274F
:1065600027FD309537FF03C0309521953F4F022F0F
:1065700025320CF43DC02091390830913A088091C1
:10658000370890913808282B392B80913B0890913F
:106590003C08282B392B8091360890E0282B392B8A
:1065A0004091330850E0242B352B2115310531F46F
:1065B000812F881F8827881F8093330811161CF4A9
:1065C000812F845202C0812F8C5D60E040E00E94E8
:1065D0004311882359F090913308992339F491E0BD
:1065E00020913608211190E090933608809333086B
:1065F0002091390830913A082F5F3F4F30933A0885
:106600002093390820913708309138082F0D311D1B
:1066100030933808209337080E94D40E20913B080D
:1066200030913C08821B930B8436910508F471C1AC
:106630002C593F4F30933C0820933B08209137085A
:1066400030913808E0913908F0913A08C901BF014A
:106650000E941476F62E462F50E04E9FC0014F9FA9
:10666000900D5E9F900D1124281B390B3093380834
:106670002093370810923A081092390800311CF420
:10668000109236080FC005326CF411161CF4812FDD
:106690008F5002C0812F815F60E040E00E94431173
:1066A000809336088091230690912406019690935A
:1066B00024068093230640912506509126064F5FBD
:1066C0005F4F5093260640932506FF2049F08091A6
:1066D000290690912A06019690932A06809329060E
:1066E00080913608882349F08091270690912806EA
:1066F00001969093280680932706F69420912B0606
:1067000030912C062F0D311D30932C0620932B0633
:10671000809197019091980190932F0680932E0677
:1067200060919501772767FD709577FF03C070959D
:1067300061957F4F662319F410922D061EC06130BB
:1067400019F4841B950B15C0603168F460FF06C016
:10675000A4E036952795AA95E1F709C0209129066E
:1067600030912A0604C02091270630912806821B0A
:10677000930B90932F0680932E0680912D068130E7
:1067800051F0813018F0823049F514C080919501A4
:10679000882321F120C080912E0690912F06181693
:1067A0001906E4F080919701909198010097B1F05B
:1067B00082E012C080912E0690912F062FEF853C2B
:1067C00092071CF483E080932D06809197019091AD
:1067D0009801009719F481E080932D0680912E0690
:1067E00090912F06209134083091350828173907E9
:1067F00009F479C020912D06213009F065C020915F
:10680000700122FF45C02091970130919801211518
:106810003105F1F18E31910519F489E10E942D7253
:1068200080912E0690912F068431910519F48AE10A
:106830000E942D7280912E0690912F068A3091052C
:1068400019F48BE10E942D7280912E0690912F06F3
:10685000843091051CF48CE10E942D7280917001AE
:1068600083FF16C080912E0690912F068E319105E0
:1068700049F08431910531F08A30910519F0843066
:10688000910534F482E390E090938604809385042C
:106890008091700181FF27C08091960120912E0682
:1068A00030912F0680FF07C0809197019091980149
:1068B000821B930B01C0C9016CE370E00E94147647
:1068C000009789F480E003C0223069F48CE10E94D3
:1068D0002D728091700183FF06C082E390E0909357
:1068E00086048093850420912E0630912F063093E4
:1068F0003508209334088091960180FF0AC080916A
:10690000970190919801821B930B90932F0680938F
:106910002E061F910F91FF90089580919501992760
:1069200087FD909597FF03C0909581959F4F982F75
:10693000823034F1803124F585959A3024F40E9418
:10694000BB6990E003C0992787FD90950197FC01F2
:10695000EE0FFF1FE952FB4F20813181809195019D
:1069600087FF05C080E094E0821B930B03C0C90140
:1069700080509C4F26E0969587952A95E1F702C0B6
:1069800080E090E00E94A83283E00E94BB69E82F7B
:10699000F0E0EE0FFF1FEB52FB4F808191818050A2
:1069A0009C4FB6E096958795BA95E1F720919601B0
:1069B00022FF0AC08530910538F0209188042223F7
:1069C00019F423E02093880420912F083091300897
:1069D0002F5F3F4F3093300820932F0820912D08D0
:1069E00030912E08280F391F30932E0820932D0840
:1069F0000E94D40E2091310830913208821B930BF3
:106A000023E0883E9207E8F10E94D40E909332086A
:106A10008093310880919901823051F485E160E0E2
:106A200040E00E944311882319F087E00E942D72F4
:106A300080912D0890912E0860912F087091300858
:106A40000E94147610922E0810922D081092300891
:106A500010922F088091A9069091AA060196909312
:106A6000AA068093A9068091A806E82FF0E0E05DD1
:106A7000F94F60838F5F8093A806883710F01092DB
:106A8000A806089510922D0610922606109225064B
:106A900010922A06109229061092280610922706B4
:106AA00010922C0610922B0608950F931F93182F07
:106AB00080912106882319F062ED7DE002C065EC2B
:106AC0007DE088E00E940C6581E060E14AE851E0E9
:106AD0002AE000E10E94B56482E460E14FE30E9495
:106AE000B16482E168E24EEB5DE00E94146582E1F0
:106AF00060E34FEA5DE00E941465113609F44AC074
:106B00001F3B21F0103609F04FC004C080E00E9406
:106B10002D724AC0809121068823A9F08DE99DE05D
:106B20000E948513809122060E943E5E882339F0E0
:106B300087E10E942D7282E08093210629C080E0C7
:106B40000E942D7225C0809157018F5F0E940261C3
:106B50001091570108C01150113108F01FE08091C9
:106B60005701181739F0812F8F5F0E94B560882375
:106B700091F301C010E01093570181E00E94D65EAE
:106B80000E94725F809157010E94005E0E94423510
:106B900080E601C081E60E94F16881E00E94BB1599
:106BA00087ED95E30E94F0151F910F910895AF9224
:106BB000BF92DF92EF92FF920F931F93CF93DF93D9
:106BC000182F8FE29CE00E94871B80910605882386
:106BD000A1F4E0910905E7FF10C0E195EA3008F063
:106BE000E9E0F0E0EE0FFF1FE452F84F25913491F9
:106BF000C9010E94E01510920905F090840884E80C
:106C000098E0612F4FE00E945E2586E360E04AE253
:106C10005CE00E9414650E94F75FAC0186E660E0CC
:106C200020E00E94286780E06AE041E00E94DA1CD0
:106C3000D090840880912106823021F4109283083C
:106C400010922106163648F4143690F5103609F4E1
:106C500056C0113609F075C00AC0113809F456C083
:106C60001F3B09F465C0103809F06BC053C0809118
:106C700083088823E9F01092830887E10E942D722F
:106C800081E60E94F1680E94725F8091840880937F
:106C900057010E94005E0E94423581E00E94D65E4C
:106CA0000E94725F82E00E94D65E0E94725F49C0BD
:106CB000809157018D15B9F0812F0E94F168809164
:106CC0008408809357010E94725F809157010E944F
:106CD000005E0E94423581E00E94D65E0E94725F93
:106CE00081E00E942D72153619F488E890E204C004
:106CF000143639F58CE69AE40E94E01522C081E052
:106D00008093830887E10E942D721BC081E00E945E
:106D1000BB1517C080918308882399F081E0809388
:106D20002106D092220685E595E30E94F01509C060
:106D300010928308809157018093840881E00E941B
:106D4000E45E80918308882341F0FD1431F06D2DBD
:106D50006F5F8F2D8F5F0E94C360CD2DDD27C7FD34
:106D6000D095809105059E01281B3109C90118168F
:106D700019065CF0CE01019797FF02C080E090E019
:106D80008093050510E1DD240BC025303105D4F3D7
:106D9000CE0104978B3091059CF38AE090E0F0CF10
:106DA000F0900505FD0CAF2CBB2495012F5F3F4FE4
:106DB000442737FD4095542FCA15DB0511F401E136
:106DC00001C000E182E1612F72E0E72E0E94F265CE
:106DD00080915701F81629F481E0612F4AE20E9460
:106DE000B1648F2D64E778E04FE00E94B85DCA156A
:106DF000DB0531F480918308882311F001E101C0A3
:106E000000E188E1612F44E758E02FE00E94B5647B
:106E1000D394185F3D2D363019F6DF91CF911F9135
:106E20000F91FF90EF90DF90BF90AF900895AF92D9
:106E3000BF92CF92DF92EF92FF920F931F93CF9367
:106E4000DF935B016C0110E1E12EF12CC0E0D0E892
:106E500000E010E89E0140E050E0CA01B9010E9444
:106E6000E975A616B706C806D90610F4C027D127BB
:106E7000169507950894E108F108E114F10461F40E
:106E8000CE01DF91CF911F910F91FF90EF90DF9096
:106E9000CF90BF90AF900895C02BD12BDBCFE1E016
:106EA000683068F4E0E070E09B01220F331F220F8E
:106EB000331F260F371FA90140595C4F0EC070E0E9
:106EC000685070409B0153E0220F331F5A95E1F741
:106ED000260F371FA90148565C4FDA012C918050CC
:106EE0009C4F97FD0FC0B8E080309B078CF0EE23DD
:106EF00019F028E030E002C024E030E0240F351F14
:106F0000F9012081332727FD3095322F222730C009
:106F1000EE2329F0692F9070880F991F03C0692F05
:106F200066959170262F30E0FA01E20FF31F618120
:106F3000772767FD7095AC0155954795649F900143
:106F4000659F300D749F300D11246081772767FD98
:106F5000709540E052E0481B590B55954795649F4A
:106F6000C001659F900D749F900D1124280F391F4B
:106F7000C90169E170E00E942876CB0108952F9243
:106F80003F924F925F926F927F929F92AF92BF9289
:106F9000CF92DF92EF92FF920F931F93DF93CF93E5
:106FA00000D00F92CDB7DEB7182F9924939480911B
:106FB0009908883008F499248AED90E10E94871B93
:106FC000992011F05AE001C056E089EB98E0612F5A
:106FD00040E020E030E000E070EEE72E70E1F72EB8
:106FE000CC24C394A52E0E94FF1C4091990850E028
:106FF0004F5F5F4F84E260E021E00E94286780914C
:107000009908992079F090E008977C0103E0EE0C54
:10701000FF1C0A95E1F7E80EF91E28E933E0E20EBD
:10702000F31E0CC090E07C01EE0CFF1CEE0CFF1C6C
:10703000E80EF91E80E793E0E80EF91E0091B9080A
:107040000150D090BA08113661F0123628F4143489
:10705000D1F0153471F50EC01436A9F0153649F586
:1070600009C0DD2031F11092BA0881E60E94F16872
:10707000DD241FC0809106058823D9F01D14CCF4AF
:107080008D2D815014C080910605882391F02D2DFF
:10709000332727FD3095992019F089E090E002C050
:1070A00085E090E02817390724F48D2D8F5F8093B9
:1070B000BA088091BA0880930605CE2C4F2C6E2C0E
:1070C0007F2C90E122243324A02EBB24A7FCB09473
:1070D000F30141913F01552747FD509521E0A2144E
:1070E000B30409F020E088E1692F99830E942867A2
:1070F0000894211C311C9981985F983349F7992095
:1071000001F1A5E06A2E712C6E0C7F1C90E1F5E078
:107110002F2E312CF30141913F01552747FD50950A
:1071200021E0A214B30409F020E080E3692F9983E1
:107130000E9428670894211C311C9981985F903324
:1071400049F70F3F11F421E0D11020E08CE068E016
:1071500043ED50E10E94E564992019F089E090E048
:1071600002C085E090E021E0A816B90609F020E011
:107170008CE068E34CEC50E10E94E564992019F042
:1071800089E090E002C085E090E0A816B90694F48A
:1071900007FD4EC0A02EBB24A7FCB094AE0CBF1CB4
:1071A000812FF50160814CE924E60E949315F501D9
:1071B00080833EC01016E4F5812F6091B8084CEF33
:1071C00024E000E00E9485158093B80890917F0428
:1071D000992371F1992021F050E194E049E003C036
:1071E00058E092E045E024E6820230011124892F24
:1071F00090E0909581959F4F869D9001879D300DE1
:10720000969D300D1124EC2DF42DA52E00E0C90122
:107210006A2D702F0E9428766193260D371D8E2FC0
:107220008C198417A0F382E00E94D65E0E94725FE0
:1072300080910605882351F0AA24ECE92E2EEFEF69
:107240003E2E4D2C552447FC5094A5C000E01CEF69
:10725000AA24BB2470E2D72EACC0C90165E0880F18
:10726000991F6A95E1F7992019F064E070E002C077
:1072700062E070E00E942876462F062F055C3701F9
:107280006A0C711CF3018081992787FD909555E068
:10729000880F991F5A95E1F7B1010E942876562F61
:1072A00090E2D92ED60E2F5F3F4F8D2D90E09B831D
:1072B0008A834216530609F050C082349105ACF41B
:1072C0008AE3C82EC40E625E8C2D45E059830E946D
:1072D00092655981EA81FB81E134F10531F0652F36
:1072E000615E8C2D45E00E949265FD2DF03430F4F6
:1072F000802F81506D2D45E00E9492652A813B814F
:107300002F33310594F401506D2D6F5F802F45E0D0
:107310000E9492658A819B818E33910531F06D2D9B
:107320006E5F802F45E00E9492658091820490916B
:107330008304009741F4123631F0133621F01234F1
:1073400011F0133439F5812FF30160814CE924E603
:107350000E949315F30180831DC02A813B81213453
:1073600031052CF4615E802F43E00E9492653D2D33
:10737000303428F4802F6D2D43E00E9492658A817D
:107380009B818F33910534F46D2D6F5F802F43E027
:107390000E949265A3942A2D30E0992019F089E08B
:1073A00090E002C085E090E0281739070CF455CF33
:1073B0004DCFC801609199080E944F37BCE3EB2E76
:1073C000EA0C9C01A5E036952795AA95E1F76D2D6D
:1073D000621B8E2D0E944665950123703070211529
:1073E000310521F48E2D60E20E9446650894A11CAF
:1073F000B11C005E1F4F90E4A916B104D1F68CE5D4
:1074000060E040E40E9496650F900F900F90CF913E
:10741000DF911F910F91FF90EF90DF90CF90BF9081
:10742000AF909F907F906F905F904F903F902F9084
:1074300008952F923F924F925F926F927F928F9218
:107440009F92AF92BF92CF92DF92EF92FF920F93F3
:107450001F93DF93CF93CDB7DEB7A2970FB6F89403
:10746000DEBF0FBECDBF8F8F98A36A8B809184043F
:10747000882309F474C080910705882319F081508E
:10748000809307058091B3069091B4062091B106D0
:107490003091B206820F931F2091B5063091B60647
:1074A000820F931F2091B7063091B806820F931F69
:1074B00020914007309141072C01421A530A920152
:1074C00057FE03C0309521953F4F41E021303407EE
:1074D0003CF0909341078093400781E080938704BC
:1074E00080916F01863FD9F1909108019233B8F1F4
:1074F00090913D079F5F90933D07903160F0209100
:107500003E0730913F072F5F3F4F30933F07209357
:107510003E0710923D0790918704992321F0109225
:107520003F0710923E0720913E0730913F07992771
:1075300087FD90950A9667E771E0869FA001879F77
:10754000500D969F500D11244217530740F423709D
:1075500030702130310519F480E10E942D72809144
:107560006E01582F51705F5F598781FF02C01D86E1
:1075700002C063E06D876090A201662009F44AC0F2
:107580008985E82FF0E0EE0FFF1FE952FB4FA08046
:10759000B180CC24B7FCC094DC2C9D85E92FF0E0B1
:1075A000EE0FFF1FE952FB4F20813181442737FD49
:1075B0004095542FCA01B9010E94E9757B018C01E5
:1075C000C601B501A60195010E94E975E60EF71EF8
:1075D000081F191F662D70E080E090E0EAE0660F5A
:1075E000771F881F991FEA95D1F724E630E040E025
:1075F00050E00E945D76B901CA010E94E9756E15DE
:107600007F058007910730F4C801B7010E94173742
:107610004C0102C088249924B40180E090E024E663
:1076200030E040E050E00E94E9756B8F7C8F8D8FD9
:107630009E8F6AE2662E61E0762EA1EBB6E0BE8BED
:10764000AD8BFE013196F88FEF8B50E0252E51E087
:10765000352E2AE831E03F872E8747ED54E05A8FD8
:10766000498F2901F98BE88BBC8BAB8BEE24FF246F
:107670001B865A89517059A3AE2C8E2D0E948216FA
:107680009C01D30111968D919C911297281B390B67
:10769000B901882777FD8095982F4AE0660F771FFC
:1076A000881F991F4A95D1F7121613062CF45D9680
:1076B0002D913C915E9703C0F301278530892436D4
:1076C000310514F424E630E0442737FD4095542F6B
:1076D0000E945D768901FCEF21303F072CF024E009
:1076E0000030120724F405C000E01CEF02C000E0E7
:1076F00014E08091700180FF0FC080916E0190E0D6
:107700008170907042E050E0481B590BE416F5067A
:1077100019F4109501951F4FA98DBA8D0D931D93E6
:10772000BA8FA98FC8010F968F319105F0F4B4E09C
:10773000EB16F1047CF48A2D8F5F0E94BB6990E008
:107740000197E1E0F0E002C0EE0FFF1F8A95E2F73B
:10775000CF0108C081E090E00E2C02C0880F991F75
:107760000A94E2F7FB85F82BFB872A2D243008F0DA
:107770007AC139A1332309F05FC08091960181FF5E
:107780005BC06701CC0CDD1C44E651E0C40ED51E85
:10779000D60111968C911197807C09F44DC08C9183
:1077A00085958595859561E040E00E944311882389
:1077B00009F442C0D601EC91E770F0E0DF01AA0FB6
:1077C000BB1FA457BB4FEE0FFF1FE45AFE4F8D9116
:1077D0009C91119720813181821B930B62E070E0B4
:1077E0000E942876F701EE0FFF1FEB59FE4F208114
:1077F000422F440F440F45954595552747FD509519
:10780000649FC001659F900D749F900D11246FE1DE
:1078100070E00E942876660F771F660F771F22950B
:10782000269526952370213019F0223029F403C0C3
:10783000060F171F01C08B018114910409F1B9854E
:10784000AB1619F0ED85AE16D9F46091A20170E087
:1078500080E090E04AE0660F771F881F991F4A95E5
:10786000D1F79801442737FD4095542F0E94E975C0
:107870002B8D3C8D4D8D5E8D0E945D76022F132FDA
:10788000F201EA54FE4F808160E040E00E94431123
:10789000882369F0F201E954FE4F808160E040E006
:1078A0000E944311882329F4CC24C39404C0CC241F
:1078B00002C032E0C32E80916E0190E08170907022
:1078C00022E0A22EB12CA81AB90AAE14BF0469F5A1
:1078D00080919B01807F49F1C80180509C4F62E0FC
:1078E00070E00E9428769B01EC2DF0E0EE0FFF1F68
:1078F000EE0FFF1FA701440F551FCA01A3E0880F19
:10790000991FAA95E1F7841B950BE80FF91FEC5C12
:10791000FC4F6081772767FD7095C9010E94022C9A
:10792000AC01440F551F30E028C031E0101611069D
:107930000CF430E08C2D90E0A701440F551FFA01A4
:1079400063E0EE0FFF1F6A95E1F7E41BF50B880F6C
:10795000991F880F991FE80FF91FE657FE4FE30F95
:10796000F11DE655FE4F6081772767FD7095C801D0
:107970003AA30E94022CAC013AA1EC2DF0E0EE0FEC
:10798000FF1FEE0FFF1FB701660F771FCB0113E03C
:10799000880F991F1A95E1F7861B970BE80FF91FBF
:1079A000E657FE4FE30FF11DE455FE4F6081772748
:1079B00067FD70956C597F4F882777FD8095982FCC
:1079C000DA019D01442737FD4095542F0E94E97547
:1079D00024E630E040E050E00E945D76022F132F55
:1079E000AE14BF0499F580919B01982F907F09F404
:1079F00066C60050144063C6D101ED91FC91119709
:107A000060818091700180FD6195772767FD709599
:107A1000872F972F63587F4F8F4F9F4F20E034E081
:107A2000201B310B442737FD4095542F0E94E975E8
:107A300020E038E040E050E00E945D762030B8E081
:107A40003B07B0E04B07B0E05B0739F4D101ED91A3
:107A5000FC912081332727FD3095220F331FE889C1
:107A6000F98931832083AB89BC890D931D93BC8B2D
:107A7000AB8B0894E11CF11CE2E0F0E06E0E7F1E7F
:107A8000288939892E5F3F4F398B288B2E0E3F1E58
:107A90004EE050E0440E551E57E0E516F10409F0A3
:107AA000EBCD00919F016B85062380914207809565
:107AB000802319F088E10E942D720093420780E034
:107AC00094E09093C0068093BF069093C206809383
:107AD000C106ECE8F4E02CE531E0A9ECB6E0BD012C
:107AE00081919191D9014D915D919D01841B950BDF
:107AF000880F991FDB018D939D93BD01B4E0E4399C
:107B0000FB0771F78091940490919504880F991F59
:107B10009093D2068093D106809196049091970419
:107B2000880F991F9093D4068093D3068091980470
:107B300090919904880F991F9093D6068093D5064B
:107B400080919A0490919B04880F991F9093D80676
:107B50008093D706EDEFF6E0FC87EB8729ED36E062
:107B60004191519161917191D9014D935D939D0125
:107B7000B7E0ED33FB07A1F7C090A201CC2009F4D8
:107B80007AC0E985AE2EBB24AA0CBB1C21EB422E89
:107B900026E0522EA40CB51CD5012D903C90442417
:107BA00037FC4094542CBD850B2F10E0000F111FA3
:107BB0000F54194FF80120813181442737FD40953A
:107BC000542FCA01B9010E94E9753B014C01C20161
:107BD000B101A20191010E94E975660E771E881E0F
:107BE000991EDD24EE24FF248AE0CC0CDD1CEE1C63
:107BF000FF1C8A95D1F7C701B60124E630E040E0CA
:107C000050E00E945D76B901CA010E94E9756615CF
:107C100077058805990578F5C401B3010E941737E7
:107C2000BC0180E090E024E630E040E050E00E94BB
:107C3000E9753B014C01C201B101A70196010E9407
:107C4000E975A40193010E945D76D5012D933C93C3
:107C5000F80160817181882777FD8095982FA701B1
:107C600096010E94E975A40193010E945D76D801F6
:107C700011963C932E93E090A0018E2D807E09F406
:107C8000DEC0B9852B2F30E0220F331FF901EF54EE
:107C9000F94F40815181CE010196280F391FD9013A
:107CA000ED91FC91BD856B2F70E0660F771FDB01B6
:107CB000AF54B94F2D913C91860F971FDC018D91E8
:107CC0009C91BA89B1FD05C0E40FF51F280F391F3B
:107CD00004C020E030E0E0E0F0E0A091A101AA23A0
:107CE00049F0B0E0AA0FBB1FA155B94F0D911C91EF
:107CF000119702C000E010E0E2FE03C0F095E195AC
:107D0000FF4FE3FE03C0309521953F4FE4FE03C0D3
:107D1000109501951F4F8091A001829586958770DF
:107D2000823071F1833020F4813009F088C007C0BF
:107D3000833009F459C0843009F081C06CC0C90196
:107D400068E070E00E9428767B01C90160E870E07D
:107D50000E94287629014E185F087201E61AF70A78
:107D6000C90160E072E00E942876E61AF70AC801AD
:107D70008E1B9F0B9093C4068093C306CF0120C037
:107D8000CF0168E070E00E9428767B01CF0160E8B7
:107D900070E00E9428763F016E187F087301E61A92
:107DA000F70ACF0160E072E00E942876E61AF70A2F
:107DB000C801821B930B9093C4068093C306C9012C
:107DC00062E070E00E942876600F711FCB018E0D7B
:107DD0009F1D9093C6068093C5066E197F09709308
:107DE000C8066093C7062BC0C8018E1B9F0B9093DB
:107DF000C4068093C306E00FF11FCF01820F931FCB
:107E00009093C6068093C506E21BF30BF093C80659
:107E1000E093C70614C0C8018E1B9F0B9093C40645
:107E20008093C306C801820F931F9093C606809368
:107E3000C506021B130B1093C8060093C70680915A
:107E40008404882311F00E948D3480E4EDEFF6E085
:107E5000DF011D928A95E9F7BA89B1FF2DC08091A3
:107E60006E0190E08170907022E030E0281B390BA9
:107E700080E090E0ED89FE89AF89B88D2817390739
:107E800029F01182108211961C921E920196329650
:107E900012968430910591F71092CA061092C90685
:107EA0001092CC061092CB061092CE061092CD0600
:107EB0001092D0061092CF068CE693E090930101C9
:107EC000809300019C012F5F3F4F3093030120936B
:107ED00002019C012E5F3F4F309305012093040166
:107EE0000396909307018093060123E0422E28E039
:107EF000522E93E8692E97E0792E83E4282E87E0AE
:107F0000382E19861D8689850E94DC0E7C01FC01B5
:107F100080818150803108F0ADC2838161E040E012
:107F20000E944311D2019C918823A1F4292F1C9215
:107F3000F7019181892F8850823008F08AC28781A9
:107F40008E70843009F485C2993009F04BC000E08E
:107F50001CEF4AC021E0911120E081E0D2018C9316
:107F6000D7011196EC913E2F3150832F90E0DC0128
:107F7000AA0FBB1FAF54B94F0D911C91119734310B
:107F800060F0B9853B1748F4DC01AA0FBB1FAA0FAC
:107F9000BB1FA350B94F0D911C91D70117963C916F
:107FA0001797832F807381F0832F8295837090E0E1
:107FB000019741E050E002C0440F551F8A95E2F757
:107FC000CA015D85582B5D8736FF0EC0E53060F431
:107FD000F0E0EE0FFF1FE250FF4FC70108969183BC
:107FE000808302C000E010E0D7011796CC9017976D
:107FF000C6FC0BC018968C911897882331F02AA3E1
:108000000E94BF0E080F191F2AA1F701868188233D
:1080100021F48581882309F458C1D3016D917D91A4
:108020008D919C911397222389F420E031E040E068
:1080300050E00E945D7650954095309521953F4FD8
:108040004F4F5F4F4801820E931E5AC08C2D8E7089
:10805000843051F5D701EC91F0E0EE0FFF1FE952AB
:10806000F94F60817181882777FD8095982F20E0F6
:1080700034E640E050E00E94E975F30160837183CB
:1080800082839383D70112962C911297222361F059
:10809000332727FD3095432F532F0E945D76F30140
:1080A0002083318342835383D3016D917D918D91E0
:1080B0009C91139720E031E040E050E00E945D7613
:1080C00050954095309521953F4F4F4F5F4F480158
:1080D000820E931E8114910499F0F701258197FE79
:1080E00022952F7030E044E650E0249FC001259F88
:1080F000900D349F900D1124D10111969C938E9375
:10810000F10180819181009799F0209184042223CC
:1081100019F0019791838083D1018D919C911197E2
:10812000009731F0F3016081718182819381B7C042
:108130008114910409F4C9C0D70116968C91169741
:10814000882309F4B4C080918404882309F476C09C
:1081500012962C9112972223B1F0332727FD3095E8
:1081600037FF03C0309521953F4F332727FD3095CA
:10817000432F532F60E070E080E293E00E945D7631
:1081800059016A0106C0A12CB12CF0E2CF2EF3E018
:10819000DF2EF701868118141904FCF48F7090E02B
:1081A0000097F1F144E650E0849F9001859F300DE7
:1081B000949F300D1124442737FD4095542FC6015C
:1081C000B5010E945D76F30180819181A281B38126
:1081D000280F391F4A1F5B1F2CC082958F7090E0BB
:1081E0000097F1F044E650E0849F9001859F300DA8
:1081F000949F300D1124442737FD4095542FC6011C
:10820000B5010E945D7659016A01D3012D913D911E
:108210004D915C9113972A193B094C095D0909C0DE
:108220009801442737FD4095542F542F432F322F68
:108230002227F3012083318342835383D3016D913D
:108240007D918D919C9120E031E040E050E00E94D2
:108250005D76C801AA2797FDA095BA2F18141904B6
:1082600034F482179307A407B50734F012C0281717
:1082700039074A075B076CF4222717FD2095322F38
:10828000322F212F102F0027F30100831183228327
:108290003383D3016D917D918D919C91139720E053
:1082A00031E040E050E00E945D7689010EC0C801D7
:1082B000AA2797FDA095BA2FBA2FA92F982F882704
:1082C000F30180839183A283B383D70114966C91C9
:1082D0001497633061F1643028F4613051F06230FA
:1082E000A0F444C0653069F1653038F1663081F53D
:1082F0002BC0F7018181893029F417FD35C000506A
:1083000012400EC017FF32C02CC0D70111968C91BD
:108310001197893041F41016110604F100501E4FD8
:10832000000F111F23C010161106DCF01FC017FF2D
:108330001DC0109501951F4F19C01016110674F03D
:1083400010C017FF0EC010C0101611063CF00CC074
:108350006750C8010E944F378C0108C000E014E04C
:1083600005C000E010E002C000E01CEFF7018781CB
:1083700080FD13C0E181EE2381F0E53070F4F0E080
:108380003197EE0FFF1F21E030E02C0F3D1FE20F71
:10839000F31F80819181080F191FB801882777FD8D
:1083A0008095982FD70112962C911297332727FD8D
:1083B0003095432F532F0E94E975F701008110E09B
:1083C00001501040278126952770213071F0F80167
:1083D000EE0FFF1FEE0FFF1F223069F5E350F94F3C
:1083E000608371838283938334C024E630E040E06D
:1083F00050E00E945D76E22EC32EDA01000F111FBD
:10840000000F111F0350194FF80120813181428163
:1084100053816E2D7C2DCD010E94E97520E034E062
:1084200040E050E00E945D76D8012D933D934D933E
:108430005C9313970EC0E350F94F20813181428144
:108440005381260F371F481F591F208331834283D2
:108450005383B985BF5FB9870894411C511CE4E080
:10846000F0E06E0E7F1E22E030E0220E331EB032AE
:1084700009F049CD0E94D40E8C01ED84E0FE05C0C8
:10848000882319F48EE10E942D72E1FE0BC0C80111
:1084900090708034910519F08834910519F48FE1BA
:1084A0000E942D72E2FE0DC010700038110531F0EF
:1084B0000838110519F00039110519F480E20E94FD
:1084C0002D72B5EE4B2EB4E05B2E3F8D28A1832F8D
:1084D000922F9A87898722243324598A488AAB8528
:1084E000BC85ED90FD900D911C91C801B70124E66B
:1084F00030E040E050E00E945D76EB85FC85208313
:10850000318342835383A889B9892D933D93B98BD5
:10851000A88BEE85FF85E35AFE4F80819181EE8521
:10852000FF85E55AFE4F2081BAE02B02600111243D
:10853000E8EEF3E0CE0EDF1EEE85FF85E65AFE4F35
:1085400020812B0250011124A8E14A2EACEF5A2EB3
:10855000A40CB51C96014C2D232F8C159D0514F4ED
:10856000482F292F842E922E8A149B040CF4450147
:10857000E114F1040105110569F19401442737FD67
:108580004095542F1E141F041006110654F4B60112
:10859000882777FD8095982F621B730B840B950BB2
:1085A0000DC0C501AA2797FDA095BA2F29013A0150
:1085B000481A590A6A0A7B0AC301B201A801970145
:1085C0000E94E97520EA36E841E050E00E945D76BD
:1085D00079018A01C4010E94681B3C01882477FC50
:1085E0008094982C6E0C7F1C801E911EC6010E94E8
:1085F000681B8C01C5010E94681B222717FD20956E
:10860000322F061517052805390514F438014901DC
:10861000AA2797FDA095BA2F8401730168167906E1
:108620008A069B0614F47C018D01EE85FF85E45AD1
:10863000FE4F8081882341F010950095F094E094DE
:10864000E11CF11C011D111DFAE8CF2EF1E0DF2E17
:10865000C20CD31CF601E358FD4F8081882389F0BA
:1086600060E040E00E944311882359F0F601E2588F
:10867000FD4F80810E94BF0E7C010027F7FC009512
:10868000102FF894A985BA85ED92FD92BA87A98733
:108690007894EB85FC853496FC87EB87E2E04E2EE0
:1086A000512C240C351C2E853F852B5F3F4F3F8777
:1086B0002E8730E22316310409F011CF04C08F70E9
:1086C00009F09AC9C3C9A2960FB6F894DEBF0FBECF
:1086D000CDBFCF91DF911F910F91FF90EF90DF9071
:1086E000CF90BF90AF909F908F907F906F905F9052
:1086F0004F903F902F900895EF92FF920F931F930A
:10870000DF93CF93CDB7DEB7C054D0400FB6F89407
:10871000DEBF0FBECDBF8E010F5F1F4FC80163E0EC
:108720000E94193A81E2E82EF12CEC0EFD1EC701E1
:1087300061E00E94193AE6EEF2E0418152816081E7
:10874000D8012D913C91D7018D919C911197662371
:1087500029F0B901681B790BCB0102C0821B930B76
:10876000840F951F73E0883E97072CF4ACEF893196
:108770009A0724F005C088EE93E002C088E19CEFE0
:108780009283818335960E5F1F4F62E070E0E60EA4
:10879000F71E73E0E633F70781F680916E0190E0F3
:1087A0008170907022E030E0281B390B80E090E06F
:1087B0002817390721F0FC01E459FC4F108201967B
:1087C00084309105A9F786E00E94D65E81E00E9480
:1087D0002D72C05CDF4F0FB6F894DEBF0FBECDBF69
:1087E000CF91DF911F910F91FF90EF9008952F92FD
:1087F0003F924F925F926F927F928F929F92AF9231
:10880000BF92CF92DF92EF92FF920F931F93DF936D
:10881000CF9300D000D0CDB7DEB790916C01192F67
:108820001F708038B9F18138A8F4833209F47EC012
:10883000843230F4803221F1823209F0C3C083C027
:10884000853209F465C0853208F45DC0813609F0CF
:10885000B9C092C0833809F483C0843838F48138B1
:1088600009F49AC0823809F0ADC080C0853809F497
:1088700057C0853808F43FC08F3B09F0A3C096C0AD
:10888000153009F09FC08091880491E0892780937A
:10889000880488C0163049F5892F90E08073907065
:1088A0008032910561F48091E90E9091EA0E9095E5
:1088B00081959F4F9093B0068093AF0683C0009739
:1088C000A1F480912A04807C803C21F489E99EE017
:1088D0000E94CD7380912E04807C803C09F072C090
:1088E0008DE99EE00E94CD736DC00E94B1150E947B
:1088F000F01580E805C087ED95E30E94F01584E847
:108900000E94F1685FC0163009F05CC0905F04C03F
:10891000163009F057C090519F7390936C0142C07C
:1089200083EF91E50E94F01585E8EACF812F8F5FF4
:1089300080936C01883010F010926C0181E00E94ED
:10894000D65E83E130C0112319F0812F815001C020
:1089500087E080936C0181E00E94D65E84E123C0B1
:108960008EE89BE10E94E01583E8CACF89E29CE192
:108970000E94E01582E8C4CF80912D06823021F458
:1089800083E080932D060EC0153019F40E942F1637
:1089900009C01630B9F404C00E9442350E942F1657
:1089A0000E94C77487E10E942D720CC081E00E9472
:1089B000F16883E00E94F16882E00E94F16881E042
:1089C00080932C0880919E0160E040E00E9443115A
:1089D000882331F080912C08882311F40E947C4375
:1089E00080919E0160E040E00E94431180932C083A
:1089F00080916C01803108F0D3C090910801809182
:108A00005901981710F496E001C094E0EAE8EE2EC0
:108A1000E1E0FE2E0AE0D7014D917D01802F60E05C
:108A200024E09A830E94F263055F9A81083799F7E0
:108A3000492F406884E260E10E94770F84E268E198
:108A400046E50E94B16480912D06882399F082301A
:108A500011F406E001C004E040912E0650912F066B
:108A60008EE560E1202F0E94F80E83E368E140E08C
:108A70000E941C1040919C0183E04802A001112437
:108A80004358574F84E260E123E000E00E94B56460
:108A900080919B018F7031F089E360E149E758E0F4
:108AA0000E9414657EE0C72E71E0D72E60E0A62EEE
:108AB00061E0B62E662477245FE1E52EF601019190
:108AC0006F01D501ED91FD915D01808187FD8D5F85
:108AD00085958595843E0CF484EEF82E8D3114F046
:108AE0004CE1F42E862D81508230F8F4802F64E022
:108AF00046E30E94966520916E0130E026253725D9
:108B000020FD04C080919B018F7061F4802F815003
:108B10006EE143E00E949665802F8F5F6EE143E037
:108B20000E9496659E2D9F1914C0802F8B516BE378
:108B300046E30E949265802E8A94882D6AE343E082
:108B40000E949265882D6CE343E00E9492650F0DB0
:108B50009BE33DEF832E800E2DEFF22EF90E882D34
:108B60006F2D47E09A830E9496659A81692F6D5F09
:108B7000882D47E00E949265802F8D5F6F2D47E022
:108B80000E949665882D6F2D47E00E94926508949B
:108B9000611C711CB4E06B16710409F08FCF27C003
:108BA00080E060E04AE851E02AE001E10E94B5641B
:108BB0009091080180915901981710F442E001C08A
:108BC00040E084E560E00E94770F80912D068823C5
:108BD00071F0823011F402E001C000E040912E06F5
:108BE00050912F068FE660E0202F0E94F80E123081
:108BF00008F08DC09BE0C92E95E0D92E00E089E1F8
:108C0000882E912CBBE1EB2EA0E24A2E512CF0E8ED
:108C10002F2E312CF601219131916F013C832B8352
:108C2000113031F1802F83708E9DA02C1124F02EF5
:108C3000F694F694FF0CFF0CFF0C38E2F30E8B81D8
:108C40009C81B2010E9428769B018B819C81B1019D
:108C50000E942876AB01421B530B8B819C81480FED
:108C6000591F8A2D8F5D6F2D20E20E9428674AC010
:108C7000043018F4E2E2AE2E02C07EE5A72E802F6B
:108C80008370F82EFF0CFF0CF80E96E2F90E8B8124
:108C90009C8197FF03C0909581959F4F889DA0016F
:108CA000899D500D989D500D112440505E4F452FC9
:108CB000550F550B45954595642E4A3114F049E101
:108CC000642E8A2D89516F2D43E325E50E9464654A
:108CD0006F2D62508A2D45E00E949665EB81FC81E4
:108CE0001E161F0614F4A39401C0A6186F2D6F5F03
:108CF0008A2D462D0E9492656F2D61508A2D462D3A
:108D00000E9492650F5F083009F084CFAEC3163021
:108D100009F021C38091960E882309F414C3809131
:108D20002B088F5F80932B08823360F110922B0801
:108D300009E91EE037E2A32E38E0B32E23E2C22E6B
:108D400028E0D22EEE24FF24D8018C91F5018193E6
:108D50005F01F2E0EF16F10444F48E2D62E00E9410
:108D6000E372D60111969C938E930894E11CF11C3A
:108D70000C5F1F4FE2E0F0E0CE0EDF1EF4E0EF16D6
:108D8000F10411F780916C0190E080739070803154
:108D9000910509F0C9C097E2A92E94E0B92E8DEA99
:108DA000882E8EE0982E0AE9C02E0EE0D02E13E217
:108DB000612E18E0712E2224332410E0D5018C910D
:108DC000882309F453C001E0F30180819181009769
:108DD00009F400E0812F68E145E758E00E9414653E
:108DE000F22C422D4F5C812F8A5F68E10E94B164B2
:108DF000B2E14B2E410EF101E95DF74F0464812F82
:108E0000805F60E14081222DEE24E3940E946D108A
:108E1000F101EE0FFF1FEE0FFF1FE65DFB4F90818C
:108E20009295969596959370812F885E933041F434
:108E3000D4014D915C9160E220E00E94286709C056
:108E400060E2F6014081222D00E0EE24E3940E94CE
:108E50006D10842D8E5E60E2D60111964C912F2DFF
:108E600000E4EE24E3940E946D1010E40894211CA9
:108E7000311CE4E0F0E0AE0EBF1E26E030E0820ED2
:108E8000931ECE0EDF1E82E090E0680E791E92E007
:108E90002916310409F092CF8091970E882369F04A
:108EA00088E06FE678E00E940C654091D10E8EE17B
:108EB00068E050E020E40E94286780E36BE678E0F9
:108EC0000E940C654091290880E168E250E024E4AA
:108ED0000E9428674091A20E88E168E350E020E0FC
:108EE0000E9428674091A30E84E268E350E020E4EA
:108EF0000E94286780E460E347E658E00E9414651A
:108F000040912A0880E568E250E024E40E94286746
:108F10004091A60E88E568E350E020E00E942867B3
:108F20004091A70E84E6FDC08032910509F0FFC094
:108F30008091970E882309F4A5C080E163E678E06C
:108F40000E940C65E090CD0EF090CE0E80919601BF
:108F500085FF13C097012E5E3F4F83E790E0289F67
:108F60007001299FF00C389FF00C1124E6E0F59475
:108F7000E794EA95E1F716E401C013E48CE068E0B9
:108F8000412F0E94B16486E168E0A70124E40E94B9
:108F9000286784E568E34FE558E00E94146588E798
:108FA00068E3412F0E94B1644091D30E5091D40EDA
:108FB0008091960185FF11C09A012E5E3F4F83E795
:108FC00090E0289FA001299F500D389F500D11243B
:108FD00076E0559547957A95E1F786E668E320E4D3
:108FE0000E94286786E360E14AE558E00E94146524
:108FF0004091CF0E5091D00ECA01880F991F35E0D5
:10900000440F551F3A95E1F7481B590B8EE468E071
:1090100024E40E94286780E265E578E00E940C6500
:109020000091AF061091B0068091E90E9091EA0E82
:10903000080F191F80919601982F98719830A9F008
:1090400085FF15C0C80195958795959587959801D9
:10905000220F331F200F311F820F931FA5E015959C
:109060000795AA95E1F7080F191F46E601C04DE6DE
:1090700082E168E10E94B16488E168E1A80124E42A
:109080000E942867809127048823C1F080912308DB
:1090900090912408009711F003E001C000E080E304
:1090A00061E578E00E940C65046480E168E240912B
:1090B000270820E0EE24E3940E946D1080912B0499
:1090C0008823C9F08091250890912608009711F017
:1090D00003E001C000E080E460E34DE458E00E945A
:1090E0001465046482E568E24091280821E0EE24DA
:1090F000E3940E946D1088E369E478E00E940C65B7
:109100004091290882E168E350E020E40E9428674A
:1091100080E368E345E458E00E94146540912A0822
:1091200082E468E350E020E40E9428679EC1803317
:10913000910509F0ADC080E160E478E00E940C6523
:109140002091EF0E3091F00E442737FD4095542FBB
:1091500080E360E100E1FBEFEF2E0E94F26580E327
:1091600060E14EE20E94B1642091FF0E3091000F49
:10917000442737FD4095542F88E460E1ECEFEE2E54
:109180000E94F26588E16BE378E00E940C65209113
:10919000ED0E3091EE0E442737FD4095542F80E3BD
:1091A00068E17BEFE72E0E94F26580E368E14EE222
:1091B0000E94B1642091FD0E3091FE0E442737FDD0
:1091C0004095542F88E468E19CEFE92E0E94F265F7
:1091D00080E266E378E00E940C654091CB0E5091EE
:1091E000CC0E80E360E220E00E94286788E268E21B
:1091F00078E00E940C654091EB0E5091EC0E80E3FC
:1092000068E220E00E94286740911B0F88E768E22F
:1092100050E020E00E94286780E36CE178E00E9443
:109220000C6588E360E178E00E940C651CE1C12ECA
:109230001FE0D12E10E070E394E225C0133011F44A
:1092400078E394E2D6012D916D01809104042817F2
:1092500010F000E001C002E030E0220F331F44278D
:1092600037FD4095542F0063892F672FA4E0EA2E25
:1092700079839A830E94F26579819A81153009F485
:10928000F4C0965D1F5F8091280F1817B8F2EDC0EB
:10929000F7E2CF2EF4E0DF2EE3E2AE2EE8E0BE2EC2
:1092A0008824992415E1F6018081882321F1D501D4
:1092B0002D913C9111972115310511F003E401C066
:1092C00000E4812F68E24CE058E00E941465482DCC
:1092D0004F5C812F8A5F68E20E94B164F401E95D0E
:1092E000F74F812F8E5E68E24081282DEE24E394B3
:1092F0000E946D101BE40894811C911CE4E0F0E0D6
:10930000CE0EDF1E22E030E0A20EB31E32E0831646
:10931000910449F685E160E348E058E00E94146555
:109320004091290887E260E350E020E40E9428672A
:109330008BE460E344E058E00E94146540912A0801
:109340008DE560E3EFCE86E168E24CEF57E024E084
:109350000E94E5648AC0153008F07DC00E946A252D
:10936000123061F0812F880F810F880F8950912F63
:109370009150192F110F190F110F02C080E016E044
:10938000A82E992787FD90951C01220C331C280ECE
:10939000391E60E2F62ECC24DD2452E0652E712CBD
:1093A000680E791E2C011AC00E9419104C018A2DDA
:1093B00060E040E00E944311082FA401420D531DBC
:1093C0008AE06F2D23E00E94B5640894C11CD11C73
:1093D00083E090E0280E391E98E0F90EA394C601B0
:1093E000840D951D68167906FCF6812F992787FD57
:1093F00090952C01440C551C480E591E30E2F32E5A
:10940000CC24DD2422E0822E912C880E991E3C0172
:109410001AC00E9419105C01812F60E040E00E9498
:109420004311082FA501440D551D85E66F2D23E03E
:109430000E94B5640894C11CD11CA3E0B0E04A0EA0
:109440005B1EB8E0FB0E1F5FC601860D971D8816D8
:109450009906FCF60AC040918A0450918B048CE373
:1094600068E224E004E00E94F80E0F900F900F9045
:109470000F90CF91DF911F910F91FF90EF90DF90B0
:10948000CF90BF90AF909F908F907F906F905F90A4
:109490004F903F902F90089518161CF010920505DC
:1094A0000895282F332727FD309590910505291B16
:1094B0003109462F50E04217530724F4861B80934E
:1094C00005050895465050402417350724F48A5F57
:1094D000861B809305050895AF92BF92CF92DF92CD
:1094E000EF92FF920F931F93DF93CF930F92CDB71D
:1094F000DEB7D82E8BE89DE00E94871B86E898E0B7
:109500006D2D41E02CED37E00AE0A1E9EA2EADE057
:10951000FA2EFBE0CF2EE0E1AE2E0E94FF1C109150
:109520008608F0908708812F67E00E944C4A2091BE
:10953000570130E02F5F3F4F442737FD4095542FB0
:109540008AE260E001E172E0E72E0E94F2652D2DD3
:10955000253451F0263418F4243401F511C03D2D82
:10956000343671F03536D1F41130C1F4FF20B1F04A
:1095700080910605882391F08091870881500CC066
:10958000113061F44F2D493048F48091060588234D
:1095900029F0809187088F5F809387088091050567
:1095A000882309F088C088E066E87DE00E940C65A9
:1095B000113031F481E090E020910605222311F072
:1095C00080E090E0082F00618CE368E04AE851E019
:1095D0002AE00E94B56480910605882359F48091A1
:1095E000090587FF07C081E08093060510920905F1
:1095F0001092870880910605882381F02091090543
:10960000332727FD30958F2D90E08217930734F490
:10961000109206051092090510928708113009F082
:109620004DC080910605882309F448C080918708C1
:1096300090910905891B8093870887FF02C01092CB
:109640008708809187088A301CF089E0809387081A
:1096500010920905AF2CBB24F501E657FE4F80811F
:109660000E946E32682F209182043091830421156C
:10967000310549F47D2D723631F0733621F07234A4
:1096800011F0733431F48D2D40E021E40E949315E4
:10969000682F862F0E947E32482FF501E657FE4F35
:1096A00080838F2D880F8F0D880F845C68E021E008
:1096B0000E94F26303C048E0E42E02C030E1E32ED2
:1096C00080910505823008F084C08E2D60E87DE031
:1096D0000E940C654091970150919801123099F4C5
:1096E000FF2039F480910605882309F01AC421E08F
:1096F00019C48F2D813039F480910605882329F013
:1097000020E002E004C020E00DC420E001E087E496
:109710006E2D0E94F80E123009F059C08091060596
:10972000882339F48091820490918304009709F48E
:109730004EC0FF2029F09F2D913009F048C022C073
:1097400080919701909198012CE3A22EB12CB50144
:109750000E9414768D2D40E02BE30E9493152CE39C
:10976000482F420390011124809197019091980114
:10977000B5010E941476280F391F30939801209369
:10978000970125C080919701909198016CE370E05A
:109790000E941476082F0E5F8D2D602F41E02EE37E
:1097A0000E949315081B602F772767FD7095209105
:1097B000970130919801261B370B30939801209325
:1097C000970137FF04C0109298011092970168E04A
:1097D000E60E809105058330F8F48E2D68E77DE074
:1097E0000E940C6501E0133009F000E08CE36E2D5F
:1097F000402F0E941C10002349F08D2D609195018F
:1098000047EC29E30E9493158093950178E0E70ED9
:109810008E2D893308F088C3809105058430C8F502
:109820008E2D61E77DE00E940C6591E0143009F017
:1098300090E080919601282F217030E0A901440F1B
:10984000551FB3E0220F331FBA95E1F7420F531FA4
:10985000445A524F8CE36E2D2AE0092F99830E94BF
:10986000B5649981992379F06091960161708D2D8D
:1098700040E021E00E9493158170909196019E7FB7
:10988000982B9093960198E0E90EEE2DE93308F0BD
:109890004BC380910505853030F500919B010F7019
:1098A0008E2D65E57DE00E940C6521E0153009F004
:1098B00020E08CE36E2D402F0E94BA1C153069F415
:1098C0008D2D602F40E021E00E9493158F709091C4
:1098D0009B01907F982B90939B01F8E0EF0E2E2D2B
:1098E000293308F021C380910505863040F50091A9
:1098F0009B0102950F708E2D6EE47DE00E940C6539
:1099000021E0163009F020E08CE36E2D402F0E94FC
:10991000BA1C163071F48D2D602F40E021E00E94BA
:1099200093158295807F90919B019F70982B9093C7
:109930009B0138E0E30E4E2D493308F0F5C28091CB
:109940000505873050F58E2D65E47DE00E940C659D
:1099500091E0173009F090E040919C0186E04802C8
:10996000A00111244A5D524F8CE36E2D26E0092F91
:1099700099830E94B5649981992349F08D2D609156
:109980009C0140E024E00E94931580939C0168E0D4
:10999000E60E7E2D793308F0C7C280910505883028
:1099A00008F58E2D6EE17DE00E940C6501E0183017
:1099B00009F000E086E36E2D40919E01202F0E9469
:1099C000C90F002349F08D2D60919E014AEE26E1DA
:1099D0000E94931580939E0188E0E80E9E2D993396
:1099E00008F0A2C280910505893008F051C08E2D83
:1099F00065E17DE00E940C659CE3AA24BB24A501DF
:109A0000435F524FFA1411F4193061F020919F0115
:109A100030E00A2C02C0359527950A94E2F7022F10
:109A2000017001C002E0892F6E2D21E099830E9410
:109A3000B5640894A11CB11C99819A5F9636F9F619
:109A4000193001F5ED2DE03631F0809182049091CE
:109A500083040097B9F08D2D0E94F16810920605DD
:109A600081E090E00F2C02C0880F991F0A94E2F762
:109A700020919F01282720939F0182E00E94D65EBB
:109A80000E94725FF8E0EF0E2E2D293308F04CC2D1
:109A9000809105058A3008F0E3C08E2D67E07DE0F7
:109AA0000E940C654091990186E0489FA001112415
:109AB0004251534F1A3041F4FF2031F48091060592
:109AC000882321F002E003C000E001C001E084E24D
:109AD0006E2D26E00E94B56480919901882321F0C3
:109AE000833009F04DC009C086E66E2D49EE5CE07A
:109AF00020E00E94E5649CE308C082E76E2D46EEFC
:109B00005CE020E00E94E56498E440919A015527CA
:109B100047FD5095440F551F440F551F4F52534F4B
:109B20001A3049F43F2D313031F4809106058823F5
:109B300021F002E003C000E001C001E0892F6E2D9A
:109B400024E099830E94B5649981892F865D4091B4
:109B50009D0192E34902A0011124445D5E4F1A3039
:109B600049F46F2D623031F490910605992321F06C
:109B700022E003C020E001C021E06E2D0E94286792
:109B800080919901813001F582E46E2D42EC5CE018
:109B900020E00E94E56440919A01552747FD5095C9
:109BA0004F5F5F4F1A3049F47F2D713031F480914F
:109BB0000605882321F022E003C020E001C021E057
:109BC0008EE76E2D0E9428671A3009F043C08091FD
:109BD0000605882331F480918204909183040097D4
:109BE000C9F18F2D813079F0813018F0823091F5F4
:109BF00022C08D2D6091990140E023E00E949315D1
:109C00008093990127C080919901882311F08330B6
:109C100031F48D2D60919A014EEF24E007C0813020
:109C2000C9F48D2D60919A0140E02CE70E949315B4
:109C300080939A010FC080919901882311F083309D
:109C400049F48D2D60919D014CEF2AE00E949315FF
:109C500080939D0198E0E90EEE2DE93308F064C190
:109C6000809105058B3008F07AC080919901882396
:109C700011F0833019F58E2D63EB7CE00E940C65AA
:109C80004091A30185E04802A00111244F515F4F8C
:109C90001B3011F421E201C020E28EE46E2D0E94FF
:109CA00028671B3009F055C08D2D6091A3014CEE43
:109CB00024E10E9493158093A3014BC08130B9F435
:109CC00001E01B3009F000E080E06E2D4DE95CE022
:109CD000202F0E94E5640023E1F1FD2DF038C9F545
:109CE00081E08093620E80E00E942D7232C08E2D42
:109CF00064E97CE00E940C6580919A0187FD03C0B5
:109D000083301CF403C080E001C082E080939A019C
:109D100049E08402A00111244858534F1B3031F40C
:109D200080910605882321F002E003C000E001C015
:109D300001E08CE36E2D29E00E94B5641B3049F4EC
:109D40008D2D60919A0140E022E00E94931580934E
:109D50009A0128E0E20E3E2D393308F0E5C08091EB
:109D600005058C3098F58E2D6EE67CE00E940C6522
:109D700031E01C3009F030E08091A001817090E06A
:109D8000AC01440F551F480F591F4959534F8CE3DD
:109D90006E2D23E0032F39830E94B564398133236C
:109DA00079F06091A00161708D2D40E021E00E946A
:109DB000931581709091A0019E7F982B9093A001A4
:109DC00048E0E40E6E2D693308F0AEC080910505C1
:109DD0008D3040F50091A001069501708E2D6DE546
:109DE0007CE00E940C6521E01D3009F020E08CE34E
:109DF0006E2D402F0E94BA1C1D3071F48D2D602FE6
:109E000040E021E00E9493158170880F9091A0019D
:109E10009D7F982B9093A00178E0E70E8E2D8933DB
:109E200008F082C0809105058E3040F500919601C2
:109E3000069501708E2D65E57CE00E940C6521E0A1
:109E40001E3009F020E08CE36E2D402F0E94BA1CDA
:109E50001E3071F48D2D602F40E021E00E9493159B
:109E60008170880F909196019D7F982B9093960119
:109E700098E0E90EEE2DE93308F056C08091050513
:109E80008F3048F5009196010695069501708E2D4C
:109E90006CE47CE00E940C6521E01F3009F020E0BA
:109EA0008CE36E2D402F0E94BA1C1F3079F48D2D4B
:109EB000602F40E021E00E9493158170880F880F89
:109EC000909196019B7F982B90939601F8E0EF0E6E
:109ED0002E2D293348F580910505803128F5809194
:109EE0000705882319F421E0103109F020E080E013
:109EF0006E2D48E35CE00E94E5641031A9F43D2D2D
:109F0000303891F41092060589E18093070580E8C6
:109F10000E94F1681092210685E595E30E94F015F4
:109F200003C022E000E0F3CB0F90CF91DF911F91AF
:109F30000F91FF90EF90DF90CF90BF90AF9008957A
:109F40006F927F928F929F92AF92BF92CF92DF9249
:109F5000EF92FF920F931F93DF93CF930F92CDB7A2
:109F6000DEB7B82E86ED9FE00E94871B8CE998E053
:109F70006B2D46E02CED37E00AE076EEE72E7FE031
:109F8000F72ECC24C3945CE0A52E0E94FF1C809089
:109F90009C088A94D0909D08882D66E00E944C4AC7
:109FA00018E0CC24992487FC9094909105059C0D91
:109FB0009C3009F463C1E92EFF248E149F0439F408
:109FC00080910605882329F022E0A22E04C0AA244D
:109FD00002C0AA24A39480E0612F43ED5FE022E059
:109FE00000E099830E94B5649981993010F048E3AC
:109FF00001C041E3490F8CE0612F0E94B164F70179
:10A00000EE0FFF1FEE0DFF1DEE51FC4F408187E06C
:10A01000489FA00111244059504FDD2011F000E06D
:10A0200001C00A2D88E1612F27E00E94B564C701B5
:10A03000880F991F8E0D9F1D86579E4FFC01E85A71
:10A04000FD4F2081253008F40AC1FC01EA5AFD4F7A
:10A05000283008F40DC140819D2D913009F04DC08C
:10A060004EC020E001C02A2D88E4612F0E947D0FA0
:10A07000C701880F991F8E0D9F1D86579E4FFC01AB
:10A08000EA5AFD4F2081FC01E95AFD4F253254F078
:10A090004081552747FD509543585F4FED2DE230E5
:10A0A00041F409C04081552747FD5095FD2DF23000
:10A0B00011F020E001C02A2D88E7612F0E94286757
:10A0C00000E035C020E001C02A2D88E4612F0E9405
:10A0D000C90FF701EE0FFF1FEE0DFF1DEF51FC4FF3
:10A0E00040818D2D823011F020E001C02A2D80E6C4
:10A0F000612F0E94C90F01E01AC020E001C02A2D83
:10A1000088E4612F0E947D0FF701EE0FFF1FEE0D17
:10A11000FF1DEF51FC4F40819D2D923011F020E04A
:10A1200001C02A2D86E6612F0E947D0F02E08091FA
:10A130000605882339F48091820490918304009766
:10A1400009F486C0AA2009F483C0ED2DE130D1F1D5
:10A15000E13020F0E23009F07BC046C03701660CE8
:10A16000771C6E0C7F1C82EE93E0680E791E8B2D9F
:10A17000F301608140E02DE00E949315F30180839C
:10A18000202F30E0853028F0883030F481E090E0F6
:10A1900005C080E090E002C082E090E02817390717
:10A1A00009F456C0C701880F991F8E0D9F1D865751
:10A1B0009E4FFC01EA5AFD4F1082895A9D4FFC01C7
:10A1C000108246C0013041F0C701880F991FE80E88
:10A1D000F91E80EE93E031C03701660C771C6E0CDF
:10A1E0007F1C80EE93E01AC0013089F0C701880F10
:10A1F000991F0230F1F0E80EF91E81EE93E0E80EAF
:10A20000F91E8B2DF701608143E82DE71DC0370152
:10A21000660C771C6E0C7F1C81EE93E0680E791E35
:10A220008B2DF30160814AEE26E10E949315F30124
:10A230000EC0E80EF91E81EE93E0E80EF91E8B2D9C
:10A24000F701608140E026E20E949315F7018083C8
:10A25000C394185FFC2DF73009F0A7CE0FC08A5ABF
:10A260009D4FFC014081FD2DF13009F0FACEFBCE6F
:10A2700040818D2D813009F025CF26CF0F90CF91D1
:10A28000DF911F910F91FF90EF90DF90CF90BF90E3
:10A29000AF909F908F907F906F9008956F927F9274
:10A2A0008F929F92AF92BF92CF92DF92EF92FF92E6
:10A2B0000F931F93CF93DF93982E88EE9FE00E9419
:10A2C000871B8EE998E0692D47E02CED37E00AE026
:10A2D00018EFE12E1FE0F12ECC24C394B0E1AB2E99
:10A2E0000E94FF1C60909E086A9480909F08862DB3
:10A2F00066E00E944C4AA8E0FA2EDD24772467FC31
:10A300007094409105054D0D403109F45DC0A42EB7
:10A31000BB244F5F80E06F2D20E00E94A90FEE2448
:10A32000E501CC0FDD1FC85FDB4F8501000F111F5A
:10A33000095F1B4F6A147B0471F48E1461F48091E1
:10A340000605882359F48091820490918304009734
:10A3500039F421E001C020E0CC2405C022E001C096
:10A3600021E0CC24C394EE2091F48EE16F2DF8010E
:10A3700040810E94C90FCC20D9F0892DF80160815D
:10A380004AEE26E10E949315F801808311C04881AE
:10A39000552747FD509580E66F2D0E942867CC20F9
:10A3A00039F0892D688143E82DE70E949315888351
:10A3B000E394FE2DF33009F0BDCFD39488E0F80E7E
:10A3C000ED2DE73009F09DCFDF91CF911F910F91D7
:10A3D000FF90EF90DF90CF90BF90AF909F908F90C5
:10A3E0007F906F900895AF92BF92CF92DF92EF92DD
:10A3F000FF920F931F93DF93CF9300D0CDB7DEB7BB
:10A40000182F90917901992321F08AEF913011F45E
:10A4100003C08BEF58E101C05BE19150923030F402
:10A420009091700197FF02C05D5F8350F82EF50E8A
:10A430008DE39BE059830E94871B8DE398E0612F99
:10A4400040E020EF37E006E05981E52E0E94ED2341
:10A45000D0903D08C0903E088D2D67E00E944C4A88
:10A46000609105055981852F90E0462F50E09C01B1
:10A47000275030404217530761F42D2D30E00497E8
:10A480002817390714F48FEF01C081E0680F60933B
:10A490000505113629F1123678F4143409F448C050
:10A4A000153420F4123408F46AC063C0153419F16D
:10A4B000103609F064C009C0143608F45AC01436C6
:10A4C000B9F1153609F05BC016C0DD2009F457C09C
:10A4D00081E090910605911180E0809306054FC0C0
:10A4E00080910605882309F44AC01092060581E68A
:10A4F0000E94F16844C02D2D213059F4CC2049F040
:10A5000080910605882329F080913E088150809330
:10A510003E082D2D30E08F2D992787FD9095281727
:10A52000390769F5CC2059F180913E0881501EC051
:10A530003D2D313061F48C2D893048F48091060531
:10A54000882329F080913E088F5F80933E082D2D4F
:10A5500030E08F2D992787FD90952817390779F4DA
:10A560009C2D973060F480913E088F5F80933E0869
:10A5700006C080910605882311F410923E08809150
:10A580000505882309F089C088E062E37BE00E942A
:10A590000C65ED2DE13031F481E090E0209106056D
:10A5A000222311F080E090E0082F006182E468E04F
:10A5B0004BE751E02AE00E94B564809106058823AC
:10A5C00059F48091090587FF07C081E08093060553
:10A5D0001092090510923E0880910605882381F0AB
:10A5E00020910905332727FD30958C2D90E08217A7
:10A5F000930734F4109206051092090510923E0854
:10A60000FD2DF13009F04CC080910605882309F436
:10A6100047C080913E0890910905891B80933E08B0
:10A6200087FF02C010923E0880913E088A301CF0DD
:10A6300089E080933E0810920905EC2CFF24F70175
:10A64000E558FE4F80810E946E32682F209182046F
:10A65000309183042115310541F4123631F013365F
:10A6600021F0123411F0133431F4812F40E021E451
:10A670000E94A215682F862F0E947E32482FF70174
:10A68000E558FE4F80838C2D880F8C0D880F8E5BD4
:10A6900068E021E00E94F26303C028E0F22E02C0CD
:10A6A00090E1F92E809105058230A0F5E0906D01D2
:10A6B000E694E694E69427E0E2228F2D6BE27BE0BD
:10A6C0000E940C6591E03D2D323009F090E046E0AB
:10A6D0008E2D849FA00111244050554F8CE56F2D85
:10A6E00026E0092F9A830E94B5649A81992381F00C
:10A6F000812F6E2D40E026E00E94A2158770880F02
:10A70000880F880F90916D01977C982B90936D0125
:10A7100098E0F90E80910505833058F5E0907901B5
:10A720008F2D65EF7AE00E940C6591E0ED2DE3300E
:10A7300009F090E046E0FE2DF49FA001112448515D
:10A74000554F8CE56F2D26E0092F9A830E94B56442
:10A750009A81992341F0812F6E2D40E021E00E94E3
:10A76000A2158093790128E0F20E3F2D393308F0CD
:10A77000A8C480917901813041F58091050584302C
:10A7800030F58F2D6AED7AE00E940C6540917701DB
:10A790008D2D843011F421E401C020E486E66F2D74
:10A7A00050E00E9428679D2D943049F4812F6091DC
:10A7B000770141E024E60E94A21580937701E8E04A
:10A7C000FE0EFF2DF93318F07CC404E001C005E053
:10A7D000809179018150823038F58091050580178C
:10A7E00010F58F2D6AEC7AE00E940C65409178019B
:10A7F000D01611F421E401C020E486E66F2D50E06C
:10A800000E942867D01649F4812F6091780140E0BA
:10A8100025E00E94A2158093780128E0F20E3F2DDA
:10A82000393308F04EC40F5F80910505801720F57D
:10A830008F2D61EC7AE00E940C6540915801D01692
:10A8400011F421E401C020E486E66F2D50E00E945F
:10A850002867D01659F4812F609158014AE02DE203
:10A860000E94A215809358010E94886788E0F80E24
:10A870009F2D993308F025C4E02EE39480910505BF
:10A880008E1508F58F2D61EB7AE00E940C654091E2
:10A890005901DE1411F421E401C020E486E66F2D95
:10A8A0000E94630FDE1449F4812F6091590148E240
:10A8B00028E70E94A21580935901E8E0FE0EFF2DC3
:10A8C000F93308F0FEC3E394809105058E1560F519
:10A8D0008F2D60EA7AE00E940C6540916F01552748
:10A8E00047FD5095465F5F4FDE1411F421E401C02F
:10A8F00020E486E66F2D0E94286780919E0D6F2DC3
:10A900004DE60E94B164DE1449F4812F60916F011D
:10A9100046EF2EE60E94A21580936F0128E0F20E0A
:10A920003F2D393308F0CDC3E394809105058E1592
:10A9300050F58F2D65E97AE00E940C6591E0DE10FC
:10A9400090E04091710150E0440F551F440F551F96
:10A950004857554F86E66F2D24E0092F9A830E94B1
:10A96000B5649A81992349F0812F6091710140E08B
:10A9700022E00E94A2158093710188E0F80E9F2DBD
:10A98000993308F09EC3E394809105058E15C8F4B1
:10A9900080917001817021E0DE1020E06F2D47E78B
:10A9A0005AE0012F0E9488328170909170019E7F41
:10A9B000982B90937001E8E0FE0EFF2DF93308F01C
:10A9C00080C3E394809105058E15D8F480917001C1
:10A9D0008695817021E0DE1020E06F2D4BE65AE075
:10A9E000012F0E9488328170880F909170019D7FA5
:10A9F000982B9093700128E0F20E3F2D393308F028
:10AA000060C3E394809105058E15E8F48091700190
:10AA100086958695817021E0DE1020E06F2D4CE553
:10AA20005AE0012F0E9488328170880F880F909120
:10AA300070019B7F982B9093700188E0F80E9F2DFA
:10AA4000993308F03EC3E394809105058E15F8F420
:10AA500080917001869586958695817021E0DE1043
:10AA600020E06F2D4EE45AE0012F0E948832817061
:10AA7000880F880F880F90917001977F982B909383
:10AA80007001E8E0FE0EFF2DF93308F01AC3E394DD
:10AA9000809105058E1500F58F2D61E47AE00E9406
:10AAA0000C6501E0DE1000E080E66F2D40915B0157
:10AAB000202F0E94C90F002349F0812F60915B0174
:10AAC0004AEE26E10E94A21580935B0128E0F20E77
:10AAD0003F2D393308F0F5C2E394BB24809105057E
:10AAE0008E1508F048C0BB2019F461E37AE002C07B
:10AAF00061E27AE08F2D0E940C65BB2019F4A090D2
:10AB0000720102C0A0907A01AA20A9F08A2D95E0D6
:10AB1000899FA0011124DE1411F421E401C020E476
:10AB200086E66F2D0E94286780919E0D6F2D43E76A
:10AB30000E94B1640AC001E0DE1000E086E66F2DDD
:10AB40004DE15AE023E00E94B564DE1439F4812F10
:10AB50006A2D40E028E70E94A215A82EBB2019F418
:10AB6000A092720102C0A0927A01E8E0FE0EFF2DD1
:10AB7000F93308F0A6C2E394B3942B2D223009F0E8
:10AB8000ADCF809105058E15F8F480917001829506
:10AB90008F708095817021E0DE1020E06F2D4FE0F6
:10ABA0005AE0012F0E948832809581708295807FC3
:10ABB000909170019F7E982B9093700138E0F30E76
:10ABC0008F2D893308F07DC2E394809105058E15A1
:10ABD000F8F48091760182958F708095817021E0E4
:10ABE000DE1020E06F2D43E05AE0012F0E948832F2
:10ABF000809581708295807F909176019F7E982BC1
:10AC00009093760198E0F90EEF2DE93308F059C2E0
:10AC1000E394809105058E15D8F480916D0180959F
:10AC2000817021E0DE1020E06F2D42EF59E0012F0E
:10AC30000E9488328095817090916D019E7F982B43
:10AC400090936D01F8E0FF0E2F2D293308F039C2E3
:10AC5000E394809105058E15E8F480916D01869549
:10AC60008095817021E0DE1020E06F2D43EE59E0E9
:10AC7000012F0E94883280958170880F90916D011C
:10AC80009D7F982B90936D0138E0F30E8F2D8933C3
:10AC900008F017C2E394809105058E1508F086C070
:10ACA0008F2D68ED79E00E940C6592E4AA24BB2404
:10ACB000A5014153564FE0918501F0E00A2C02C0F6
:10ACC000F595E7950A94E2F7E170F070892F6F2D02
:10ACD00021E00E2F9A830E94B5640894A11CB11C38
:10ACE0009A819A5F923721F7DE1409F059C080915A
:10ACF0003E0890910905891B80933E0887FF02C09A
:10AD000010923E0880913E088A301CF089E08093C2
:10AD10003E08109209058C2D880F8C0D880F4C2D44
:10AD200050E04A53564F8E5B6F2D21E002E00E94A7
:10AD3000B564103631F080918204909183040097BD
:10AD400079F1812F0E94F1681092060581E090E070
:10AD500002C0880F991FCA94E2F790918501982745
:10AD600090938501803151F0803271F0883099F4F0
:10AD700093FF02C09F7C0DC098600BC094FF02C07F
:10AD8000977D07C0906105C095FF02C0977E01C006
:10AD900090629093850181E00E94D65E0E94725F6E
:10ADA00098E0F90EEF2DE93308F08BC1E394809120
:10ADB00005058E15F8F480916D0186958695809530
:10ADC000817021E0DE1020E06F2D47EB59E0012F6C
:10ADD0000E94883280958170880F880F90916D0154
:10ADE0009B7F982B90936D01F8E0FF0E2F2D293358
:10ADF00008F067C1E394809105058E1500F59091E8
:10AE00006D01991F9927991F81E0891B21E0DE10B0
:10AE100020E06F2D49EA59E0012F0E948832809589
:10AE200087958827879590916D019F77982B9093B0
:10AE30006D0138E0F30E8F2D893308F042C1E394A1
:10AE4000809105058E1508F5809170018295869593
:10AE500087708095817021E0DE1020E06F2D4FE932
:10AE600059E0012F0E948832809581708295880F69
:10AE7000807E909170019F7D982B9093700198E057
:10AE8000F90EEF2DE93308F01CC1E394809105051C
:10AE90008E1518F580917001829586958695837040
:10AEA0008095817021E0DE1020E06F2D47E959E0A8
:10AEB000012F0E948832809581708295880F880FBB
:10AEC000807C909170019F7B982B90937001F8E0AB
:10AED000FF0E2F2D293308F0F4C0E39480917901FF
:10AEE0008150823048F5809105058E1520F5C0907F
:10AEF0007001CC1CCC24CC1C21E0DE1020E08C2D79
:10AF00006F2D46E859E0012F0E9488328170282F6A
:10AF1000279522272795909170019F77922B9093E8
:10AF20007001C81611F00E94B87538E0F30E8F2D2D
:10AF3000893308F0C6C0E394809179018150823052
:10AF400008F075C08091700187FF71C0CC2480919A
:10AF50007501982F9F70209105052E1508F061C08E
:10AF6000CC2029F4B92E8F2D6AE779E012C09C2DF0
:10AF7000913041F4B82EB2940FE0B0228F2D6EE6DE
:10AF800079E007C0B0907601EFE0BE228F2D62E637
:10AF900079E00E940C6591E0DE1090E0FB2D26E048
:10AFA000F29FA00111244F5F564F8CE56F2D092FA2
:10AFB0009A830E94B5649A81992369F1812F6B2D40
:10AFC00040E02FE00E94A215682FCC2031F4982F8A
:10AFD0009F7080917501807F09C03C2D313051F404
:10AFE000982F9295907F809175018F70892B809317
:10AFF000750108C0982F9F7080917601807F892B02
:10B000008093760180917F04882329F08FE294E079
:10B0100046E40E94BA7088E0F80E9F2D993308F03C
:10B0200050C0E394C394EC2DE33009F090CF8091AD
:10B0300005058E1508F045C086E06F2D4CEF58E0F1
:10B040000E941465FF2DF83390F434E290E0832FD2
:10B050006F2D41E957E0292F00E039839A830E9440
:10B0600093639A819F5F3981385E943081F728E03D
:10B07000F20E3F2D393328F5CC24C394DE10CC24B6
:10B0800040916E014F5C82E16F2D2C2D0E94F26386
:10B0900094E200E00F5F892F6F2D402F20E09A830C
:10B0A0000E947D0F9A81985E0430A1F7CC2049F070
:10B0B000812F60916E0140E023E00E94A2158093F1
:10B0C0006E010F900F90CF91DF911F910F91FF9024
:10B0D000EF90DF90CF90BF90AF9008954F925F9226
:10B0E0006F927F928F929F92BF92CF92DF92EF9258
:10B0F000FF920F931F93DF93CF9300D0CDB7DEB7AE
:10B10000182F85EC90E10E94871B86EB98E0612F59
:10B1100045E02CED37E00AE070E1E72E0E94ED23D8
:10B120006090B6086A94862D66E00E944C4A1036FC
:10B1300011F0143641F467FC06C0609299088FEB59
:10B1400097E30E94F015CC24DD24EE24E39458E02C
:10B15000F52E772467FC7094309105053C0DBB24D7
:10B16000B394383028F4BB248E2D883028F074C076
:10B170009E2D973008F070C0032F10E091E060160C
:10B18000710609F090E0DD2019F0DD24D39401C0B0
:10B19000D92E80E06F2D42EC50E1292F3A8399831C
:10B1A0000E94E5643A819981393010F482E101C04E
:10B1B00087E1A8014F5F5F4F6F2D292F0E942867FD
:10B1C000BB2079F008501040280143E0440C551C86
:10B1D0004A95E1F7400E511EE8E9F3E04E0E5F1E7E
:10B1E0000BC02801440C551C440C551C400E511E2C
:10B1F00080E793E0480E591E42010AE2F4014191B2
:10B200004F01552747FD5095802F6F2D20E00E945C
:10B2100028670B5E033991F7F8E0FF0EE394BB203B
:10B22000B1F085E090E0480E591E0AE2F20141912A
:10B230002F01552747FD5095802F6F2D20E00E944C
:10B2400028670B5E0E3791F7F8E0FF0EE394C39486
:10B250008C2D873009F080CFDD2029F48091050501
:10B260008F5F809305050F900F90CF91DF911F9115
:10B270000F91FF90EF90DF90CF90BF909F908F90B5
:10B280007F906F905F904F900895AF92BF92CF9252
:10B29000DF92EF92FF920F931F93CF93DF93F82EDD
:10B2A0008AE998E06F2D4DE00E945E25809192081A
:10B2B000882319F084E69FE002C08AE59FE00E949F
:10B2C000871B182F809193080E94DC0EEC01812FC0
:10B2D0008A5F60E0488120E00E94A90FA0909A0850
:10B2E0008A2D66E00E944C4A18E0EE24BB24A7FC9D
:10B2F000B094209105052E0D822F90E0DD24D3948B
:10B30000A816B90609F0DD24263009F4FAC0273062
:10B3100090F4223009F457C0233030F4222309F18D
:10B32000213009F0E8C134C0243009F499C0253037
:10B3300008F0BAC069C02A3009F46BC12B3038F468
:10B34000283009F420C1293008F044C1F1C02C3064
:10B3500009F49CC12C3008F47AC12D3009F0CBC11E
:10B36000B2C18CE0612F43E55FE00E94146584E583
:10B37000612F49812D2D0E947D0FDD2009F4BBC175
:10B380008F2D698141E026E20E9493158983B3C124
:10B390008CE0612F4CE45FE00E9414654A815527E0
:10B3A00047FD50952D2D206484E5612F0E9428676C
:10B3B000DD2009F4A0C18F2D6A8143E82DE70E94AA
:10B3C00093158A8398C18F8186FF03C042E45FE0B2
:10B3D00002C04BE35FE08CE0612F0E94146548855A
:10B3E000552747FD50952D2D206484E5612F0E943F
:10B3F0002867DD2009F47FC18F2D688543E82DE79C
:10B400000E949315888777C1CF80C294C694C69452
:10B41000A3E0CA2281E0C8228CE0612F40E35FE014
:10B420000E94146543E09C2D949FA0011124475D68
:10B43000504F84E5612F23E00D2D0E94B564DD207F
:10B4400009F459C18F2D6C2D40E021E00E94931525
:10B4500081708295880F880F807C9F819F7B90C030
:10B460008CE0612F44E25FE00E9414658F8181705F
:10B4700090E0AC01440F551F480F591F435E504FD9
:10B4800084E5612F23E00D2D0E94B564DD2009F4D1
:10B4900032C16F8161708F2D40E021E00E949315D1
:10B4A00081709F819E7F6CC08CE0612F46E15FE0E0
:10B4B00020E00E94E5644C8183E0489FA0011124B4
:10B4C00040515F4E84E5612F23E00D2D0E94B5644D
:10B4D000DD2009F410C18F2D6C8140E026E10E942F
:10B4E00093158C83873008F406C19F2D903609F0A0
:10B4F00002C18750809399088FEB97E30E94F01563
:10B50000FAC08CE0612F4FE05FE00E9414658EE48A
:10B51000612F4B812D2D0E94C90FDD2009F4EBC056
:10B520008F2D6B814AEE26E10E9493158B83E3C039
:10B530008CE0612F47E05FE00E9414650F81029567
:10B54000037049F02D2D206484E5612F402F50E0D9
:10B550000E94286707C084E5612F43E05FE02D2D3E
:10B560000E94E564DD2009F4C6C08F2D602F40E005
:10B5700023E00E94931583708295807F9F819F7C3A
:10B58000982B9F83B8C08CE0612F4CEF5EE00E9447
:10B5900014654F814695477050E0E3E0440F551F16
:10B5A000EA95E1F74D51514F84E5612F28E00D2DCB
:10B5B0000E94B564DD2009F49EC06F8166956770B6
:10B5C0008F2D40E022E00E9493158770880F9F81A5
:10B5D000917FD6CF8CE0612F48ED5EE00E9414652C
:10B5E0004D8142954F7080E6612F50E02D2D0E94D5
:10B5F0002867DD2009F47FC06D8162956F708F2D03
:10B6000040E02FE00E9493158295807F9D819F707E
:10B610001BC08CE0612F4FEC5EE00E9414654D81F1
:10B620004F7080E6612F50E02D2D0E942867DD20AD
:10B6300009F461C06D816F708F2D40E02FE00E9492
:10B6400093158F709D81907F982B9D8354C08CE0C3
:10B65000612F44EC5EE00E9414654E8142954F706C
:10B6600080E6612F50E02D2D0E942867DD2009F42F
:10B6700042C06E8162956F708F2D40E02FE00E9476
:10B6800093158295807F9E819F701AC08CE0612FF8
:10B690004BEB5EE00E9414654E814F7080E6612F97
:10B6A00050E02D2D0E942867DD2029F16E816F70FA
:10B6B0008F2D40E02FE00E9493158F709E81907F28
:10B6C000982B9E8318C08CE0612F49EA5EE02D2DF7
:10B6D0000E94E564DD2079F08F2D803861F40E94AE
:10B6E000F168809193080E947B2781E00E942D726F
:10B6F00080E00E94BB15E394185F9E2D973009F0FF
:10B70000F8CDDF91CF911F910F91FF90EF90DF90D7
:10B71000CF90BF90AF9008955F926F927F928F927B
:10B720009F92AF92BF92CF92DF92EF92FF920F93D0
:10B730001F93CF93DF93D82E89EA90E10E94871B55
:10B7400084EB98E06D2D44E02CED37E00AE0E0EB6F
:10B75000EE2EE0E1FE2E71E1C72E51E1A52E0E94F2
:10B76000FF1CF090B408FA948090B5088F2D66E025
:10B770000E944C4A8D2D803821F59F2D903108F57F
:10B78000EF2DFF27E7FDF09580910505E81BF109F6
:10B79000EE0FFF1FE55FFA4FC081D1818F2D0E9410
:10B7A000EC0EFC01882069F48281882319F0D09581
:10B7B000C195DF4FD483C38382E00E94D65E0E948E
:10B7C000725F18E09924552453946F2C772467FCFA
:10B7D000709400910505090D003109F4E1C0802F36
:10B7E0000E94EC0EEC018A816B817C81882319F028
:10B7F000709561957F4FA02EBB24F501EE0FFF1FC2
:10B80000E55FFA4F20813181261B370B2333310549
:10B8100024F0F501EC55F74F08C09FEF2E3C390797
:10B820002CF4F501EC55F74F85258083402F4F5FB1
:10B8300080E0612F20E00E94A90FF501EC55F74F41
:10B840008081882311F04FE701C04EE78BE4612F20
:10B8500020E00E94F263EE246A147B0471F48E14DB
:10B8600061F480910605882359F4809182049091B7
:10B870008304009739F401E001C000E0CC2405C046
:10B8800002E001C001E0CC24C3948E2D823009F483
:10B890003FC0833009F45DC08130C1F04B815C81D1
:10B8A000202F206280E3612F0E942867CC2009F4BA
:10B8B0006BC06B817C818D2D48E15CEF28EE33E01D
:10B8C00002E00E94CF149C838B835EC04881445663
:10B8D000552747FD509588E4612F202F0E94286747
:10B8E000CC2009F451C06881645668838091A0011E
:10B8F00081FF04C08D2D43E82DE703C08D2D4CE959
:10B9000024E60E949315888388818C5988833CC0E3
:10B9100049814C59552747FD509586E6612F202FC8
:10B920000E942867CC2081F169816C5969838091DC
:10B93000A00181FF04C08D2D43E82DE703C08D2DAC
:10B940004CE924E60E949315898389818456898372
:10B950001BC08A8190E0AC01440F551F480F591F4E
:10B960004E555F4E8CE6612F23E00E94B564CC20DB
:10B9700059F08D2D6A8140E021E00E94931591E0FD
:10B98000882309F490E09A83E3949E2D943009F083
:10B9900063CF9394185F892D873009F01ACF1FC0A9
:10B9A00001E09F2D903109F000E080910705882388
:10B9B00011F020E001C0202F82E1612F41E950E128
:10B9C0000E94E564002359F08D2D803841F489E10F
:10B9D0008093070580E80E94F1680E947C43DF9114
:10B9E000CF911F910F91FF90EF90DF90CF90BF907C
:10B9F000AF909F908F907F906F905F900895F89494
:10BA00002091CC0D3091CD0D7894C9010895CF933C
:10BA1000DF93CAE2D1E080E6FE0111928A95E9F750
:10BA20008AE080932A0189E1809358018AE5809316
:10BA3000590181E080936E012196FE0120E032E001
:10BA400080E891E02193319395878487938F828F4B
:10BA500041E0E933F407B1F78BE791E062E971E186
:10BA60004AE050E00E947E7680E090E02991399192
:10BA7000820F931FE1E0C334DE07C1F790935601B4
:10BA800080935501DF91CF9108951F93CF93DF935A
:10BA90008FEB98E060E00E9432616AE271E080E63C
:10BAA000FB0111928A95E9F78FEB98E040E650E0B0
:10BAB0000E94BE61182FCBE7D1E088810E946E32D0
:10BAC0000E947E328993F1E0C538DF07B1F780919B
:10BAD0002A018A3028F4809167048160809367048A
:10BAE0008AE080932A011D3468F0EBE2F1E020E067
:10BAF00030E081919191280F391F81E0E334F807FC
:10BB0000C1F702C020E030E081E040915501509142
:10BB100056014217530709F080E0DF91CF911F9142
:10BB200008951F93182FEAE8F1E025EA32E0DF01DB
:10BB3000C9011D920197E9F7CF0167E871E14AE079
:10BB400050E00E947E76812F90E001966AE070E0DE
:10BB50000E942876605D60938F01805D80939001E4
:10BB60008AE08093940180E00E94C8691F91089543
:10BB7000CF92DF92EF92FF920F931F93DF93CF93B9
:10BB80000F92CDB7DEB76B01803160F5682F6F5F24
:10BB90008FEB98E049830E9432614981042F10E0C5
:10BBA000C60160E270E050E00E949F768FEB98E063
:10BBB000B6014AE050E00E94BE618A30910591F4DE
:10BBC0008FEB98E00E942461F601E00FF11F2AE05C
:10BBD00030E006C0B9010E941476805D8293CB01EB
:10BBE0000097C1F70F90CF91DF911F910F91FF90B8
:10BBF000EF90DF90CF9008958F5F0E94B560089519
:10BC00001F93CF93DF93182F8031A0F5682F6F5FBC
:10BC10008FEB98E00E9432616AE871E025EA32E039
:10BC2000FB01C90111920197E9F78FEB98E045EA12
:10BC300052E00E94BE618F3F910509F018F4812FF8
:10BC40000E94915DCAE8D1E088810E946E320E9414
:10BC50007E32899391E0C439D907B1F78AE08093A5
:10BC600094010E942F1680912A0F806480932A0FDE
:10BC70000E94B875DF91CF911F9108950F931F9384
:10BC8000DF93CF93CDB7DEB760970FB6F894DEBFE2
:10BC90000FBECDBF682F6F5F062F0AC0102F1F5F2A
:10BCA000812F688B0E94B5606889882329F0012F55
:10BCB0000031A0F3003139F18FEB98E00E9432613E
:10BCC000602F6F5F88EC98E042E028E532E00E9448
:10BCD000A4628E010F5F1F4F06C088EC98E0B80188
:10BCE0000E941F62A8958FEB98E0B8014FE050E0EA
:10BCF0000E944D61482F882381F788EC98E00E94CC
:10BD0000CD6281E001C080E060960FB6F894DEBF9E
:10BD10000FBECDBFCF91DF911F910F910895EF928C
:10BD20000F931F930E94A060882341F00E940B6034
:10BD300087FD04C00E94455D882381F587E791E176
:10BD400061E00E949E1385E691E10E9485130E94A6
:10BD50007A600E94075D8FEB98E060E041E02AE2A4
:10BD600031E000E610E078ECE72E0E94FC628036BD
:10BD7000910529F086E591E160E00E949E1380E044
:10BD80000E94915D8FEB98E061E042E02AE831E0AB
:10BD900005EA12E058ECE52E0E94FC628091570102
:10BDA0000E94005E1F910F91EF900895882359F033
:10BDB0009091DB08982B9093DB080E94D40E90930F
:10BDC000DD088093DC080895EF920F931F93CF93C3
:10BDD000DF931091DB08112309F47EC0882309F05A
:10BDE00076C00E94D40E2091DC083091DD08AC01B1
:10BDF000421B530B4436510508F46EC068C081E005
:10BE00008093DA08812F90E0EC01C470D07012FFAB
:10BE100003C023E02093DA081092DB0880FF1CC0E7
:10BE200081ED98E061E141E02AE231E000E610E0D6
:10BE3000F4E1EF2E0E94FC628036910511F480E05F
:10BE400020C08091D708823021F48091DB08816086
:10BE500029C086E491E135C081FF36C081ED98E0CC
:10BE600061E142E02AE831E005EA12E0E4E1EE2E89
:10BE70000E94FC6252E0853A950739F4809157019F
:10BE80008F5F61E10E94C3601FC08091D70882303C
:10BE9000A1F48091DB08982F92609093DB082097A3
:10BEA00019F086608093DB080E94D40E845690407F
:10BEB0009093DD088093DC0807C0209729F486E37F
:10BEC00091E160E00E949E131092DA0805C0809113
:10BED000DA08882309F493CFDF91CF911F910F9156
:10BEE000EF9008950AC081E00E94E45E8091600EA8
:10BEF000833019F4A8951092600E8091DB08882396
:10BF000091F70895DF93CF930F92CDB7DEB7682FE7
:10BF100070E084E0660F771F8A95E1F7CE01019605
:10BF200041E050E00E94A67689810F90CF91DF9189
:10BF30000895DF93CF930F92CDB7DEB76983682F53
:10BF400070E094E0660F771F9A95E1F7CE010196B5
:10BF500041E050E00E94C5670F90CF91DF910895B6
:10BF60008EED98E060E070E040E450E00E94C5672C
:10BF7000089580EE98E062E070E041E050E00E94B9
:10BF8000C56708950F931F93182F082F04C0802FA3
:10BF90000E94825F082F802F0E94825F8823B9F75A
:10BFA000802F6091E0080E94995F1093E0080E9442
:10BFB000B95F1F910F9108951F931091E00811230D
:10BFC00059F0812F0E94825F8093E0080E94B95F40
:10BFD000812F60E00E94995F812F1F910895F8944E
:10BFE0002091CC0D3091CD0D7894C9010895EF9238
:10BFF000FF92CF93DF938091E008C0E0D0E003C0D0
:10C000002F960E94825F8823D9F7CE01DF91CF91CE
:10C01000FF90EF900895CF92DF92EF92FF920F93EF
:10C020001F93CF93DF9380E8EEE1F9E0DF011D92EB
:10C030008A95E9F702EE18E0C0E0D0E08C2FC43119
:10C0400039F4D090E00830EEE32E38E0F32E0BC048
:10C050007E01EE0CFF1CEC0EFD1E22EE38E0E20E1F
:10C06000F31ED801DC9090E0C82EC3941DC08D2D26
:10C0700084508C3738F4ED2DF0E0E25EF64F80818D
:10C08000882361F0992329F0892F60E00E94995F4D
:10C090000DC0F70110820E94B05F08C0C0828D2DD4
:10C0A0000E94825F9D2DD82EDD2009F721960D5F1D
:10C0B0001F4FC531D10511F604E0E02FF0E0E25E3C
:10C0C000F64F8081882349F4802F6091E0080E9418
:10C0D000995F0093E0080E94B95F0F5F003869F72D
:10C0E00080E0DF91CF911F910F91FF90EF90DF9053
:10C0F000CF9008951F9380E4EEEDF8E0DF01982FD4
:10C100001D929A95E9F794E09093DE088093DF08FA
:10C1100080E18093E10884E001C0812F182F1F5F28
:10C12000612F0E94995F1038C1F78FE760E00E948D
:10C13000995F84E08093E0080E94B05F1F910895AA
:10C140008EED98E060E070E040E450E00E94A6765A
:10C150008091DE08843039F481E09091DF089034DA
:10C1600019F080E0089580E0089590E0FC01EE0F62
:10C17000FF1FE80FF91FE252F74F81E094819923E6
:10C1800009F480E00895DF93CF9300D00F92CDB7EC
:10C19000DEB790E0FC01EE0FFF1FE80FF91FDE0194
:10C1A0001196EE51F74F23E001900D922150E1F7E7
:10C1B00070E0DC01AA0FBB1FA80FB91FFB01EE0F37
:10C1C000FF1FE60FF71FAE51B74FEE51F74F83E059
:10C1D00001900D928150E1F7FB01EE0FFF1FE60F7A
:10C1E000F71FEE51F74FDE01119683E00D9001929B
:10C1F0008150E1F70E94B05F0F900F900F90CF91A8
:10C20000DF910895DF93CF930F92CDB7DEB790E023
:10C210009C01220F331F280F391FF901E252F74FFB
:10C2200084812E51374F93E0D9011D929A95E9F7F9
:10C2300089830E94B05F8981882311F00E94C25FC8
:10C240000F90CF91DF910895FC01808190E0FC0177
:10C25000EE0FFF1FE80FF91FED51F74F918180811D
:10C260009F700895FC0160831282118270E0CB01FF
:10C27000880F991F860F971FDC01A252B74F1496A3
:10C280002C91149723831482158216828C51974F18
:10C29000FC01808182958F7008958F929F92AF925A
:10C2A000BF92CF92DF92EF92FF920F931F93DF9393
:10C2B000CF930F92CDB7DEB78C015B01FC0180817B
:10C2C00090E0FC01EE0FFF1FE80FF91FED51F74F53
:10C2D00080812181922F9F70F80121813281821B00
:10C2E000930BE42EF52E8E159F0508F47C01670153
:10C2F0004E010894811C911C25C0F80163816623BE
:10C3000021F184818F5F848370E0B4E0660F771F32
:10C31000BA95E1F7680F711DC40141E050E00E9439
:10C32000A6768981F50181935F01F80184818F30C0
:10C3300030F0148283810E94825FF8018383089425
:10C34000C108D108C114D104C1F6F80181819281DC
:10C350008E0D9F1D8C199D09928381838E2D8C19C2
:10C360000F90CF91DF911F910F91FF90EF90DF9091
:10C37000CF90BF90AF909F908F9008958F929F9293
:10C38000AF92BF92DF92EF92FF920F931F93CF93E2
:10C39000DF938C015B017A01C0E0D0E045E0842EA0
:10C3A000912C880E991E3BC0F801858190E08F7713
:10C3B0009070009741F4C801B40141E050E00E9440
:10C3C0004D61813079F5F80145813FE7D32ED422C4
:10C3D0002D2D30E0C7018C1B9D0B8217930710F4A5
:10C3E000DE2CDC1AB5016C0F7D1F47FF08C0CB01A6
:10C3F00060E070E04D2D50E00E949F760AC0C801B9
:10C400004D2D50E00E944D618D1519F0C80FD11DC2
:10C4100009C0CD0DD11DF80185818D198583CE15FB
:10C42000DF0510F2CE01DF91CF911F910F91FF90A8
:10C43000EF90DF90BF90AF909F908F9008959F9264
:10C44000AF92BF92CF92DF92EF92FF920F931F9322
:10C45000CF93DF93EC018B01C42E8B81882389F469
:10C4600089819A81009769F4E880FF240E94DC5F4B
:10C470008B83F701EE0FFF1FEE0DFF1DE252F74F0A
:10C480008483DC2C6FE0962E44C0EF80F8840E94F9
:10C49000D40EE81AF90AF7FE02C082E004C08B81CC
:10C4A000882319F481E08E8337C09C819F3080F00F
:10C4B0001C820E94825F882339F4EB800E94DC5F3B
:10C4C000682F8E2D0E94995F8B810E94825F8B83E3
:10C4D0008B81882339F36C81992D961BED2C9D154A
:10C4E00008F4E92EAE2CBB2470E06F5F7F4F90E024
:10C4F00054E0880F991F5A95E1F7680F791FC8011A
:10C50000A5010E94C5670A0D1B1D8C818E0D8C83B1
:10C51000DE18DD2009F0B9CF2C2D30E02D193109BE
:10C5200089819A81820F931F9A8389838C2D8D191B
:10C53000DF91CF911F910F91FF90EF90DF90CF90FF
:10C54000BF90AF909F9008950F931F93CF93DF9369
:10C55000EC01890168831A82198270E0CB01880F8F
:10C56000991F860F971FFC01E252F74F24812B83FE
:10C570001C821D821E82FC01ED51F74F10824295F4
:10C58000407F41830E94D40E080F191F18870F8324
:10C59000DF91CF911F910F9108951F93CF93DF9358
:10C5A000EC01888190E0FC01EE0FFF1FE80FF91FFE
:10C5B000ED51F74F898180839A819F708181807FBF
:10C5C000892B81838B81882389F00E94825F182FB9
:10C5D000882361F08B8160E00E94995F0E94B05FC8
:10C5E000112331F0812F0E94C25F02C010E0F6CF0C
:10C5F000DF91CF911F9108954F925F926F927F923A
:10C600009F92AF92BF92CF92DF92EF92FF920F93E1
:10C610001F93DF93CF930F92CDB7DEB75C01290153
:10C6200068012E2D30E00E94A4621982720100E0A0
:10C6300010E081E03E010894611C711CF7019191AA
:10C640007F01992341F4882349F49081992349F487
:10C65000992493941EC0882371F403C09924939461
:10C6600001C0992499819F3718F40C151D0561F5B7
:10C67000882379F001C099248981882321F1806879
:10C680008983C501B30141E00E941F628130D1F06E
:10C6900025C089818823B9F0C501B30141E00E941A
:10C6A0001F628130D9F44981B801641B7109640D9E
:10C6B000751DC5010E941F629981891719F0981B89
:10C6C00099830CC01982892D99819F5F99830F5F8F
:10C6D0001F4FC016D10608F0B1CF05C089818F77F2
:10C6E0006801C81AD108C5010E94CD62C6010F9029
:10C6F000CF91DF911F910F91FF90EF90DF90CF903E
:10C70000BF90AF909F907F906F905F904F900895F3
:10C7100080E094E0EEE9F9E0DF019C011D922150F8
:10C720003040E1F708950F931F93CF93DF93DA0121
:10C730001196FA014491ED012196FD01A491B0E01A
:10C74000179613E0B595A7951A95E1F71A2FDE0114
:10C750001196FE019491929FE0011124AC0FBD1F30
:10C7600000FD08C001FF08C09091CE0D51E096FD7C
:10C7700004C002C051E001C050E066956695669520
:10C7800070E09B013695322F22273795279590E050
:10C79000280F391F610F711D7695762F66277795C3
:10C7A0006795680F791F042F10E014C0E901C25685
:10C7B000D64F80E090E008C0FD01E80FF91FE4913A
:10C7C0005111E095E99301968417B0F3A00FB11FC2
:10C7D00020583F4F2617370749F7DF91CF911F9118
:10C7E0000F910895FF920F931F93CF93DF93942F90
:10C7F00046313CF4440F490F440F22FFABC0440FB5
:10C80000A9C0482F4A5F092F112707FD109520FD69
:10C8100009C021FF0AC03091CE0DFF24F39436FDEC
:10C8200005C003C0FF24F39401C0FF2466956695FC
:10C83000669570E07695762F662777956795680FF1
:10C84000711DEB01C256D64F22FF4FC09E3209F038
:10C850004A5FC801809760E170E00E94287680EA14
:10C8600090E0689F9001699F300D789F300D1124F2
:10C87000C801880F991F53E0000F111F5A95E1F767
:10C88000800F911F280F391F2D5B3D4E85E08823B7
:10C8900069F0F9019491E056FF4F54912F5F3F4F9B
:10C8A000F9016491E056FF4F749104C060E050E0DC
:10C8B00090E070E0FF2021F0909560955095709584
:10C8C000DE01AF57BF4FFDE0AE39BF0740F498839C
:10C8D0006983FE01E058FF4F50837C93229681507C
:10C8E0008F3FC1F12F5F3F4FD2CF23FF0DC0FF20FD
:10C8F00011F08FEF01C080E06256764FFB0180831C
:10C9000021964F5F91E001C090E09801220F331F04
:10C91000220F331F200F311F20503F4E85E0F901B9
:10C920002F5F3F4FE491992311F0843039F0FDE0FF
:10C93000CE39DF0718F4F110E095E993815079F7CB
:10C940005DE0CE39D50730F4FF2011F08FEF01C044
:10C9500080E08883842FDF91CF911F910F91FF900A
:10C96000089520E00E94F2630895CF92DF92EF9243
:10C97000FF920F931F93CF93DF93162FF22EF0E1C8
:10C98000EF2EE022C42EE6016E01D52EE6010CC08A
:10C99000EE2011F0488102C0FE014491612F202F4A
:10C9A0000E94F263FA942196FF2091F7DF91CF91D4
:10C9B0001F910F91FF90EF90DF90CF9008950F930C
:10C9C00000E00E94B5640F910895CF92DF92FF922C
:10C9D0000F931F93CF93DF93162F022FA0E1FA2E10
:10C9E000F222C42EE6016E01D52EE601FF2011F0E1
:10C9F000488102C0FE0144912196442329F0612F11
:10CA0000202F0E94F263F2CFDF91CF911F910F91FF
:10CA1000FF90DF90CF900895982FAB0180E0692FB1
:10CA200020E00E94E564089520E00E94E5640895F6
:10CA3000EF92FF920F931F93DF93CF930F92CDB797
:10CA4000DEB7182F062F7A01982F9C5E95504E2D39
:10CA50004F704A301CF0495C28E002C0405D20E085
:10CA6000892F602F99830E94F2639981911731F089
:10CA7000B4E0F694E794BA95E1F7E8CF0F90CF9140
:10CA8000DF911F910F91FF90EF900895E62FE695AB
:10CA9000E695E695F0E0F695FE2FEE27F795E795FB
:10CAA000E80FF11DE256F64F8DE0EE39F80758F425
:10CAB000677081E090E002C0880F991F6A95E2F7E5
:10CAC000208128272083089547FF02C0840F4195C5
:10CAD000E62FE695E695E695F0E0F695FE2FEE2733
:10CAE000F795E795E80FF11DE256F64F6770A1E064
:10CAF000B0E001C0AA0F6A95EAF711C08DE0EE39E7
:10CB0000F80778F4822F90E09C013595279580FFF7
:10CB100004C080818A278083206841503196442355
:10CB200069F708952FEF0E94646508950F931F938E
:10CB3000CF93DF93C82FD0E0E62FE695E695E695F4
:10CB4000F0E0F695FE2FEE27F795E795EC0FFD1F29
:10CB5000E256F64F062F10E0242F332727FD30959D
:10CB6000200F311FC90168E070E00E942876769599
:10CB7000762F6627779567956C0F7D1F6256764FE7
:10CB80000770107081E090E002C0880F991F0A952D
:10CB9000E2F781959081892708C0E058FF4F8DE02A
:10CBA000EE39F807D0F4808180958083E617F70787
:10CBB000A0F38DE0EE39F80780F4C90168E070E079
:10CBC0000E94287621E030E002C0220F331F8A95B0
:10CBD000E2F72195808182278083DF91CF911F9199
:10CBE0000F9108952F923F924F925F926F927F9292
:10CBF0008F929F92AF92BF92CF92DF92EF92FF926D
:10CC00000F931F93DF93CF9300D00F92CDB7DEB772
:10CC1000182F662E59016A01F02E802F05FF04C0DF
:10CC200004FF04C002E003C000E001C001E0E7FE31
:10CC300004C0E1942224239401C02224D7FE0BC017
:10CC4000D094C094B094A094A11CB11CC11CD11C60
:10CC50004424439401C0442482FF06C09CE0909386
:10CC60009E0D3AE0932E05C096E090939E0D25E030
:10CC7000922E86FF2FC04110190D28EEA21623E038
:10CC8000B20620E0C20620E0D20614F0190D06C05C
:10CC900034E6A316B104C104D10414F0190D06C082
:10CCA0008AE0A816B104C104D1040CF0190D0023C8
:10CCB00091F0023039F4E4E6AE16B104C104D104B7
:10CCC00054F4190DFAE0AF16B104C104D1041CF4F8
:10CCD000190D01C0191B80919E0D810F80939E0D2F
:10CCE000023011F420EFF20E5524539492E0792E85
:10CCF00088242E2D332727FD3095862D8A5F898342
:10CD00003B832A8370C0C601B5012AE030E040E0D1
:10CD100050E00E945D76E62E80E3382E3E0C812F97
:10CD2000662D432D2F2D0E94F2630515D9F5F2FED5
:10CD300023C08E2D8150833008F47394C601B50151
:10CD40002AE030E040E050E00E945D76CA01B9017F
:10CD50002AE030E040E050E00E945D76623011F061
:10CD60006430C1F4E32DE43319F4812E839413C0AD
:10CD7000812E8A9473940FC01250812F8F5FF0FE22
:10CD800005C0662D47E00E94966505C069810E9436
:10CD9000466501C0812EFAE0AF16B104C104D1048A
:10CDA0000CF000E0C601B5012AE030E040E050E0C0
:10CDB0000E945D7659016A01211531054105510531
:10CDC00081F4002331F0023059F4252D223040F453
:10CDD00008C0F4FE10C0222021F430EFF30E01C091
:10CDE00000E019195394852D90E0EA81FB81E81742
:10CDF000F9070CF088CF882061F0662D645F882DDC
:10CE0000472D0E949265662D635F882D472D0E94F5
:10CE10009265442039F0812F8919662D4DE22F2D1E
:10CE20000E94F2630F900F900F90CF91DF911F91AE
:10CE30000F91FF90EF90DF90CF90BF90AF909F90B9
:10CE40008F907F906F905F904F903F902F900895BC
:10CE5000EF920F93022FFA019F01442737FD40956F
:10CE6000542F75E0E72E0E94F2650F91EF90089520
:10CE700020E00E9428670895A998AB98AC988BBBD6
:10CE8000AD9AAD98AB9AA99A089520E030E006C01B
:10CE900045E04A95F1F700002F5F3F4F281739070B
:10CEA000BCF30895AA9885E08A95F1F7000085E023
:10CEB0008A95F1F70000AA9A8CED95E00E944567EB
:10CEC00082EE0E943C678EEA0E943C6781EA0E94E3
:10CED0003C6786EA0E943C6784EA0E943C6782EADB
:10CEE0000E943C6780EC0E943C678FE20E943C6796
:10CEF00085E20E943C6781E80E943C6782E20E94D2
:10CF00003C678FEA0E943C6782E280935801089553
:10CF10001F93182F81E80E943C67812F0E943C6775
:10CF20001F9108951F93CF93DF9310E0CEE9D9E0CE
:10CF300084E00E943C6780E10E943C67812F806B07
:10CF40000E943C67A998AB9AAC98FE0180E2908160
:10CF50009BBBAD9AAD9891819BBBAD9AAD989281E8
:10CF60009BBBAD9AAD9893819BBB3496AD9AAD981F
:10CF7000815069F7C058DF4FAB9AA99A1F5F1830EC
:10CF8000B9F6DF91CF911F910895BF92CF92DF92B2
:10CF9000EF92FF920F931F93CF93DF93EA01E82E56
:10CFA000F92E062F172F21C0F701B1907F016801DC
:10CFB0000894C11CD11C04C0009739F00E94B81914
:10CFC0008091DA0890E082709070E199F5CF1FBBF4
:10CFD0000EBBE09A8DB3B81631F0BDBA8FB7F89496
:10CFE000E29AE19A8FBF219786012097E9F6DF91B7
:10CFF000CF911F910F91FF90EF90DF90CF90BF9056
:10D0000008958093CF0D08958091CF0D1092CF0D8C
:10D010000895FC018081982F990F9E70807F892B45
:10D020008083662321F09160807F892B80838181BA
:10D030008F5F81839281992391F020812F7079F401
:10D04000933659F0242F20622093CF0D903111F4A4
:10D05000803118F080818F7C8083118212828281DE
:10D06000883009F443C0893058F4813009F446C04F
:10D070008130A0F08230D1F1843009F052C036C046
:10D080008F3549F1803620F4803109F04AC02EC036
:10D09000813689F0823609F044C03DC08081982FE6
:10D0A0009F709F30F1F591E6928391819131E0F08C
:10D0B0008F7C808319C040664093CF0D9081892F6B
:10D0C00082958F708F5F83708295807F9F7C982B75
:10D0D00090838FE508C08181883111F4406818C0C1
:10D0E0008832F9F480E1828311820895918190332E
:10D0F00028F090E09595879582831182828190E057
:10D100000197218130E082239323009751F44064FA
:10D110004093CF0D08958181803418F088E0828398
:10D12000118208958E3091056CF4FC01EE0FFF1F03
:10D13000E80FF91FEE55F24F90819F7081E09F300C
:10D14000E9F53FC0823131F1833160F48F30C9F0AD
:10D15000803118F48E3091F52AC0803161F0813130
:10D1600069F513C0843151F08431D0F08531E1F09C
:10D17000863121F51EC091B194701DC093B3907893
:10D180001AC090916300917016C0909163009095C1
:10D19000987011C08091630083FF12C091B102C0EA
:10D1A00091B19095907407C091B1907104C093B300
:10D1B000F9CF91B1907281E0992319F480E008953C
:10D1C00080E008958F708E3058F490E0FC01EE0FEF
:10D1D000FF1FE80FF91FEE55F24F82E6828311829E
:10D1E00008958F708E3068F490E0FC01EE0FFF1F01
:10D1F000E80FF91FEE55F24F83E6828380818F7C22
:10D20000808308950F931F93CF93DF938091CC0D6C
:10D210009091CD0D01969093CD0D8093CC0D809182
:10D22000CE0D8F5F8093CE0D06B3009540E050E0A9
:10D2300010E001C0AE01EA012196CA01880F991FD2
:10D24000840F951FB8010C2E02C0759567950A943E
:10D25000E2F7617070708E55924F50E00E9409683D
:10D26000C630D10539F700B30095C0E0D0E0FE012B
:10D27000ED5FF44EE4919E012A5F3F4FC901880F94
:10D28000991F820F931F8E55924FE02361E009F49E
:10D2900060E09E012A5F422F50E00E9409682196BB
:10D2A000C830D10521F7DF91CF911F910F910895DB
:10D2B000FF920F931F93CF93DF93F82EE4EAF1E0F0
:10D2C00080E090E0582F9C014081F41638F0442310
:10D2D00029F001963A9681329105A1F75032B9F1C1
:10D2E000E901CC0FDD1FC901A3E0880F991FAA95A2
:10D2F000E1F7C80FD91F8E010C551E4FA9014F5FD2
:10D300005F4FCA01880F991FE3E0440F551FEA954C
:10D31000E1F7840F951F20953095205E3F4FA901BE
:10D32000440F551F63E0220F331F6A95E1F7420F48
:10D33000531F8C559E4FB8010E948D768AE0D8010C
:10D340001D928A95E9F7C657DE4FFA8E02C004EAAD
:10D3500011E0C801DF91CF911F910F91FF900895C7
:10D3600080E491E0E4EAF1E0DF019C011D922150AC
:10D370003040E1F70895E0916E01F0E0EE0FFF1FFD
:10D38000EE0FFF1FE80FF11DE151FB4F849108954F
:10D39000EF92FF920F931F93DF93CF9300D000D0B3
:10D3A000CDB7DEB719821A821B821C82E09173010D
:10D3B000F0E0E852FB4F26E030E091E0E491EE2E01
:10D3C000FF24DE0111960FC06F5F7F4F061717070E
:10D3D00011F4FA01908364307105B1F79F5F225018
:10D3E0003040953089F060E070E0A701022E02C065
:10D3F000559547950A94E2F7437050708A010F5F84
:10D400001F4F4A0F5B1FE0CF882361F50E94B06970
:10D4100089810E9458698C0181E00E94BB69F801F2
:10D42000818324E6F22EF2828A810E9458698C015F
:10D4300082E00E94BB69F8018183F2828B810E94A5
:10D4400058698C0183E00E94BB69F8018183F282F4
:10D450008C810E9458698C0184E00E94BB69F801AC
:10D460008183F2820F900F900F900F90CF91DF91F8
:10D470001F910F91FF90EF9008956F927F928F927E
:10D480009F92AF92BF92CF92DF92EF92FF920F9353
:10D490001F93CF93DF938091A00181FF03C060E0D1
:10D4A00075E002C060E074E090919D0184E698020E
:10D4B000C0011124885A9D4FE091A301FF27E7FD89
:10D4C000F09548EE53E0E49F9001E59F300DF49F06
:10D4D000300D112428533045AA24BB24A81AB90AB8
:10D4E000281B390BFBE0EF2EF5E0FF2E40919A014F
:10D4F000440F485F50E0440F551F440F551F4053E1
:10D50000524FE0EDFDE0CC24DD24C61AD70AA8E591
:10D51000B2E0A81BB90B1CC0E701699079907E01AD
:10D520004B01661677060CF4430184018C149D04AC
:10D530000CF48601005A164FE501C01BD10B2C0FCD
:10D540003D1F0A0F1B1F1183008393838283349630
:10D55000E417F50709F731832083938382831582CB
:10D560001482DF91CF911F910F91FF90EF90DF9088
:10D57000CF90BF90AF909F908F907F906F900895C5
:10D58000E0911201F09113018193F0931301E09364
:10D5900012010895FF920F931F93CF93DF93B9E089
:10D5A000FB2E90E120E0C82FD0E08E0101701070BA
:10D5B000201711F4905F07C0892F90E001970E9417
:10D5C000C06A202F90E1FA9431F0D595C795AE014D
:10D5D0004068842FE8CF892F90E00F960E94C06AA0
:10D5E000DF91CF911F910F91FF9008951F93CF93DB
:10D5F000DF93182F20ED3DE03093130120931201AB
:10D6000080911801877471F080919A01882319F034
:10D61000813029F402C080E803C080E901C088E9B4
:10D62000809318018091180187FF0BC086E190E07C
:10D630000E949268882329F4809118018F77809343
:10D6400018018091180187FD5AC085E160E040E033
:10D650000E944311882309F452C08091180180620E
:10D6600080931801809157018F5F80931901EAE13F
:10D67000F1E0ABE0B5E080E01CC02D913D91359527
:10D68000279520503E4F37FD05C093E02F3F3907C7
:10D6900024F405C020E030E002C02FEF33E0932FE8
:10D6A0009370482F440F440F942B908321838F5FF6
:10D6B0003296811711F7C8E1D1E089910E94CA6AB8
:10D6C00081E0C632D807C9F7809112019091130109
:10D6D000019790931301809312018FEF90E00E94C5
:10D6E000C06A80E090E00E94C06A80ED9DE0909367
:10D6F000170180931601DF91CF911F9108958091BA
:10D7000018018F7DADCF1F920F920FB60F9211248B
:10D710002F938F939F93EF93FF9388B391E0892783
:10D7200088BBE0911601F09117012191F093170148
:10D73000E0931601822F90E097BD86BD293C08F04A
:10D74000C09A8091600E81608093600EFF91EF918E
:10D750009F918F912F910F900FBE0F901F90189552
:10D760001F920F920FB60F9211242F933F938F9316
:10D770009F93EF93FF9388B391E0892788BBE09153
:10D780001201F0911301208130E020FD04C088B522
:10D7900099B5809603C088B599B5409699BD88BD66
:10D7A000C90195958795009791F4CF0101969093C3
:10D7B0001301809312018181882351F480917800B4
:10D7C000909179008053984F99BD88BD01C08083A6
:10D7D0008091600E81608093600EFF91EF919F9128
:10D7E0008F913F912F910F900FBE0F901F90189522
:10D7F000EDE7F0E08081857E808317981F9AAAE884
:10D80000B0E01C9210928B0082E88C938081806241
:10D8100080830895EDE7F0E080818F7D8083179A03
:10D82000AAE8B0E01C9210928B008AE08C93808171
:10D830008861808308951F920F920FB60F92112472
:10D840008F939F93AF93BF93EF93FF9380916C0E51
:10D85000882321F01F9A10926C0E04C01F9881E05B
:10D8600080936C0EA0911401B0911501FD0181917E
:10D8700091919093870080938600F0931501E09337
:10D8800014018091630E9091640E909385008093B3
:10D89000840012968D919C911397009759F488E11A
:10D8A0009EE090931501809314018091A0018170F6
:10D8B00080936C0E8091600E81608093600EFF916A
:10D8C000EF91BF91AF919F918F910F900FBE0F90ED
:10D8D0001F901895AF92BF92CF92DF92EF92FF9276
:10D8E0000F931F93CF93DF938091A00181FF03C01B
:10D8F00040E055E002C040E054E0F0909A01FF0C97
:10D9000080E1F80E20919D0184E628029001112407
:10D91000285A3D4FE091A301FF27E7FDF09568EEFF
:10D9200073E0E69FC001E79F900DF69F900D1124D4
:10D9300088539045CC24DD24C21AD30A821B930B52
:10D9400068EFE62EEF0CE8E1FEE000271127041B4C
:10D95000150B68E572E0621B730B21C0AE2DB0E0C1
:10D96000AA0FBB1FA55FBA4FAC901196BC90D50112
:10D970004A175B070CF4DA01A017B1070CF4D801C1
:10D98000A05AB64FE601CA1BDB0B8C0F9D1F3183DB
:10D990002083A60FB71FB383A2833496E394EF14BA
:10D9A000E8F23183208393838283885E934090934F
:10D9B000640E8093630E15821482DF91CF911F91C4
:10D9C0000F91FF90EF90DF90CF90BF90AF900895B0
:10D9D0001F920F920FB60F9211242F933F934F93E4
:10D9E0005F936F937F938F939F93AF93BF93EF93C7
:10D9F000FF9378940E946A6CFF91EF91BF91AF9171
:10DA00009F918F917F916F915F914F913F912F9156
:10DA10000F900FBE0F901F9018952091690E3091B6
:10DA20006A0E90E0822793279070880F991F855F78
:10DA3000944EFC0145915491232F332742275327BD
:10DA400050936A0E4093690E08959091650E9695D5
:10DA50009695982B9093650E8091660E8F5F8093BC
:10DA6000660E843068F0E091670EF091680E919335
:10DA7000F093680EE093670E1092650E1092660E9A
:10DA8000089503C080E00E94256D8091660E882372
:10DA9000C9F7E091670EF091680E1082089588230F
:10DAA00039F080916B0E8F5F80936B0E80E803C01E
:10DAB00010926B0E80EC0E94256D80916B0E85306C
:10DAC000B8F708950F931F93182F0E940D6D08E06B
:10DAD000812F81700E944F6D16950150C9F71F91DB
:10DAE0000F91089580EC0E94256D80E80E94256DBD
:10DAF00080E80E94256D80E80E94256D80E80E94E4
:10DB0000256D80E80E94256D80E80E94256D80ECDF
:10DB10000E94256D0895AF92BF92CF92DF92EF924F
:10DB2000FF920F931F93CF93DF9380ED9DE090932F
:10DB30001301809312019093680E8093670E1092E8
:10DB40006A0E1092690E1092650E1092660E109277
:10DB50006B0E0E94726D80919A010E94626D80919D
:10DB6000620E0E94626D80E00E94626D1092620EF1
:10DB70000BE015E054E0C52ED12CF8012081318155
:10DB8000C901880F991F820F931FB6010E94287642
:10DB9000EB0122813381C901880F991F820F931FE6
:10DBA000B6010E94287660507C4FC050DC4FF8E0F0
:10DBB000C030DF0710F0CFEFD7E07B0128E0603006
:10DBC000720720F0AFEFEA2EA7E0FA2E8C2F0E940A
:10DBD000626D5E019B2D9F708E2D8295807F892BBB
:10DBE0000E94626DC701F4E096958795FA95E1F77A
:10DBF0000E94626D0C5F1F4F25E00B31120709F088
:10DC0000BCCF00916A0E8091690E0E94626D802FD8
:10DC10000E94626D0E94726D0E94416D8091780039
:10DC200090917900805C934690937900809378007E
:10DC3000C09ADF91CF911F910F91FF90EF90DF90ED
:10DC4000CF90BF90AF900895809199019091610E0F
:10DC5000981709F494C08093610E8130F9F08130F7
:10DC600030F08230F1F1833009F089C05EC00E944B
:10DC7000F86B1EBC80E49CE99BBD8ABD1DBC1CBC2E
:10DC800087B7837C87BF8CE386BF8FE380937C005C
:10DC900087B7806187BF1FBC8AE021C00E94F86BF4
:10DCA0001EBC1DBC1CBC80E797E199BD88BD80EA05
:10DCB0009FE0909379008093780087B7837C87BF3B
:10DCC0008CE386BF8FE380937C0087B7886087BF33
:10DCD00080917D00816080937D001FBC82E08EBDBD
:10DCE0004EC00E94F86B1EBC88EC90E090937900C7
:10DCF000809378008CE291E09DBD8CBD80EE9BEA24
:10DD000097BD86BD87B7837C87BF8CE386BF8FE3D3
:10DD100080937C0087B7806287BF80917D0081609F
:10DD200080937D001FBC8AE1DACF1EBC80E49CE9B1
:10DD30009BBD8ABD1DBC1CBC87B7837C87BF8091FF
:10DD40007D008E7F80937D008CE386BF8FE3809380
:10DD50007C0087B7806187BF1FBC8AE08EBD0E94B0
:10DD60006A6C80E593EC909387008093860088E846
:10DD700093E190938500809384000E940A6C8091C7
:10DD80009901813051F0813028F0823051F0833098
:10DD900079F40CC00E943D6A089578940E948B6DBE
:10DDA0000895789486E00E94F66A08950E943D6A7C
:10DDB00008951F920F920FB60F9211242F933F9345
:10DDC0004F935F936F937F938F939F93AF93BF9383
:10DDD000EF93FF93809199018230C1F480E492EA3D
:10DDE00097BD86BD80917800909179008F3F910515
:10DDF00038F488E598E9909379008093780008C01A
:10DE000088EC90E090937900809378000E94246ED3
:10DE1000FF91EF91BF91AF919F918F917F916F9102
:10DE20005F914F913F912F910F900FBE0F901F90D8
:10DE300018951F920F920FB60F9211242F933F93B4
:10DE40004F935F936F937F938F939F93AF93BF9302
:10DE5000EF93FF938CB59DB520916D0E222321F099
:10DE6000C09A10926D0E04C0C09821E020936D0EF0
:10DE7000A0912601B0912701FD01219131913BBD77
:10DE80002ABDF0932701E09326012091AB06309143
:10DE9000AC062817390720F49093AC068093AB06A4
:10DEA00020910C0130910D018217930720F490937B
:10DEB0000D0180930C0112968D919C911397009700
:10DEC000D9F480ED9DE09093270180932601809105
:10DED000A0018095817080936D0E87B78F7E87BF7C
:10DEE0000E94246E80919901882311F0833021F4DF
:10DEF00087B7806187BF78948091600E816080933E
:10DF0000600EFF91EF91BF91AF919F918F917F91A3
:10DF10006F915F914F913F912F910F900FBE0F9096
:10DF20001F90189590916D019873903121F463E0E2
:10DF30000E9408760895983111F4869508959832D4
:10DF400011F4880F0895903319F4982F990F890FC1
:10DF50000895FC01A5E6B0E08C918B7F8C93148230
:10DF600015821082118216A617A608950E94A96F25
:10DF7000089521E0FC018481882309F420E0822FA8
:10DF80000895FC0181819081891B877098E0981B1E
:10DF900081E0933008F480E00895FC0184818823B7
:10DFA000F9F08150848382819381890F828386A5D1
:10DFB000882309F44CC087A5982F915097A78823F0
:10DFC00031F08091650084608093650008958091B0
:10DFD00065008B7F809365008091780187A7089505
:10DFE0001B98809165008B7F8093650085818823D5
:10DFF00019F081508583089580819181891739F1C5
:10E0000090E0DF01A80FB91F16962C911697228376
:10E0100056962C91569724831E962C911E972383F7
:10E020005E962C915E972583D0962C91D09726A74B
:10E0300017A696962C919697322F315096963C9330
:10E040009697222321F4019687709070808308951B
:10E050008F929F92AF92BF92CF92EF92FF920F93C7
:10E060001F93DF93CF9300D0CDB7DEB74C01122FB3
:10E070004A8369830E94C16F4A816981882331F193
:10E0800080916D01887311F1F401A180BB24C50159
:10E09000019697E0F92EF8228081F816B9F06623F0
:10E0A00029F080917701865F860F01C080E0A80C7F
:10E0B000B91CF5018683842F0E94926FF501868B2F
:10E0C000168FE0AA06A3C686F401F1820F900F9086
:10E0D000CF91DF911F910F91FF90EF90CF90BF9064
:10E0E000AF909F908F900895AF92BF92CF92EF9292
:10E0F0000F93DF93CF9300D00F92CDB7DEB75C01C3
:10E100002B834A8369830E94C16F2B814A81698175
:10E11000882329F180916D01887309F1662329F024
:10E1200080917701865F860F01C080E0F5018283D0
:10E13000842F2B834A8369830E94926FF501848325
:10E140002B812583E6A617A6C382808181834A811D
:10E150006981002321F00150C5010E9428700F90B1
:10E160000F900F90CF91DF910F91EF90CF90BF90D4
:10E17000AF900895CF92EF920F93CF93DF93EC017E
:10E1800080916D0186958695869587702881998105
:10E19000291709F05CC1E62FF0E0E132F10508F043
:10E1A00056C1EA5BFF4FEE0FFF1F0590F491E02D83
:10E1B0000994CE0166E44AE0DEC0CE0166E444E1A3
:10E1C000DAC0CE0166E44EE1D6C0CE0164E64AE094
:10E1D00022E002E0EE24E39452E0C52E36C1CE01E7
:10E1E0006FE545E022E00AE0EE24E394CC240E94AF
:10E1F0002870CE016FE545E02AE001E00E9428701A
:10E20000CE016FE545E022E00AE01FC1CE0160E5E6
:10E210004AE023E002E0EE24CC24CA940E94287055
:10E22000CE016CE34AE023E0CC24C3940E94287022
:10E23000CE0166E44AE021E000E032E0E32E96C041
:10E24000CE0166E445E021E001E0EE24E394CC2435
:10E250000E942870CE0162E34FE022E00E94287005
:10E26000CE0160E54FE022E0F0C0CE016EE645E071
:10E2700021E002E0EE24E394CC240E942870CE0139
:10E280006CE745E021E02AC0CE0162E345E025E0ED
:10E2900000E0EE24CC240E942870CE016AE545E01F
:10E2A00025E00E942870CE016EE643E024E002E003
:10E2B000CCC0CE0160E545E02AE003E0EE24E39423
:10E2C000CC240E942870CE0160E545E024E101E005
:10E2D0000E942870CE0160E545E02AE003E0B5C069
:10E2E000CE016AE044E125E002E0EE24E394CC2490
:10E2F000C394ABC0CE0162E344E02AE002E0EE2426
:10E30000E394CC240E942870CE0166E448E024E126
:10E3100001E00E942870CE0162E348E02AE002E0BA
:10E320000E942870CE0166E444E024E101E08DC043
:10E33000CE0168E745E02AE00AE016C0CE0168E7B2
:10E3400045E022E30AC0CE0160E044E12AE001E0BA
:10E350000BC0CE0160E044E12AE002E005C0CE013E
:10E3600060E044E12AE003E0EE24E394CC246DC0B5
:10E37000CE0166E448E221E000E048C0813009F4C3
:10E3800066C0CE016BE405C0813009F460C0CE01E7
:10E3900061E44AE021E000E041C0CE01642F46E0A4
:10E3A000F9CFCE0166E44AE022E0E6CF813009F4FD
:10E3B0004EC0CE0166E44AE022E0EDCFCE0168E730
:10E3C000E8CFCE0168E74AE021E01FC0CE016AE74E
:10E3D0004AE021E00FC0CE016CE74AE021E004C032
:10E3E000CE0168E74FE023E003E010C0CE0168E70C
:10E3F0004FE023E002E00AC0CE0168E74FE023E0EF
:10E4000004C0CE0166E444E129E101E0EE24E39496
:10E4100006C0CE0166E44AE022E002E0EE24CC240D
:10E420000E94747014C0CE016CE344E123E002E06A
:10E43000EE24CC24C3940E942870CE0160E544E110
:10E4400023E0EE24E394CC24CA940E942870DF9148
:10E45000CF910F91EF90CF900895682F8FE294E0C5
:10E4600046E40E94BA70089590919601987109F05F
:10E470006AC09091C50E992321F48E3509F076C0BB
:10E4800002C08E3511F481E019C08D3521F481E090
:10E490008093C60E08952091C60E222321F010927B
:10E4A000C60E20E68227913021F48093C70E82E0C9
:10E4B00005C0923031F48093C80E83E08093C50E7E
:10E4C00008954091C70E4932D8F5382F20E0809149
:10E4D000C80EB901680F711DE42FF0E0EE0FFF1FA9
:10E4E000E753F14F71836083413149F420911B0F51
:10E4F00030E02617370724F560931B0F21C0463004
:10E50000F9F48091D50E9091D60E592F52955F70E7
:10E51000E52FF0E02091280F30E0E217F3074CF0F0
:10E52000E530F1051CF04093280F03C05F5F509366
:10E53000280FE45EF04F6AE070E00E942876608366
:10E540001092C50E0895983089F49091970E9233E9
:10E5500018F48093C80E0895382F20E08091C80EDB
:10E56000280F311D3093EA0E2093E90E08951F9273
:10E570000F920FB60F9211242F938F939F93EF93C7
:10E58000FF938091940E882379F09091290FE92FC1
:10E59000F0E0EF57F14F20812CB99F5F9093290F46
:10E5A00081508093940E01C05598FF91EF919F91F7
:10E5B0008F912F910F900FBE0F901F901895109272
:10E5C000290F559A0895CF92DF92EF92FF920F9301
:10E5D0001F93CF93DF9390E09C01220F331F220FF4
:10E5E000331FD901A85DBB4F40E050E0C62EDD24AB
:10E5F000F901E65DFB4F89010756114FC416D50698
:10E6000011F0623020F18081282F2F7030E07A01E4
:10E61000EE0CFF1C02C035952795EA94E2F72370B3
:10E6200030702115310599F0E801E8807C918295E0
:10E63000837090E0042E02C0959587950A94E2F7C6
:10E6400080FF03C07E1518F40AC0E71640F04F5F44
:10E650005F4F11964230510589F620E030E0C90144
:10E66000DF91CF911F910F91FF90EF90DF90CF90AE
:10E670000895E82FF0E0EE0FFF1FEE0FFF1FE65D9D
:10E68000FB4F80818F70909179019150923038F5D5
:10E690009091700197FF23C090E0660F02C095959E
:10E6A00087956A95E2F78370823039F0833079F08C
:10E6B0008130A9F46091750103C060917501629584
:10E6C0006F708FE294E046E40E94BA700895609102
:10E6D00076016F708FE294E046E40E94BA7008956C
:10E6E0001092940E8AB188628AB90895549A579A02
:10E6F0000895FC016E3721F06D3761F46DE501C0BE
:10E700006EE58081A82FB0E0AF57B14F9DE79C9395
:10E710008F5F80838081A82FB0E0AF57B14F6C939B
:10E720008F5F808308951F93DF93CF9300D00F9264
:10E73000CDB7DEB71EE71093810E8093820E82E084
:10E740008983CE0101962B834A830E947973898144
:10E75000A82FB0E0AF57B14FFD014A8141932B8103
:10E7600011962C93DF0111961182FD0131961196BD
:10E770001C92DF0111961182FD01319611961C92B7
:10E78000119711821283885F8093940E0F900F90DF
:10E790000F90CF91DF911F910895FC0180818383B9
:10E7A00010820895FC018381861710F4681B01C054
:10E7B00060E060838281861708F462838181882308
:10E7C00011F0681708F461830895FF920F931F9367
:10E7D000CF93DF93EC0188818D3F40F4893F60F453
:10E7E000863FD1F1873F09F04DC02FC08D3FD9F151
:10E7F0008E3F09F047C013C090E0895F9040FC0154
:10E80000EE0FFF1FE80FF91FE754F14F8981828354
:10E810008A81817081838B818370808333C089E991
:10E820009EE069810E94D2738DE99EE06A810E9418
:10E83000D27381EA9EE06B810E94D2736C816695EF
:10E8400085EA9EE00E94D2731DC089818093B60E36
:10E850008B818093B80E16C089818093B50E8B8111
:10E860008093B70E0FC009810D5F239613E0BCE3C0
:10E87000FB2E06C089910E943472F092970E1F5FA2
:10E880001017C0F31092950E84E18093960EDF91DD
:10E89000CF911F910F91FF9008951F920F920FB685
:10E8A0000F9211242F933F934F935F936F937F9316
:10E8B0008F939F93AF93BF93EF93FF935798789461
:10E8C0009BB18CB19C7129F01092950E10922E0F75
:10E8D0004BC09091950E992309F046C090912D0F51
:10E8E000913039F09130C8F1923079F09330E1F500
:10E8F00024C08E37C9F190912E0F933160F5E92F26
:10E90000F0E0E259F14F808323C08D3711F483E0AA
:10E9100029C08E3739F48EE69EE00E94E57310928E
:10E920002D0F22C090912E0FE92FF0E0E259F14F08
:10E9300080839F5F90932E0F17C090912E0F93317D
:10E9400050F4E92FF0E0E259F14F20E2282720832C
:10E950009F5F90932E0F82E005C08E3729F41092AE
:10E960002E0F81E080932D0FF894579AFF91EF912D
:10E97000BF91AF919F918F917F916F915F914F91D7
:10E980003F912F910F900FBE0F901F90189580E12F
:10E99000E9E9FEE0DF011D928A95E9F71092AE0EDB
:10E9A0001092AD0E1092B40E1092B30E08958CE03A
:10E9B000E9EBFEE0DF011D928A95E9F70E94C7743A
:10E9C000109818981092900087E689B959981AB84B
:10E9D00086E08093950001C08CB15F99FDCF0E94C5
:10E9E00070730E9476730895FC0182819381860F73
:10E9F000911D93838283208131812817390748F440
:10EA0000821B930B938382838481958101969583E6
:10EA1000848308958091960E882319F08150809305
:10EA2000960E8091970E882319F081508093970E4F
:10EA300090912A0F992309F471C080912B0F88239C
:10EA400021F0815080932B0F69C08091940E882310
:10EA500009F064C0E0E081E0282F292321F4EF5F72
:10EA6000880FE730C9F78095892380932A0FE43017
:10EA7000C0F58E2F87509E2F969521E0291B30E000
:10EA8000F0E0E095F095E170F070D901AA0FBB1F9E
:10EA9000AA0FBB1FAE0FBF1FA85DBB4F6C91D90162
:10EAA000AA0FBB1FAA0FBB1FA65DBB4F2C91422F05
:10EAB0004295437050E00E2E02C0559547950A943A
:10EAC000E2F741709091700197FD20C02F7030E007
:10EAD000EE0FFF1F02C035952795EA95E2F72370E8
:10EAE00016C0E63070F48E2F8170E82FF0E0DF0161
:10EAF000AB54B14FE954F14F8A506C9140E0208102
:10EB000006C0E63059F481EF60E040E020E00E946A
:10EB1000937385E080932B0F0E94DF7280912A040B
:10EB20008295869586958370833031F489EA9EE0DC
:10EB30006091990E0E94F47480912E0482958695BE
:10EB400086958370833031F48FEA9EE060919D0E4C
:10EB50000E94F474809128018150809328018823B9
:10EB600031F488EC8093280181E08093980E089519
:10EB7000EF92FF920F931F931092280F80912A0F0C
:10EB80008F6080932A0F2091270430E040E050E00E
:10EB900060E4E62E6EE7F62E65E0062F112DC80123
:10EBA000B7010E945D763093AA0E2093A90E2091A2
:10EBB0002B0430E040E050E0C801B7010E945D76D0
:10EBC0003093B00E2093AF0E1F910F91FF90EF90F6
:10EBD0000895629FD001739FF001829FE00DF11DA7
:10EBE000649FE00DF11D929FF00D839FF00D749FC7
:10EBF000F00D659FF00D9927729FB00DE11DF91F73
:10EC0000639FB00DE11DF91FBD01CF0111240895CF
:10EC1000991B79E004C0991F961708F0961B881F6E
:10EC20007A95C9F780950895AA1BBB1B51E107C0CF
:10EC3000AA1FBB1FA617B70710F0A61BB70B881F8C
:10EC4000991F5A95A9F780959095BC01CD0108951B
:10EC500097FB092E07260AD077FD04D0E5DF06D002
:10EC600000201AF4709561957F4F0895F6F79095FE
:10EC700081959F4F0895A1E21A2EAA1BBB1BFD018F
:10EC80000DC0AA1FBB1FEE1FFF1FA217B307E4078B
:10EC9000F50720F0A21BB30BE40BF50B661F771FE3
:10ECA000881F991F1A9469F76095709580959095C3
:10ECB0009B01AC01BD01CF01089597FB092E0526EC
:10ECC0000ED057FD04D0D7DF0AD0001C38F4509581
:10ECD0004095309521953F4F4F4F5F4F0895F6F780
:10ECE00090958095709561957F4F8F4F9F4F0895B8
:10ECF000EE0FFF1F0590F491E02D0994FB01DC015C
:10ED00004150504048F005900D920020C9F701C0D5
:10ED10001D9241505040E0F708956817790768F454
:10ED2000FB01DC01E40FF51FA40FB51F02C0029028
:10ED30000E9241505040D8F708950C94B676DC01FD
:10ED400001C06D9341505040E0F70895DC01CB01C4
:10ED5000FC01E199FECF06C0FFBBEEBBE09A319605
:10ED60000DB20D9241505040B8F70895FB01DC01FF
:10ED700002C001900D9241505040D8F70895F89488
:02ED8000FFCFC3
:10ED82006C036D036E036F034AF0004DFF0722040C
:10ED92007C5ED00D180ED00DFF0000AA05FF09FF02
:0AEDA2000DFF135414AAD00DC80091
:00000001FF
